:020000040800F2
:108000000080012069790108191001081B1001087E
:108010001D1001081F1001082110010800000000B8
:108020000000000000000000000000002310010814
:10803000251001080000000027100108DD8100085C
:10804000AD790108AD790108AD790108AD79010874
:10805000AD790108AD790108AD790108AD79010864
:10806000AD790108AD790108AD790108AD79010854
:10807000AD790108AD790108AD790108AD79010844
:10808000AD790108AD790108AD7901089990000832
:10809000218F0008DD8F0008AD7901089D8B000855
:1080A000AD790108AD790108AD790108AD79010814
:1080B00061F20008AD790108AD790108AD790108D8
:1080C000AD790108AD790108AD790108E5F1000845
:1080D000AD790108AD790108B18D0008AD790108CD
:1080E000AD790108AD790108AD790108AD790108D4
:1080F000AD790108AD7901089D000108AD7901084D
:10810000AD790108AD790108AD790108AD790108B3
:10811000AD790108AD790108AD790108AD790108A3
:10812000AD790108AD790108AD790108AD79010893
:10813000AD790108AD790108AD790108AD79010883
:10814000AD790108AD790108AD790108B1AA00083F
:10815000AD790108AD790108AD790108AD79010863
:10816000AD790108AD790108AD790108AD79010853
:10817000AD790108AD790108AD790108AD79010843
:04818000AD790108CC
:1081880010B5054C237833B9044810B10448AFF34F
:1081980000800121217010BD0806002000000000A9
:1081A8009C9A010808B5064B1BB106480649AFF36F
:1081B80000800648016811B1054B03B1984708BD16
:1081C800000000009C9A01080C060020040600200C
:1081D80000000000684620F007018D4601B5124BEB
:1081E8001A787AB15A6801325A60104B1A6801320B
:1081F8001A600F4B1A6812B11A68013A1A60002205
:10820800094B00E001221A700A4B1A683AB11A6841
:10821800013A1A601B6813B9074B01221A70BDE8AE
:1082280001408546704700BF2406002050540020B6
:10823800FC4B0020004C0020044C0020074B41F66A
:108248004B525A60064AF02182F8231000229A60A5
:108258006FF0040007221A600BF0B6BB10E000E0D4
:1082680000ED00E0014B5868704700BF240600206D
:108278002DE9F341664F01200146002402250AF04A
:1082880021F9092338466946012600938DF80440F0
:108298008DF806408DF807408DF8055009F05AFF13
:1082A80048F216033846694600938DF806408DF863
:1082B80007408DF804608DF8055009F04BFF48F22F
:1082C80015033B8338467D834FF4807369460093DA
:1082D8008DF806408DF807408DF804508DF805504C
:1082E80009F038FF21464FF480000AF041F807F5FD
:1082F8008067284631460AF0E5F840F6FC733846B0
:10830800694600934FF480588DF804408DF8064074
:108318008DF807408DF8055009F01CFF384669466E
:10832800CDF800808DF806408DF807408DF8046080
:108338008DF8055009F00EFFA7F81880042007F5FE
:10834800806731460AF0BEF84AF2C23338466946B9
:1083580000938DF804408DF806408DF807408DF89D
:10836800055009F0F7FE44F20403384669460093C5
:108378008DF806408DF807408DF804608DF805509B
:1083880009F0E8FE4FF480433B83DFF88C80042338
:108398007B83082031460AF095F84FF68C734046E7
:1083A8006946009310278DF804408DF806408DF833
:1083B80007408DF8055009F0CDFE404669468DF816
:1083C80006408DF8074000978DF804608DF8055039
:1083D80009F0C0FE38463146A8F81A700AF072F85B
:1083E8008DF806408DF807400A4C4FF6FF7320467B
:1083F800694600938DF804608DF8055009F0AAFECF
:108408004FF610736383EF232383BDE8FC8100BF1D
:108418000000024000100240000C0240C90802F0AF
:1084280095B8072820D8DFE800F004070A0D1013D4
:10843800161B4FF4807210E04FF400720DE04FF4F9
:1084480080620AE04FF4006207E04FF4805204E0D3
:108458004FF4005201E04FF48042044B5A837047B6
:10846800024B4FF400425A83704700BF001002408D
:10847800072820D8DFE800F004070A0D1013161BA0
:108488004FF4807210E04FF400720DE04FF48062F8
:108498000AE04FF4006207E04FF4805204E04FF422
:1084A800005201E04FF48042034B1A837047024B9D
:1084B8004FF400421A8370470010024038B5054651
:1084C800002445FA04F3DB07E0B202D5FFF7D0FF3A
:1084D80001E0FFF7A6FF0134082CF2D138BD08B53A
:1084E80007282ED8DFE800F004060B10151E2328F5
:1084F80000200FE0144B1869C0F3802008BD124B10
:108508001869C0F3C02008BD0F4B1869C0F30030CC
:1085180008BD012001F098F9B0F5006F34BF0020C4
:10852800012008BD084B1869C0F3403008BD064B50
:108538001869C0F3803008BD034B1869C0F3C03018
:1085480008BD002008BD00BF000C024007282DD838
:10855800DFE800F004090E13181D2227144B586990
:10856800C0F300207047124B5869C0F34020704791
:108578000F4B5869C0F3802070470D4B5869C0F302
:10858800C02070470A4B5869C0F300307047084B49
:108598005869C0F340307047054B5869C0F38030C4
:1085A8007047034B5869C0F3C030704700207047CC
:1085B8000010024010B50020FFF7C8FF041C18BFC8
:1085C80001240120FFF7C2FF10B144F00204E4B215
:1085D8000220FFF7BBFF08B144F004040320FFF7B3
:1085E800B5FF08B144F008040420FFF7AFFF08B155
:1085F80044F010040520FFF7A9FF08B144F0200457
:108608000620FFF7A3FF08B144F040040720FFF756
:108618009DFF08B144F08004204610BD034B202282
:1086280008B15A8370471A83704700BF0010024090
:10863800082008B501F008F9592805D9074B1A7818
:1086480052B901221A7008BD082001F0FDF854281B
:1086580002D8024B00221A7008BD00BF2C06002069
:10866800044B18780138C0B201288CBF00200120C3
:10867800704700BF2C060020044B1878012802D14F
:1086880002221A7070470020704700BF2C06002095
:1086980020B9034B1869C0F3402070470020704789
:1086A8000004024008B580B9094B1A78094B1868CC
:1086B80022B95B68000C40EA034008BD596842F2E1
:1086C800107200230DF018FE08BD002008BD00BF81
:1086D800F94B0020484D002010B508BB72B6114B6D
:1086E8000A461878CB171049C1E9002330B9086841
:1086F8004C680204230443EA104307E00A6842F284
:108708001070A2FB00234C6800FB0433C1E900236E
:10871800064A00231360064A1360064A536262B68B
:1087280010BD00BFF94B0020484D0020244D00200B
:10873800744D002000040140024B1869C0F300206A
:10874800704700BF0008024010B598B90A4A0B4BA1
:10875800127819600A4C186832B10DF0E3FB094928
:108768000DF0E8FC206010BD0DF0DCFB06490DF0B3
:10877800E1FC206010BD00BFF94B0020404D0020F7
:10878800F44B002000401C4600FF7F47164B70B595
:1087980053F82060154B360253F82030144C96FBE2
:1087A800F3F203FB1266350495FBF3F103FB115555
:1087B80055B10121215442F2107404FB06F191FBDA
:1087C800F3F104FB021102E001EB02412554094BCD
:1087D80021F07F4403EB40131A6902F07F422243E1
:1087E8001A61BDE87040AFE7EC4B0020E84B002071
:1087F800F94B0020544D002038B5044620BB01F049
:108808004403042B194B9A680BD1C80602D542F4CD
:10881800807208E022F480729A60DA6842F480720A
:1088280005E022F480729A60DA6822F48072DA60D5
:108838000F4BC1F3C00211F001011A700D4B02D0A9
:1088480001221A7000E019700B4B0C4D1A5D0C4B8D
:1088580018681AB10DF066FB0A4902E00DF062FBD8
:1088680009490DF067FC45F8240038BD003C01407B
:10887800F84B0020F04B0020F94B0020F44B00206F
:10888800404D002000401C4600FF7F47F0B5524D88
:108898008DB00024C0230226284607A907938DF827
:1088A80020608DF822408DF821608DF8234009F072
:1088B80051FC28460621032209F0CFFC0322284652
:1088C8000721A5F5823509F0C8FC0121304609F0D9
:1088D80029FE28460AF0F4F801A80AF0D9F94FF65B
:1088E800FF73284601A90293ADF80440ADF80C4087
:1088F800ADF806400AF08EF92246234603212846A1
:108908000AF002FE04A80AF03DFC284604A9ADF8C6
:1089180018400AF0ABFC04A92846ADF810400AF04C
:10892800A5FC04A80AF02EFC284604A9ADF81840B6
:108938000AF09CFC0423284604A9ADF810300AF07C
:1089480095FC284641F65F610AF03BFD6C622846BB
:1089580001210AF0F4F9082130460AF04DF84FF4E5
:1089680080730125099309A808238DF829308DF80B
:108978002A508DF8284009F013FB184B0BA89A6869
:10898800274622F480729A60DA6822F48072DA60EC
:108998008DF82F501723124D8DF82C3007238DF8A2
:1089A8002D308DF82E400AF0C5FF2969204621F0A8
:1089B8007F41FFF7C9FE2046E97CFFF71DFF094B01
:1089C800C8221A60084B4FF400421A602046FFF78D
:1089D800DDFE0DB0F0BD00BF00080240003C0140C4
:1089E800544D0020EC4B0020E84B002030B5284BBC
:1089F800284A1978526A284B09B1C2F580321A60A0
:108A08001868264B244A196888421068196816DDC8
:108A1800411AB1F5004F22490868044648680546DE
:108A280005DA10681B681F4AC31A126825E018681F
:108A380013681C4AC31A126803F5803311E0884290
:108A480021DA18681168411AB1F5004F144908680D
:108A580004464868054609DA18681368114AC31AB3
:108A680012685343E41A65EBE3750AE010681B6863
:108A78000C4AC31A126803F580335343E41845EBD4
:108A8800E375C1E90045044B1A68044B1A6030BD10
:108A9800F04B002000040140244D0020744D0020BC
:108AA800484D0020404D00200C4B1A6912F0040F6D
:108AB8001A690CBF08200020110703D4002814BF2E
:108AC8000C2004201B691A06044B58BF40F0020012
:108AD8001B69DB0558BF40F001007047000C0240DD
:108AE800034B08B1034A00E0034ADA60704700BF4D
:108AF80000ED00E00400FA050100FA050C49002326
:108B08004FF0FF3203F1200041F8202003F160000C
:108B18000133082B41F82020F4D100231946044AD8
:108B28009A180133F02B82F80013F8D1704700BF70
:108B380000E100E0064B02225A83064A042313830D
:108B48004CF2503300BF013BFCD1042353837047E0
:108B58000000024000080240064B04225A83064ADD
:108B6800022313834CF2503300BF013BFCD1022394
:108B780053837047000802400000024028B9044BA4
:108B8800186900F00800C0B270470020704700BFA5
:108B980000000240684620F007018D4601B54FF4F9
:108BA800807009F057FAD0B14FF4807009F060FA7C
:108BB8000020FFF71BFF002007F0CCFE0A4B1B78B4
:108BC8006BB90A4B9A6822F480729A60DA6822F4C8
:108BD8008072DA60064B1A6922F080621A61BDE879
:108BE80001408546704700BFF84B0020003C01401B
:108BF800544D0020014B53F820007047E84B0020EB
:108C0800014B53F820007047EC4B0020014B43F810
:108C18002010BBE5E84B0020014B43F82010B5E5D8
:108C2800EC4B002070477047704700BF70B5044692
:108C380088B058480AF096FC4FF40030012109F03A
:108C480065FC0820012109F03DFC022600252023AF
:108C5800514805A905938DF818608DF81A508DF8BC
:108C680019608DF81B5009F075FA40234A4805A988
:108C780005938DF818608DF81A508DF819608DF8E5
:108C88001B5009F067FA44480521072209F0E5FA64
:108C980041480621072209F0E0FA01A80AF012FD6E
:108CA8000B2C25D8DFE804F02406090C0F12151840
:108CB8001B1E20224FF461531CE04FF4964319E029
:108CC8004FF4E14316E04FF4164313E04FF46143C9
:108CD80010E04FF496330DE04FF4E1330AE04FF41F
:108CE800613307E02D4B05E02D4B03E02D4B01E0F0
:108CF8004FF4165301A9274801930AF087FC26234D
:108D0800002401258DF81C3007A806238DF81D3096
:108D18008DF81E408DF81F500AF00CFE1D4840F2D9
:108D2800FF310AF0D0FD282122461A480AF0ACFD8E
:108D38002A46184840F227710AF0A6FD2A46154827
:108D480040F226610AF0A0FD2A46124840F2255159
:108D58000AF09AFD22460F4840F224410AF094FD99
:108D680022460C4840F646010AF08EFD2246094884
:108D780040F66A110AF088FD6021224605480AF08B
:108D880083FD054B10225A83024829460AF0BBFC92
:108D980008B070BD00440040000C024090D00300B1
:108DA80020A1070040420F00684620F007018D46C9
:108DB80019B529490B889B061BD5284B5B69D80632
:108DC80001D58B8815E0264B1A6858680132202A8D
:108DD80008BF0022824205D01C6888881919C0B2D1
:108DE80008721A601F4B0A221A601D4B9A6A1E4BA2
:108DF8001A60194803881A061AD51B4B1A68BAB99B
:108E0800174BDC6A196B8C420ED0144910240C8362
:108E1800196B5C1894F83440013184801963196B1C
:108E2800202905D11A6303E040F227710AF02CFDCE
:108E3800094803885B060BD540F226610AF067FDF6
:108E4800074B1A6BDB6A9A4202D1044B10225A83F1
:108E5800BDE819408546704700440040000C0240B8
:108E680030060020004C0020FC4B00200A4BDA6A38
:108E7800196B0132202A08BF00228A420AD0D96A17
:108E8800591881F834000548DA6240F22771012246
:108E98000AF0FABC704700BF3006002000440040CA
:108EA8000A4B59681A6891420CD05A6899180132CD
:108EB800097A5A605A680170202A05D100225A603E
:108EC80001207047002070470120704730060020BD
:108ED800014B9862704700BF30060020034B18789A
:108EE80010B100221A700120704700BF044C002006
:108EF80072B6034B00225A601A6062B6704700BF10
:108F08003006002010B5044601E0FFF7AFFF14F863
:108F1800010B0028F9D110BD684620F007018D46E5
:108F280071B5284D284B2C681B680134082C08BFE4
:108F3800002400219C4287B024483CD001AA08F0B4
:108F4800C9FC9DF80C302A68042B214B03EB021254
:108F580006D1012151702A6803EB0213029A05E039
:108F6800002151702A6803EB0213019A5A609DF898
:108F78000D30174A022B134B196802EB011201D16D
:108F8800012100E0002191701B689DF80E10104A25
:108F98001B010C48D1540DF10E010023056811F88E
:108FA800016F02EB0515ED180133082B2E72F5D170
:108FB800044B1C6001E008F0D3FC07B0BDE8714029
:108FC80085467047944C0020084C002000640040FF
:108FD800144C0020684620F007018D4671B5284DD5
:108FE800284B2C681B680134082C08BF0024012179
:108FF8009C4287B024483CD001AA08F06BFC9DF83D
:109008000C302A68042B214B03EB021206D10121F4
:1090180051702A6803EB0213029A05E0002151708F
:109028002A6803EB0213019A5A609DF80D30174A1B
:10903800022B134B196802EB011201D1012100E048
:10904800002191701B689DF80E10104A1B010C48F6
:10905800D1540DF10E010023056811F8016F02EBE0
:109068000515ED180133082B2E72F5D1044B1C6041
:1090780001E008F075FC07B0BDE87140854670470F
:10908800944C0020084C002000640040144C002040
:10909800684620F007018D4631B52B4B2B4A1968DD
:1090A800126886B0914205D129480121002208F0B2
:1090B800DDFC44E01968274A02EB0111497851B1F7
:1090C80004211B688DF80C100021019102EB03129A
:1090D8005368029307E01B688DF80C1002EB03122B
:1090E80053680291019318491A4B0A680DF10E0052
:1090F80003EB021292781C46002A14BF02220022B7
:109108008DF80D200A6812019A5C8DF80E20002255
:109118000D680D4B04EB0515AD182D7A0132082AA0
:1091280000F8015FF4D11A6801321A601A68082A37
:1091380001D100221A60064801A908F034FB06B0E4
:10914800BDE8314085467047104C00200C4C00208B
:1091580000640040984C00202DE9F04101388AB0A5
:109168000E461546072829D8DFE800F02018161201
:10917800100E0C040223ADF810300B238DF81430B8
:10918800012322E003231AE0062318E00C2316E04B
:109198000F23ADF8103015E01E2310E03C23ADF886
:1091A80010300F238DF8143007230EE07823ADF824
:1091B80010300C238DF81430032306E00823ADF893
:1091C80010300F238DF8143002238DF815308A489B
:1091D80000238DF8133008F089F901214FF0007051
:1091E80009F094F90820012109F06CF903230024FF
:1091F80008200121079302238DF820308DF82130B3
:109208008DF822408DF8234009F05CF97B4807A9C6
:1092180008F0A0FF09227948214609F01EF801212B
:109228000922764809F019F80127734804A98DF82E
:1092380012408DF816408DF817708DF818408DF88B
:1092480019408DF81A708DF81B7008F069F9B6F599
:10925800006F8DF80A408DF80B408DF80C704FF6B2
:10926800FF730DDA7201ADF80020ADF80240ADF8D9
:109278000430ADF80630ADF808408DF80D700BE0FD
:10928800ADF80040ADF80240ADF80430ADF8063056
:10929800ADF808408DF80D40684608F0ADF9012397
:1092A80000228DF80A308DF80B208DF80C3095B11E
:1092B800B5F5006F0FDA6901ADF802204FF6FF72BD
:1092C800ADF80010ADF80420ADF80620ADF8083070
:1092D8008DF80D300EE01146ADF80020ADF80220F3
:1092E8004FF6FF72ADF80420ADF80620ADF808304F
:1092F8008DF80D10684608F07FF902238DF80A30C2
:109308007313F60046F0040600270124ADF8026046
:1093180068464FF6FF76ADF800308DF80B708DF883
:109328000C40ADF80460ADF80660ADF808708DF833
:109338000D4008F061F94FF00303BD42B8468DF8BF
:109348000A308DF80B708DF80C4010DD6B13ED00B2
:1093580045F00405ADF80030ADF80250ADF80460F2
:10936800ADF80660ADF808408DF80D400CE0042318
:10937800ADF80070ADF80230ADF80460ADF80660E5
:10938800ADF808408DF80D70684608F035F90124ED
:1093980014230726002509A88DF824308DF82560A8
:1093A8008DF826508DF827400AF0C4FA152309A82D
:1093B8008DF824308DF825608DF826508DF82740DB
:1093C8000AF0B8FA132309A88DF824308DF825601F
:1093D8008DF826508DF827400AF0ACFA0221224673
:1093E800054808F043FB04481021224608F03EFBDC
:1093F8000AB0BDE8F08100BF00640040000C0240E4
:10940800F0B5437887B00746426833B104238DF836
:109418000C3000230292019303E08DF80C30019286
:109428000293BB780DF10E02002B14BF0223002318
:109438008DF80D303B788DF80E300023F918097A35
:109448000133082B02F8011FF8D1114801A908F0CF
:10945800AAF9042817D10F4D0F4B2C681B6801344B
:10946800082C08BF00249C420FD02E680B4B03EB3E
:10947800061697E80F0086E80F00012104480A46FF
:109488002C6008F0F3FA012000E0002007B0F0BDDE
:10949800006400400C4C0020104C0020984C002028
:1094A80070B50D4B0D4C054622681B689A420FD0CB
:1094B80026680B4B03EB061301360FCB85E80F002C
:1094C80026602368082B05D100232360012070BD86
:1094D800002070BD012070BD944C0020084C002075
:1094E800144C00202DE9F04F012189B04FF4805031
:1094F80009F018F8464E01200024E0230225014611
:1095080006938DF81E408DF81F408DF81C508DF87D
:109518001D5008F0D7FF304606A908F01BFE0521AC
:1095280030460A4608F099FEDFF8F0B030460621CA
:10953800052208F092FE05223046072108F08DFE2C
:1095480001264FF482794FF400784FF0100A5846FC
:1095580001A9ADF80440ADF80840ADF81240ADF8E7
:109568001440ADF80690ADF80A50ADF80C60ADF8AF
:109578000E80ADF810A009F0D9F85846314609F028
:1095880070F9244F31464FF4804008F0BFFF4FF484
:1095980060432846314606938DF81E408DF81F40DB
:1095A8008DF81C508DF81D5008F08CFF384606A920
:1095B80008F0D0FD38460D21052208F04EFE384649
:1095C8000E21052208F049FE38460F21052208F031
:1095D80044FEADF80440ADF80840ADF81240ADF8CF
:1095E80014400D4C01A92046ADF80690ADF80A507C
:1095F800ADF80C60ADF80E80ADF810A009F096F843
:109608002046314609F02DF909B0BDE8F08F00BFBA
:1096180000000240000402400038004000300140D1
:1096280070B504460D46164610B101283FD103E037
:10963800214B02225A8313E0204B10225A832048E0
:10964800022109F09FF90028F9D01D48294609F0A0
:1096580063F91B48012109F095F90028F9D00FE0BA
:109668001848022109F08EF90028F9D01548294632
:1096780009F052F91348012109F084F90028F9D0BA
:109688005EB114B1012C12D103E00B4B02221A83F4
:1096980008E00A4B10221A8302E01CB1012C08D101
:1096A800074800E0074809F034F9C0B270BD00204F
:1096B80070BD304670BD00BF00100240000002407F
:1096C80000300140003800402DE9F04101219CB0F4
:1096D8004FF4800008F0F6FE01214FF48070002559
:1096E80008F020FF032733231AA950481A938DF84E
:1096F8006C708DF86F5008F02DFD1AA94C480124A4
:109708001A978DF86C708DF86F5008F023FD1AA920
:109718004848494E1A948DF86C708DF86F5008F0CF
:1097280019FD21464FF4800008F0CCFE21464FF485
:10973800807008F0F7FE304608F088FA3F4B4FF08B
:10974800070802933E4B304603934FF48063079318
:109758004FF4006308934FF4005309934FF4807358
:109768000A9301A94FF400330B9301950495CDF8A2
:10977800148006950C950D940E950F9508F0F2FA45
:10978800214630462F4E08F028FB16A81695179547
:109798001895199507F01EFD304610A910958DF8FB
:1097A80044408DF845401295139514958DF85480D2
:1097B80007F0E1FC3046214607F0DAFD30460A2181
:1097C8002246234607F052FD30460E210222234648
:1097D80007F04CFD30460F213A46234607F046FD78
:1097E800304608210422234607F040FD304609216F
:1097F8002346052207F03AFD30460B212346062270
:1098080007F034FD424623463046294607F02EFD30
:109818003046214607F0B5FD3046214607F0F4FCF6
:10982800304607F071FD1CB0BDE8F0810008024029
:109838000004024000000240106402404C20014035
:1098480084060020002001400928F8B51CD005D85E
:1098580004280ED008280FD040B17AE00B2863D036
:109868005FD30C2863D0FF2873D16EE0464B18886D
:109878006DE0454B58886AE0434B588940F27123A4
:1098880080B258430013F8BD3F4B988880B20CF063
:1098980045FB0BF027FF00223C4B0BF077FF2EA374
:1098A800D3E900230BF072FF04460D4622462B46EF
:1098B80029A1D1E900010BF0B5FD29A3D3E90023C3
:1098C80006460F46204629460CF08AF802460B4603
:1098D800304639460CF084F80CF01AFA0BF002FF07
:1098E80000222B4B0CF07CF80EF0DCF91EA3D3E918
:1098F80000230BF04BFF1EA3D3E900230BF094FDCC
:1099080002460B461CA1D1E900010CF069F81CA322
:10991800D3E900230BF086FD0CF0FAF90CF0CCFC2F
:10992800F8BD194BD88804E0174B188901E0164B8D
:10993800988944F2740380B2584340F6FF7390FB51
:10994800F3F0A0F500503A38F8BD0F4B988880B274
:10995800F8BD0020F8BD00BF6666666666660A4008
:109968009A99999999990140C3F5285C8FA27240F8
:109978000000000000FEAA409A999999FD6F2F41B6
:10998800C3F5285C8F127140840600200000303F28
:1099980000002440AFF300800C4B072202FB00308C
:1099A80090F800380B7090F801384B7090F8023836
:1099B8008B7090F80338CB7090F804380B7190F8DE
:1099C80005384B7190F806388B7170479406002063
:1099D800254938B500224FF400635A540133B3F5D2
:1099E800804FFAD14FF40064002006210122FFF7CE
:1099F80017FE002005210246FFF712FE0020012273
:109A08000146FFF70DFE8007F3D50020022102462C
:109A1800FFF706FE0020C4F307210246FFF700FE09
:109A28000020E1B20246FFF7FBFD0025A5F13F014A
:109A38004A4242EB0102002001460135FFF7F0FDE2
:109A4800402DF3D1002005210246FFF7E9FD002053
:109A580001220146FFF7E4FDC307F3D44034B4F50F
:109A6800804FC1D138BD00BF94060020F7B5072547
:109A7800454300200C4602460321FFF7D1FD05F5BA
:109A880000650020C5F307210246FFF7C9FD002045
:109A9800E9B20246FFF7C4FD002001460246FFF77F
:109AA800BFFD0746002001460246FFF7B9FD0646FE
:109AB800002001460246FFF7B3FD05460020014697
:109AC8000246FFF7ADFD8DF803000020014602466F
:109AD800FFF7A6FD8DF80400002001460246FFF7B7
:109AE8009FFD8DF80500002001220146FFF798FD33
:109AF80023788DF80600BB4210D16378B3420DD1AC
:109B0800A378AB420AD1DDF80300D4F80330C3EBE5
:109B1800000CDCF1000040EB0C0000E00020FEBD72
:109B280038B51B4B04460D46195500200621012265
:109B3800FFF776FD002005210246FFF771FD0020A2
:109B480001220146FFF76CFD8207F3D500200221B0
:109B58000246FFF765FD0020C4F307210246FFF720
:109B68005FFD0020E1B20246FFF75AFD00202946BA
:109B78000122FFF755FD002005210246FFF750FDA1
:109B8800002001220146FFF74BFDC307F3D438BD7F
:109B98009406002038B50725454305F500650C46B1
:109BA80028460978FFF7BCFF681C6178FFF7B8FF03
:109BB800A81CA178FFF7B4FFE81CE178FFF7B0FF15
:109BC800281D2179FFF7ACFF681D6179FFF7A8FF11
:109BD800A179A81DBDE83840A2E72DE9F84316464B
:109BE800424A044688460023121803E018F8031076
:109BF800D1540133B342F9D1002006210122FFF7E5
:109C08000FFD002005210246FFF70AFD0020012272
:109C18000146FFF705FD8307F3D500200221024620
:109C2800FFF7FEFC0020C4F307210246FFF7F8FC0B
:109C38000020E1B20246FFF7F3FC0025771E44E05E
:109C4800013414F03F0918F8051006D0C7EB050ECB
:109C5800DEF1000242EB0E0200E00122D2B2002047
:109C6800FFF7DEFCB9F1000F2ED1BD422CD2002047
:109C780005210246FFF7D4FC002001220146FFF728
:109C8800CFFC10F00100F2D106210122FFF7C8FC39
:109C9800002005210246FFF7C3FC002001220146EF
:109CA800FFF7BEFC8007F3D5002002210246FFF72C
:109CB800B7FC0020C4F307210246FFF7B1FC0020DF
:109CC800E1B20246FFF7ACFC0135B542B8D100203D
:109CD80005210246FFF7A4FC002001460122FFF7F8
:109CE8009FFCC107F3D4BDE8F88300BF94060020A9
:109CF800014B185C704700BF9406002010B5054C56
:109D08000023201802E0C45CCC5401339342FAD1FA
:109D180010BD00BF94060020F7B5002003210246BD
:109D2800FFF77EFC002001460246FFF779FC002081
:109D380001460246FFF774FC404D002443F6FF76C7
:109D4800A11B4A4242EB010200200146FFF768FCD2
:109D580060550134B4F5804FF2D100200521024648
:109D6800FFF75EFC002001220146FFF759FC10F0C6
:109D78007104F2D1FEF776FA40F2CF7607462F4DFE
:109D880006E095F8FF47A4F14202544244EB02046E
:109D9800FEF768FAC01B0028B8BF4042B04202DC98
:109DA800002CEED000E01CB1254B1B78002B39D0DD
:109DB80040F2FF700021FFF7B3FEFFF709FE002015
:109DC80020494022FFF709FF4FF480701E49B42252
:109DD800FFF703FF40201D492022FFF7FEFE02ADDA
:109DE800002345F8043D4FF4C36420460422294665
:109DF8000434FFF7F2FEB4F5FF6FF6D102AD00238D
:109E080045F8043D4FF4A76420460422294604344B
:109E1800FFF7E3FEB4F5C36FF6D140F2FF704221BD
:109E2800FFF77EFE002040220649FFF767FF40202B
:109E380007492022FFF762FFFEBD00BF94060020FD
:109E48003C4D002004000020788301085883010855
:109E5800544D0020F8B505460C4606F0E7FB0646CB
:109E680028B128462146BDE8F84006F0E5BB324651
:109E7800C4F307410120FFF7D3FB0B4D070232461D
:109E8800C4F307212F600120FFF7CAFB47EA000649
:109E9800360201202E60E1B20246FFF7C1FB0643FD
:109EA80036092E60F8BD00BF94460020254B0321DB
:109EB80010B501FB003292F905403F2C01DD3F242B
:109EC800547101FB003393F905203F3201DAC122B6
:109ED8005A711C4B032202FB003291791F2901D9C8
:109EE8001F2191714FF440229A60032202FB003334
:109EF8001B79012B03D1134B4FF450229A60114B5D
:109F0800032103EBC002D27C01FB00311AB94A7964
:109F180002F07F0205E0497902F0030201F07C01BA
:109F28000A439968074C41EA02229A60032303FB1B
:109F380000439979A3681943A160FFF78BFFA368D1
:109F4800636110BD94460020204B052110B501FB2C
:109F58000032147E012C01D90124147601FB003350
:109F68005A7E032A01D903225A76184B052101FB90
:109F78000032947E0F2C01D90F24947601FB003314
:109F8800DA7E032A01D90322DA76104C052303FB73
:109F98000042117F0F2901D90F21117703FB0043DC
:109FA800197F1A7E41F4202141EAC2315A7E41EAE2
:109FB80042319A7EDB7E41EA022141EA4311A160E7
:109FC800FFF748FFA368236210BD00BF9446002036
:109FD800524B0B2110B501FB003292F82440032CA0
:109FE80002D9032482F8244001FB003393F8262089
:109FF800032A02D9032283F82620484B0B2101FBB0
:10A00800003292F828400F2C02D90F2482F82840F9
:10A0180001FB003393F82920072A02D9072283F885
:10A0280029203E4B0B2101FB003292F82A400F2CCD
:10A0380002D90F2482F82A4001FB003393F82D201F
:10A048000F2A02D90F2283F82D2034490B2202FB54
:10A05800001393F82E400F2C02D90F2483F82E40BA
:10A0680002FB001292F82430DB0343F400248C60D6
:10A0780092F8251019B1294A43F404239360274B19
:10A088000B2202FB003292F827201AB19A6842F498
:10A0980000529A600B2279B902FB003292F828101C
:10A0A80092F82640C90141EAC4219C6892F8292007
:10A0B800214341EA02121DE002FB003292F82C30E3
:10A0C80016491BB18B6843F480538B60134B0B22EA
:10A0D80002FB003292F82E1092F82D409A6842EA5C
:10A0E800C41201F0070442EA041209079A6002D573
:10A0F80042F400629A60094C0B2303FB004393F877
:10A108002B2022B993F82A20A3681343A360A168DF
:10A11800FFF7A0FEA368236310BD00BF944600208C
:10A1280038B51F4B4FF460229A60C2009918C97C59
:10A1380011B14FF4702199609A18517B147B09036F
:10A1480041EA84319C6821439960937B012B03D1B8
:10A15800134B41F480619960114BC1005C189A68F7
:10A16800E57B247C42EA0522012C9A6004BF42F078
:10A1780080029A605B185B7C094A012B03D19368C3
:10A1880043F040039360064C04EBC003997CA3683A
:10A1980043EA0111A160FFF75DFEA368636338BD60
:10A1A8009446002010B5144B0022C1009A605A183A
:10A1B80092F83D2012B14FF400729A605B1893F840
:10A1C8003E300D4A1BB1936843F4807393600A4C88
:10A1D800C300E21892F83F100F2902D90F2182F824
:10A1E8003F10E31893F83F10A3681943A160FFF7E5
:10A1F80031FEA368236410BD94460020214B012042
:10A2080010B50322002405211871187402209874CF
:10A2180083F8240083F82800597199711A735A73C6
:10A228009C73DC735C74DC741C765C769C76DC76E0
:10A238001C7783F83D4083F83E4083F83F4083F81D
:10A24800254083F8274083F8264083F8292083F89F
:10A258002A1083F82B4083F82C4083F82E2083F8AB
:10A268002D402046FFF770FE2046FFF71FFE2046D0
:10A27800FFF756FF2046FFF795FF2046BDE8104040
:10A28800A6E600BF94460020054B042903EBC00353
:10A2980083F83F1002D0002283F83D2082E700BFF8
:10A2A80094460020044B03EBC00383F83D1011B122
:10A2B800042283F83F2075E794460020024B03EB05
:10A2C800C00383F83E106DE794460020024B03EB71
:10A2D800C00090F83F00704794460020024B03EB03
:10A2E800C00090F83D00704794460020024B03EBF5
:10A2F800C00090F83E00704794460020034B0B22A4
:10A3080002FB003383F8241062E600BF9446002065
:10A31800034B0B2202FB003383F8251058E600BFDD
:10A3280094460020034B0B2202FB003383F82710CE
:10A338004EE600BF94460020034B0B2202FB00337D
:10A3480083F8261044E600BF94460020034B0B22F6
:10A3580002FB003383F828103AE600BF9446002039
:10A36800034B0B2202FB003383F8291030E600BFB1
:10A3780094460020034B0B2202FB003383F82A107B
:10A3880026E600BF94460020034B0B2202FB003355
:10A3980083F82C101CE600BF94460020034B0B22C8
:10A3A80002FB003383F82D1012E600BF944600200C
:10A3B800034B0B2202FB003383F82E1008E600BF84
:10A3C80094460020034B0B2202FB003090F8240037
:10A3D800704700BF94460020034B0B2202FB00305D
:10A3E80090F82500704700BF94460020034B0B22CD
:10A3F80002FB003090F82700704700BF9446002009
:10A40800034B0B2202FB003090F82600704700BF78
:10A4180094460020034B0B2202FB003090F82800E2
:10A42800704700BF94460020034B0B2202FB00300C
:10A4380090F82900704700BF94460020034B0B2278
:10A4480002FB003090F82A00704700BF94460020B5
:10A45800034B0B2202FB003090F82C00704700BF22
:10A4680094460020034B0B2202FB003090F82D008D
:10A47800704700BF94460020034B0B2202FB0030BC
:10A4880090F82E00704700BF94460020024B05222A
:10A4980002FB0033197657E594460020024B05224B
:10A4A80002FB003359764FE594460020024B052203
:10A4B80002FB0033997647E594460020024B0522BB
:10A4C80002FB0033D9763FE594460020024B052273
:10A4D80002FB0033197737E594460020024B05222A
:10A4E80002FB0030007E704794460020024B052294
:10A4F80002FB0030407E704794460020024B052244
:10A5080002FB0030807E704794460020024B0522F3
:10A5180002FB0030C07E704794460020024B0522A3
:10A5280002FB0030007F704794460020024B032254
:10A5380002FB00331971B9E494460020024B032250
:10A5480002FB00335971B1E494460020024B032208
:10A5580002FB00339971A9E494460020024B0322C0
:10A5680002FB00300079704794460020034B032219
:10A5780002FB003090F90500704700BF94460020A8
:10A58800024B032202FB003080797047944600207A
:10A59800024B03EBC0031973C2E500BF94460020C9
:10A5A800024B03EBC0035973BAE500BF9446002081
:10A5B800024B03EBC0039973B2E500BF9446002039
:10A5C800024B03EBC003D973AAE500BF94460020F1
:10A5D800024B03EBC0031974A2E500BF94460020A8
:10A5E800024B03EBC00359749AE500BF9446002060
:10A5F800024B03EBC003997492E500BF9446002018
:10A60800054B10B503EBC003D9740446FFF788FD6A
:10A618002046BDE8104049E494460020024B03EB75
:10A62800C000007B704700BF94460020024B03EB3C
:10A63800C000407B704700BF94460020024B03EBEC
:10A64800C000807B704700BF94460020024B03EB9C
:10A65800C000C07B704700BF94460020024B03EB4C
:10A66800C000007C704700BF94460020024B03EBFB
:10A67800C000407C704700BF94460020024B03EBAB
:10A68800C000807C704700BF94460020024B03EB5B
:10A69800C000C07C704700BF944600202DE9F047F9
:10A6A800314F98463B1893F8443004460D461646F9
:10A6B800DDF820A0DDF82490042B1AD8DFE803F099
:10A6C80003080D121700FFF783FC3B19012212E063
:10A6D800FFF726FD3B1902220DE0FFF735FC3B1979
:10A6E800032208E0FFF7E2FB3B19042203E0FFF72F
:10A6F80059FD3B19002207EBC40483F84420A27CCF
:10A70800194B012A0DD002D3022A23D111E015B129
:10A718001B689B0C2B70EEB1134B1B689B0A3370A4
:10A7280018E0B8F1000F15D01B689B0AC8F8003074
:10A7380010E0B8F1000F04D01B68DB0B5B01C8F810
:10A748000030BAF1000F05D0074B1B68C3F3842310
:10A758008AF80030B9F1000F03D0034B1B6889F861
:10A768000030BDE8F08700BF94460020054B0B225F
:10A7780002FB003393F82B201AB9012283F82B200F
:10A7880026E4704794460020054B0B2202FB003359
:10A7980093F82B201AB1002283F82B2018E4704775
:10A7A80094460020064B40F2826203EBC000407CD6
:10A7B80040F63B43002814BF10461846704700BFB8
:10A7C8009446002070B5104C054604EBC0039E7CEF
:10A7D800032E03D003229A74FFF7A2FC2846FFF742
:10A7E8009FFC2468200344BF6FEA04346FEA1434E2
:10A7F800032E06D0044B284603EBC5039E74FFF7CF
:10A808008FFC204670BD00BF9446002070B50A4CEE
:10A818009DF810609DF8145004EBC00484F83810BB
:10A8280084F8392084F83A3084F83B6084F83C5046
:10A83800BDE87040B6E400BF9446002006281CD846
:10A84800DFE800F004070A0D101317000B4B1B6814
:10A858000DE00A4B1B6C0AE0084B1B6B07E0074B2B
:10A868001B6A04E0054B5B6901E0044B5B6B0B6002
:10A878007047024B93F82B300B60704794460020CA
:10A88800704770477047704770477047704712238A
:10A898000B800148704700BF4400002004230B8050
:10A8A800004870475600002000207047002070477D
:10A8B8000020704770B5084C0022236806E03F2B43
:10A8C80003D8865CE5182E71013301328A42F6D12D
:10A8D800014A0020136070BDDC46002010B5044C0E
:10A8E8000A460448214609F035FD204610BD00BF40
:10A8F800276100201499010810B5044C0A46044841
:10A90800214609F027FD204610BD00BF2761002021
:10A918002299010810B5044C0A460448214609F05A
:10A9280019FD204610BD00BF276100202D990108A0
:10A9380010B5044C0A460448214609F00BFD204690
:10A9480010BD00BF276100203599010810B5044CDF
:10A958000A460448214609F0FDFC204610BD00BF08
:10A96800276100204D990108202802D0212822D1F2
:10A9780012E08A784878120442EA002208780F4BDD
:10A988000243C87842EA00629A610A791A774A79DA
:10A998005A778A799A770EE0084B9A69100A0A70F2
:10A9A8004870100C120ECA701A7F88700A715A7F8C
:10A9B8009B7F4A718B710020704700BF44000020C4
:10A9C800F7B5274C4FF4C0530026032700932046C1
:10A9D800022369468DF804308DF805708DF80660FD
:10A9E8008DF8076007F0B6FB20460B210A2207F016
:10A9F80034FC0A2220460C2107F02FFC01254FF4D5
:10AA080000732046694600938DF805708DF8046040
:10AA18008DF806508DF8076007F09CFB0A22204647
:10AA2800092107F01AFC4FF4806320466946009319
:10AA38008DF806508DF807508DF8057007F08AFBE1
:10AA48000A210A46204607F008FC29464FF48040B0
:10AA580007F068FD8020294607F040FDFEBD00BFD5
:10AA68000000024007B54FF4C06008F059FF4323C7
:10AA78008DF804300322012301A88DF805308DF8E4
:10AA880006208DF8073008F055FF0EBD782358438F
:10AA98000723B0FBF3F0002301338342FCD970474E
:10AAA8004FF47A735843F1E7684620F007018D4662
:10AAB80001B503480AF046FABDE8014085467047EB
:10AAC800EC4D00200023F0B5094C0A4F40F2FF7509
:10AAD8001E460AE0226810F803C007F802C00132D7
:10AAE800AA4288BF3246226001338B42F2D1F0BDC0
:10AAF800C84B002027590020074910B50A684AB1F9
:10AB0800002304315C5CC45401339342FAD1024BF4
:10AB180000211960104610BDDC460020084B1B6858
:10AB2800082B0BD90023064A111D595CC154013367
:10AB3800092BF8D1002313600120704700207047CB
:10AB4800DC46002007B5054B054803F120023C33DD
:10AB580000930121034B09F05DF80EBD440000206D
:10AB6800EC4D0020A001002001480AF0BFB900BF49
:10AB7800EC4D002038B54A4CA07808B104228CE08E
:10AB88006378C12B4AD015D80D2B0CD80C2B38D292
:10AB9800052B28D002D8042B7ED120E0062B26D006
:10ABA800072B79D126E08C2B32D0B52B33D0822BD2
:10ABB80072D129E0CC2B3DD006D8C32B34D030D36A
:10ABC800C82B34D0C92B03E0D42B4ED002D8D22BBB
:10ABD80062D132E0D62B4CD0FE2B5DD14DE0BDE8E2
:10ABE800384005F0DFBCBDE8384005F0D3BC49204B
:10ABF8002C4901E02C494A200122BDE83840FFF7E2
:10AC08007DB84D202949F7E7BDE8384005F0D2BCAA
:10AC18004B202749F0E75820264928E048202649B4
:10AC2800EAE74020254922E0442025491FE05F202B
:10AC38002449E1E74E2024491DE0204C184D5020BE
:10AC480004F110010422FFF759F8A87804EB401327
:10AC5800D97CFDF7D1FDA87804EB4014216921F0D7
:10AC68007F41BDE83840FDF76FBD184954200422E4
:10AC7800C3E717495C200222BFE7104D4C2005F1BD
:10AC88000C010122FFF73AF8A07805EB4015297B63
:10AC9800BDE8384005F0B0BC03220E4B1A7038BD31
:10ACA800E05300205D4D00205E4D0020614D0020E6
:10ACB8005F4D00206C4D00205C4D0020544D00205D
:10ACC800584D0020734D0020624D0020684D002033
:10ACD800704D00205454002038B58A4A9378022BCE
:10ACE80000F04681032B00F04A81002B40F0AC8134
:10ACF80053784F2B00F0B18023D8462B6ED00DD857
:10AD0800422B58D005D8402B47D0412B40F0988192
:10AD180048E0442B7C4857D05CD851E0492B78D088
:10AD280005D8472B65D0482B40F08A816AE04C2B28
:10AD380000F087804D2B00F08A804B2B40F08081FB
:10AD480073E0572B00F0D88013D8522B00F0A28064
:10AD580006D8502B00F08880512B40F0718189E093
:10AD6800542B00F0B080C0F09C80552B40F06881D7
:10AD7800B5E0842B00F0E18006D8582B00F0CA809B
:10AD8800832B40F05D81D3E0FE2B00F0E18000F2E0
:10AD9800EB80852B40F05481D4E05A4B40F2FF7091
:10ADA800D97804E0574B0020D978574B1970BDE883
:10ADB8003840FEF7B5BED178534B01205970F6E7FD
:10ADC800D17801710420F2E7D2F803304F49C3610A
:10ADD8001C2009E0D17841710520E8E7D2F803305A
:10ADE80049490C2041F80C3F0422BDE83840FEF7E1
:10ADF800F4BE444B444CD3F80330214641F8083F95
:10AE0800082056E03F4B4049DB78262001F8263FD2
:10AE180063E0D2783C4B0AB9DA7503E03C49012279
:10AE2800DA754A60D97D1720C1E7364B364CD97898
:10AE38000320E170FEF774FEE078BDE83840FEF7C5
:10AE480047B8304B0220D9782F4B9970AFE72D4B7C
:10AE58001520D9782C4B5975A9E7D2F803102A4B3D
:10AE6800C9B259761920A2E7264B1620D978264B65
:10AE780099759CE7244B234C1A7D1D4612F0010F4F
:10AE880004D0E378DB0701D4FEF7A2FDE1781420B3
:10AE980029758CE7D2F803301B49202041F8203F60
:10AEA800A2E7184B184CD3F80330214641F8103F5D
:10AEB80010200422FEF791FE6079A1682269BDE89E
:10AEC8003840FEF749B90F4BD3F80320012A11D8AF
:10AED800DB780D491A2001F81A3F012285E7094B52
:10AEE800D3F80320012A05D8DB7807491B2001F88D
:10AEF8001B3FF2E70422A4E0D3780349272001F896
:10AF0800273FEAE7E053002004000020200000204B
:10AF1800545400204E4B4F4CDB78214601F8283F13
:10AF280028200122FEF759FE94F82830A3B917E02B
:10AF3800474BD3F80320484B02E0D2F80320474B95
:10AF48001A6038BD424BD3F80320434B5A6038BDD2
:10AF58003F4BD3F803301BB9BDE83840FDF7EABDD5
:10AF6800BDE83840FDF7F8BD394BDA783C4B69E06D
:10AF780051783C4BD2F8032043F8212038BD537850
:10AF8800282B3AD00BD8022B29D003D8ABB1012BF0
:10AF980056D11BE0092B5AD0272B51D128E02B2B57
:10AFA8003AD004D8292B2DD02A2B49D12FE02D2B8C
:10AFB8003CD036D32E2B43D13DE02B4BD2F8032087
:10AFC8001A60FDF74FF9244B986038BD264BD2F82C
:10AFD80003205A60FDF746F91F4BD86038BD224B55
:10AFE800D2F803209A60FDF73DF91B4B186138BD74
:10AFF800D2F803201C4BDA6038BDD2F803201A4B74
:10B008001A6138BDD2F80320174B5A6138BDD2F8FF
:10B018000320154B9A6138BDD2F80320124BDA6130
:10B0280038BDD2F80320104B1A6238BDD2F803207D
:10B038000D4B5A6238BDD2F803200B4B9A6238BDCB
:10B0480003220A4B1A7038BD084B04221A7038BD07
:10B05800E053002004000020204700205054002026
:10B068004E54002060540020784D00205454002095
:10B0780038B54E4B1A7D9AB94D4AD2F80320511C67
:10B088004FF00A0104D14B4A12685143996101E01B
:10B098004A439A61FDF7E6F8444B0122D8611A75D4
:10B0A800434B5A78042A7FD8DFE802F003182F4F61
:10B0B8001100FDF7D7F83D4BDA69801A9A69002824
:10B0C800B8BF404290423CD900221A7538BD9878E2
:10B0D80003F046FA354C38BB207547E0987805F000
:10B0E80027FA324C054610B1002323753EE0A369C8
:10B0F80033B3FDF7B7F8E369C01AA3690028B8BFEE
:10B10800404298421CD9257544E02B4C627E1AB9FE
:10B11800987805F061FA30BB637E23B1244B9878A8
:10B1280005F05AFAF8B1214CA3694BB1FDF79AF82A
:10B13800E369C01AA3690028B8BF4042984227D8DB
:10B148001A4B1A6A013A1A6238BD1B4C627E1AB948
:10B15800987805F049FA30B9637E63B1144B987852
:10B1680005F042FA38B9114B00221A75134B1A68C8
:10B1780022F0100212E00D4CA3698BB1FDF772F8B2
:10B18800E369C01AA3690028B8BF4042984207D9AA
:10B1980000232375094B1A6842F010021A6038BD63
:10B1A800024B1A6A013A1A6238BD00BF20470020D4
:10B1B800E05300204054002004000020E853002001
:10B1C80010B51F4B9A78012A1CD003D3022A1D4CB4
:10B1D80021D11BE05878082802D8FDF780F90EE045
:10B1E8000A2803D1174B00225A6016E00B2802D117
:10B1F800FDF7A2FA03E0FF280FD1FDF7DBF9114BA9
:10B2080058600AE05878FEF71FFBF8E75878FDF712
:10B218009DF9606001E0042323700B4B1B7873B128
:10B22800084B5A68094B1A60094B22B91A6842F050
:10B2380008021A6010BD1A6822F008021A6010BDD0
:10B24800E0530020545400204F5400204054002064
:10B25800E853002038B5204B5A78812A3AD19A7899
:10B26800922A37D19A79A32A34D15A79B42A31D17A
:10B278001A79C52A2ED1DB78D62B2BD1174B04226D
:10B288001A83FFF771FCFCF7EDFF40F2E73405463F
:10B29800FCF7E8FF401B0028B8BF4042A042F7DD9A
:10B2A80072B6FDF72BFC0E4B00241C6021460D489E
:10B2B80006F093FD0B4806F0C9FC05F04FFF06F0B9
:10B2C80061FE4FF0804007F0FBFB2046BDE83840A8
:10B2D800FDF706BC38BD00BFE05300200010024057
:10B2E80010E000E01064024010B5954C6378892B9B
:10B2F80000F0428278D8722B00F0B68135D80C2B3A
:10B3080000F0508115D8032B00F00C8105D8012BD3
:10B3180000F0008400F2F780EEE0052B00F02381B6
:10B32800C0F01281062B00F02A81072B40F0008420
:10B338002DE16D2B00F077810BD80E2B00F050819A
:10B34800C0F03E81112B00F060816C2B40F0F0833F
:10B3580062E16F2B00F07481C0F06B81702B00F0FC
:10B368007581712B40F0E48377E17D2B00F0C78174
:10B378001BD8772B00F0A1810BD8742B00F08181AA
:10B38800C0F07881752B00F08281762B40F0D08355
:10B398008CE1792B00F09E81C0F095817A2B00F02A
:10B3A8009F817C2B40F0C483A2E1822B00F00882AD
:10B3B8000BD87F2B00F0F081C0F0A781802B00F024
:10B3C800F781812B40F0B483A6E1862B00F0BB8186
:10B3D80003D8842B40F0AC83A9E1872B00F0B98116
:10B3E800882B40F0A583BBE1B12B00F01B833ED82E
:10B3F800A72B00F0BB821ED8A22B00F067820ED8C4
:10B408008C2B00F0EB8103D88A2B40F09183BCE1B0
:10B41800A02B00F04982A12B40F08A834DE2A42B97
:10B4280000F06582C0F05A82A52B00F07482A62B2A
:10B4380040F07E8388E2AC2B00F0C3820BD8A92BA6
:10B4480000F0A582C0F09A82AA2B00F0A882AB2B4C
:10B4580040F06E83ACE2AE2B00F0CA82C0F0BF822F
:10B46800AF2B00F0CD82B02B40F06283D1E2C62B27
:10B4780000F029831ED8B72B00F014830BD8B32B08
:10B4880000F0E182C0F0D682B52B00F0E482B62B42
:10B4980040F04E83EEE2C12B00F0B18103D8B82B07
:10B4A80040F0468306E3C22B00F0B181C32B40F085
:10B4B8003F83B7E1D12B00F02D830ED8C92B00F0C4
:10B4C800158303D8C82B40F03383B7E1CA2B00F0AB
:10B4D8001983CC2B40F02C83B9E1D42B00F0C08128
:10B4E80003D8D22B40F024831AE3D62B00F0C08176
:10B4F800FE2B40F01D83C4E1A078D4F80310BDE80A
:10B50800104004F0BFBED4F803100E4A01F1805376
:10B51800013B934200F2C481094B9878BDE8104082
:10B5280004F056BED4F80310064A01F18053013BDB
:10B53800934200F2B581A078BDE8104004F066BEE1
:10B54800E0530020FEFFFF1F544A5548D2F803106D
:10B5580001F18053013B834200F2A2819078BDE85B
:10B56800104004F0D7BED4F80310B1F1007F80F08A
:10B5780097814A4B9878BDE8104004F0ABBE474A23
:10B5880048499378D27801EB43114A7206E0434A5E
:10B5980044499378D27801EB43118A72424A0121D7
:10B5A800D15410BDA2783F4BD4F8031003EB4213DB
:10B5B8005A7B11B942F0020210E022F002020DE0BB
:10B5C800364A384BD2F80310927803EB42135A7B71
:10B5D80011B942F0010201E022F001025A7310BDD4
:10B5E800A078022104F0B6FED4F8034003F0B4FDBD
:10B5F800002CB8BF6442844200F35281274BD3F831
:10B608000300BDE8104005F0C5B9244BD3F803008A
:10B61800BDE8104005F00ABA204BD3F80300BDE896
:10B62800104005F077B8D4F80300BDE8104005F0E5
:10B6380077B81A4BD3F80300BDE8104005F076B888
:10B64800D4F80300BDE8104005F008B8134BD3F850
:10B658000300BDE8104005F00DB8104BD3F8030007
:10B66800BDE8104005F01CB8D4F80300BDE8104050
:10B6780005F01CB8094BD3F80300BDE8104005F0ED
:10B688005DB9D4F80300BDE8104005F015B8034BC8
:10B69800D3F80300BDE8104005F014B8E0530020CB
:10B6A800FEFFFF1F544D0020B04D0020494BD3F83A
:10B6B8000300BDE8104005F00BB8D4F80300BDE85E
:10B6C800104005F00BB8434BD3F80300BDE8104019
:10B6D80005F00AB8D4F80300BDE8104005F00CB82E
:10B6E8003C4BD3F80300C0B2BDE8104005F00CB8DD
:10B6F800384BD3F80300BDE8104005F0D5B8D4F8AE
:10B708000300BDE8104005F00DB9324BD3F8030033
:10B71800BDE8104005F0D4B82E4BD3F80310987844
:10B72800003118BF0121BDE8104004F01DBE294BAF
:10B73800D3F80330002B00F0FE8105F0F3F9002860
:10B7480040F0F981ACE0D4F80300BDE8104004F003
:10B75800F9BF204BD3F80300BDE8104004F0ECBF5C
:10B768001C4BD3F80300A0F10A03282B00F29880A1
:10B77800BDE8104004F0ECBFD4F803000028C0F284
:10B788008F80BDE8104004F0E9BF124BD3F80300E6
:10B79800BDE8104004F0E8BFD4F80330022B7FD88E
:10B7A8000C4B0D499A78DB788A1882F8243010BD42
:10B7B800084B9878D3F80310BDE8104004F0CABDD0
:10B7C800D4F80310B1F1805F6AD8A078BDE81040C2
:10B7D80004F03CBDE053002020470020A078574BE0
:10B7E800E17803EB4013D97204F0D2FDE178A07838
:10B7F800C1F10801C9B2BDE81040FEF745BDA27805
:10B808004E4B03EB4213D4F803201A7210BD4C4A76
:10B81800D2F80330B3F1805F42D892784749520199
:10B828008B5010BD464AD2F80330B3F1805F37D849
:10B838009178424A02EB4112536010BD404B3F4A97
:10B848009978D3F8033002EB4112D37710BD3C4B03
:10B858003A4A9978D3F8033002EB4112D38110BDEC
:10B86800A278364B03EB4213D4F803205A6110BD7B
:10B87800334B324A9978D3F8033002EB4112938361
:10B8880010BD2F4BD3F80320052A09D89878D9780A
:10B898002A4B03EB40131973BDE8104004F0ACBE0B
:10B8A800284B04221A7010BD254BD3F80310987842
:10B8B800C9B2BDE81040FEF7F5BC214BD3F8031020
:10B8C8009878C9B2BDE81040FEF7F8BCD4F8031068
:10B8D800A078C9B2BDE81040FEF710BD184BD3F8E8
:10B8E80003109878C9B2BDE81040FEF711BDA078E2
:10B8F800FEF772FD38B9D4F80310A078C9B2BDE8D4
:10B908001040FEF719BDD4F80310A078C9B2BDE8FD
:10B918001040FEF739BD0A4CA078FEF75DFDD4F85B
:10B9280003100346C9B2A0781BB9BDE81040FEF762
:10B938000DBDBDE81040FEF73BBD00BF544D0020D3
:10B94800E053002054540020474CA078FEF744FDF3
:10B95800D4F803100346C9B2A0781BB9BDE810405B
:10B96800FEF7FEBCBDE81040FEF718BDD4F8031082
:10B97800A078C9B2BDE81040FEF7FCBC3A4BD3F83A
:10B9880003109878C9B2BDE81040FEF77FBDD4F81F
:10B998000310A078C9B2BDE81040FEF77FBD324B56
:10B9A800D3F803109878C9B2BDE81040FEF77EBD01
:10B9B8002D4BD3F803109878C9B2BDE81040FEF7B4
:10B9C8007DBDD4F80310A078C9B2FEF77FFDA27838
:10B9D800264B03EBC203D4F803205A7110BD224B47
:10B9E800D3F803109878C9B2BDE81040FEF79EBDA1
:10B9F800D4F80310A07849B2BDE81040FEF79EBD08
:10BA0800194BD3F803109878C9B2BDE81040FEF777
:10BA1800BFBD154BD3F803109878C9B2BDE81040E4
:10BA2800FEF7BEBDD4F80310A078C9B2BDE8104037
:10BA3800FEF7BEBD0C4BD3F803109878C9B2BDE829
:10BA48001040FEF7BDBDD4F80310A078C9B2BDE818
:10BA58001040FEF7C5BD044B054A9978D3F803306A
:10BA680002EB4112936110BDE05300202C4D0020E1
:10BA7800544D0020304C314BA078D4F8032043F8C3
:10BA8800302022B903EBC0035979FEF71FFDA078D7
:10BA98002B4B1B5C012B4ED1274BD978BDE81040AE
:10BAA800FCF7BCBCA278254B03EBC203D4F80320F7
:10BAB8001A7110BD204BD3F803109878C9B2BDE8AD
:10BAC8001040FEF72FBCA0781E4BD4F8032003EBE0
:10BAD8004013196912B141F0806101E021F08061E1
:10BAE8001961090EBDE81040FCF786BEA078154B19
:10BAF800E17803EB40131A6922F07F4242EA0162BF
:10BB08001A61EFE70C4B9878D3F80310BDE81040A2
:10BB1800FDF782B8D4F80300BDE8104004F01ABF5E
:10BB2800054B9878D3F80310BDE81040FDF76EB8C0
:10BB3800054B03221A7010BDE05300202C4D002045
:10BB4800B34D0020544D0020545400207FB5AF4C15
:10BB5800AF4D237864226B702A70D4F80300222B2F
:10BB6800686001F0F98257D80F2B01F0AD8026D814
:10BB7800072B00F0EF8510D8032B00F0DF8006D8E4
:10BB8800012B00F0A980022B41F04685BDE0052B72
:10BB980000F0AB8100F2C081E2E00B2B00F0F387EC
:10BBA80006D8092B00F0888600F28A8600F080BE4D
:10BBB8000D2B01F01D8001F23F8000F0FDBF192B15
:10BBC80001F07A8113D8152B01F0E08007D8132BE8
:10BBD80001F07E80142B41F01F8501F0B4B8172BBB
:10BBE8008C4B01F0518101F25B8101F04BB91E2BA6
:10BBF80001F09B8109D81B2B01F08281C1F06D8176
:10BC08001C2B41F0098501F08BB9202B01F00A8229
:10BC180001F24F8201F0C5B9812B01F053832ED870
:10BC2800412B01F0358315D8252B01F0EB8207D87D
:10BC3800232B01F09D82242B41F0EE8401F0B4BA4D
:10BC4800272B01F00E83C1F0E882402B41F0E484F9
:10BC580001F01BBB452B01F0278306D8432B01F0CD
:10BC68001D8301F21E8301F016BB472B01F02283CE
:10BC7800C1F01D83802B41F0CF8401F01EBB882BBF
:10BC880001F0BA8312D8842B01F0598307D8822B8C
:10BC980001F03083832B41F0BF8401F030BB862B49
:10BCA80001F06F8301F2DE8301F066BB8C2B01F09B
:10BCB800368406D88A2B01F0198401F22B8401F00E
:10BCC800FDBBF22B01F09C84FF2B01F09C848D2B93
:10BCD80041F0A28401F049BCA3788BB94B4C0020F9
:10BCE800012104F037FBD4F80310A07804F070FAAF
:10BCF800A37849490022CA544849CA5401F08FBC64
:10BD0800434B04221A7001F08ABC404DAC7884B9C8
:10BD18002046012104F01EFBD5F80310A8784942FB
:10BD280004F056FAAB783C4AD4543C4AD45401F057
:10BD380076BC374B04221A7001F071BCA6785EB944
:10BD4800304602F005FC04F031FEA378324AD6549E
:10BD5800324AD65401F063BC04232B7001F05FBC57
:10BD6800A378002B40F0BC80284B5B78032B00F2B3
:10BD7800B280DFE803F0021A5576274B00251D70C4
:10BD8800264B224C1D7004F081FC18B1A07829467E
:10BD980004F0E0FAA078D4F8031004F073FAA0785D
:10BDA800002104F0D7FA01F03ABC1B4B00251D70A6
:10BDB8001A4B164C1D7004F069FC18B1A07829467E
:10BDC80004F0C8FAA478134B104D1B1993F82430CB
:10BDD800012B07D002D3022B11D107E0204604F033
:10BDE8002DFB06E0204604F037FB02E02046FCF776
:10BDF80059FCD5F80330C118204604F043FA034B28
:10BE08000021987804F0A6FA01F009BCE05300205C
:10BE18005454002020470020504D0020354D00206C
:10BE2800142819DC364B00261E70364B364C1E7013
:10BE3800364B53F8205004F029FC18B1A07831464D
:10BE480004F088FAA078294604F01CFAA0780021AA
:10BE580004F080FA01F0E3BB2D4B04221A7001F0C4
:10BE6800DEBB142832DC264B00251D70254B264CE2
:10BE78001D7004F00BFC18B1A078294604F06AFA8A
:10BE8800A078244B204D1B1893F82430012B06D0A2
:10BE980002D3022B13D105E004F0D0FA04E004F039
:10BEA800DBFA01E0FCF7FEFBAB78D5F80310174A84
:10BEB800591852F821208118184604F0E3F9124B5A
:10BEC8000021987804F046FA01F0A9BB104B04222F
:10BED8001A7001F0A4BB0E4B03221A7001F09FBB2D
:10BEE8000B4B04221A7001F09ABBA3781BB9FFF719
:10BEF800FBF901F094BB064B04221A7001F08FBBCA
:10BF0800504D0020354D0020E0530020EC53002018
:10BF18005454002020470020A378044C002B40F004
:10BF28000084034B25465B7804E000BF545400208E
:10BF3800E0530020FE2B00F2F183DFE813F0FF004E
:10BF4800040109010E01130118011D012101250138
:10BF58002A0130014301560160016A0177018F010E
:10BF680093019701EF03EF03EF03EF03EF03EF03F1
:10BF7800EF03EF03EF03EF03EF03EF03EF03EF0329
:10BF8800EF03EF03EF03EF03EF03EF03EF03EF0319
:10BF9800EF03EF03EF03EF03EF03EF03EF03EF0309
:10BFA800EF03EF03EF03EF03EF03EF03EF03EF03F9
:10BFB800EF03EF03EF03EF03EF03EF03EF03EF03E9
:10BFC800EF03EF03EF03EF03EF03EF03EF03EF03D9
:10BFD800EF03EF03EF03EF03EF03EF03EF03EF03C9
:10BFE800EF03EF03EF03EF03EF03EF03EF03EF03B9
:10BFF800EF03EF03EF03EF03EF03EF03EF03EF03A9
:10C00800EF03EF03EF03EF03EF03EF03EF03EF0398
:10C01800EF03EF03EF0307020B020F0213021702ED
:10C028001B021F02230227022B022F0233023702B0
:10C038003B023F02430247024B024F02D202D702A1
:10C048005302DC02E102650269026D0271027502A7
:10C0580079027D02EF03E602EF03EF03EF03EF033C
:10C06800EF03EF03EF03EF03EF03810285028A0278
:10C078008F02940299029E02EF03EF03EF032B0352
:10C08800300335033A033F034F035F036F03740321
:10C0980079037E03830388038C03910396039B0330
:10C0A800A003A503AA03AF03B303B703BB03BF03EE
:10C0B800EF03EF03EF03EF03EF03EF03EF03EF03E8
:10C0C800EA02EE02F202F602EF03EF03EF03FA02CE
:10C0D800C403C803EF03FE02EF03020306031B03B6
:10C0E800CD03D103EF031F03EF032303EF03EF0394
:10C0F800EF03EF03EF03EF03EF03EF03EF03EF03A8
:10C10800EF03EF03EF03EF03EF03AD02B102B50254
:10C11800B902BD02C102C502C902CD02EF03EF0395
:10C12800EF03EF03EF03EF03EF03EF03EF03EF0377
:10C13800EF03EF03EF03EF03EF032703002004F0FF
:10C148007DF96060EFE2002004F086F96060EAE2C1
:10C15800002004F027F96060E5E2002004F03AF9D5
:10C168006060E0E2002004F09DF96060DBE20020FE
:10C1780004F080F96060D6E29D4B5B7A6360D2E29E
:10C188009B4B9B7A6360CEE2002004F0D1F960609B
:10C19800C9E2984B1B69C3F380236360C3E2964BE3
:10C1A800587E30B904F020FA003018BF01206060D2
:10C1B800B9E2002004F018FAD0F1010038BF0020DD
:10C1C8006060B0E28C4B587E30B904F005FA00305C
:10C1D80018BF01206060A6E2002004F0FDF9D0F14C
:10C1E800010038BF002060609DE2814B5B7B9807AF
:10C1F80002D50023636096E20123636093E27C4BDF
:10C208005B7BD90702D5002363608CE2012363605E
:10C2180089E2002004F05EF9022803D004F03EFB16
:10C22800606080E204F0BCFB60607CE2002004F007
:10C2380057F918B102F090FF606074E26F4CA07873
:10C24800FEF7B0FAA2786A4B03EB42135B7A5843C5
:10C25800FF2390FBF3F06A4B586064E204F0F2FBB2
:10C26800606060E204F0E8FB60605CE2002060600F
:10C27800634D04F05DF918B16B6843F001036B601E
:10C2880004F0E0FB20B15E4B5A6842F002025A60AB
:10C2980004F0FCF920B15A4B5A6842F004025A6083
:10C2A800564CA07804F016F920B9554B5A6842F05C
:10C2B80008025A60A07804F00DF9012804D1504B07
:10C2C8005A6842F010025A604C4B987804F002F910
:10C2D800022804D14A4B5A6842F020025A60454B62
:10C2E8001B695A0504D5464B5A6842F040025A6009
:10C2F800444B1A6912F0080F1A4604D0404B59688B
:10C3080041F0800159601369DB0604D53C4B5A683B
:10C3180042F480725A6002F03BF920B1384B5A68F7
:10C3280042F400725A6002F02DF920B1344B5A6879
:10C3380042F480625A6002F031F9002800F0F3817B
:10C348002F4B5A6842F400625A60ECE104F070FA2C
:10C358006060E8E104F072FA6060E4E104F074FA05
:10C368006060E0E104F080F96060DCE104F088F9E5
:10C378006060D8E104F0FEF96060D4E104F000FAEE
:10C388006060D0E104F0E0FA6060CCE104F0FEF90E
:10C398006060C8E104F000FA6060C4E104F002FAE9
:10C3A8006060C0E104F004FA6060BCE104F006FAE1
:10C3B8006060B8E104F00CFA6060B4E104F012FACD
:10C3C8006060B0E104F016FA6060ACE104F072FA63
:10C3D8006060A8E104F0ACFA6060A4E104F08AFAB5
:10C3E8006060A0E1002004F07BF860609BE100BF82
:10C3F800544D0020000C024004000020E0530020AF
:10C40800545400200004024004F0A2FB60608AE15A
:10C4180004F03CF9606086E104F028FA606082E18B
:10C4280004F01EFA60607EE104F026FA60607AE1AA
:10C4380004F028FA606076E104F02AFA606072E19C
:10C4480004F026FB60606EE10A20FDF7FDF96060EC
:10C4580069E10B20FDF7F8F9606064E10820FDF759
:10C46800F3F960605FE10C20FDF7EEF960605AE1D6
:10C478000920FDF7E9F9606055E10020FEF792F91F
:10C488009A4B9A789A4B03EB42139B7A5843FF23B3
:10C4980090FBF3F0606046E104F0DCF9606042E193
:10C4A80004F0BAF960603EE104F0BCF960603AE17A
:10C4B80004F0FDFA606036E104F004FB606032E1EC
:10C4C80004F018FB60602EE104F09AF960602AE13C
:10C4D800884B1B68636026E10B20FDF7B5F96060A7
:10C4E80021E1854B93F8243063601CE1002003F0C0
:10C4F800F1FF606017E1002003F08AFF606012E13D
:10C50800002003F07FFF60600DE1794BDB7A636008
:10C5180009E1774B1B7A636005E1754B1B68636023
:10C5280001E1734B5B686360FDE0744B1B686360FB
:10C53800F9E06F4BDB7F6360F5E06D4BDB8963608F
:10C54800F1E06F4B1B686360EDE06E4A00231178E1
:10C55800636011B16C490120486013706B4B197806
:10C568001A4621B1684B596841F00201596000230D
:10C578001370D8E0664B1B786360D4E05C4B5B6952
:10C588006360D0E05A4B9B8B6360CCE0584B1B7BBD
:10C598006360C8E00020FDF7A1FE6060C3E00020F2
:10C5A800FDF7A4FE6060BEE00020FDF70BFF6060B1
:10C5B800B9E00020FDF710FF6060B4E00020FDF74F
:10C5C8000BFF514C494B20B99878FDF719FF606073
:10C5D800A9E09878FDF73CFF6060A4E00020FDF733
:10C5E800FBFE494C414B20B99878FDF713FF60607A
:10C5F80099E09878FDF740FF606094E00020FDF72F
:10C60800EBFE414C394B20B99878FDF70DFF60607F
:10C6180089E09878FDF726FF606084E00020FDF748
:10C628000DFF60607FE00020FDF758FF60607AE052
:10C638000020FDF75BFF606075E00020FDF75EFFFE
:10C64800606070E00020FDF761FF60606BE0314BD7
:10C658005B79636067E00020FDF780FF606062E05F
:10C668000020FDF783FF60605DE00020FDF7D6FF46
:10C67800606058E00020FDF7D9FF606053E00020BB
:10C68800FDF7DCFF60604EE00020FDF7DFFF606033
:10C6980049E00020FDF7EAFF606044E01E4B1B788C
:10C6A800636040E0124B9B6963603CE0194B1B6878
:10C6B800636038E0174B1B79636034E00020FDF7B6
:10C6C80095FE60602FE00A4BDB7C63602BE0002066
:10C6D800FCF796FA606026E004F052F9606022E008
:10C6E8000020FCF787FA60601DE000BFE0530020DF
:10C6F800544D002064580020204700201C4D002085
:10C70800384D0020504D002054540020354D002055
:10C71800514D00202C4D0020284D0020032323706C
:10C7280001E004232370AA4B1B78002B00F07787C5
:10C73800A84B5A68A84B1A60A84B2AB91A6842F045
:10C7480008021A6000F06BBF1A6822F008021A602B
:10C7580000F065BFA3781BB104232B7000F05FBF06
:10C768006378C12B60D018D80D2B0ED80C2B41D272
:10C77800052B2CD003D8042B40F0958022E0062B03
:10C788002AD0072B40F08F802DE08C2B3ED0B52B84
:10C7980043D0822B40F0878033E0CC2B60D006D882
:10C7A800C32B4FD047D3C82B53D0C92B03E0D42B6E
:10C7B80064D002D8D22B76D159E0D62B65D0FE2B87
:10C7C80071D169E0002003F0D1FE00F028BF0020FD
:10C7D80003F0C2FE00F023BF492081490122FDF782
:10C7E800FCF900F01CBF4A207E490122FDF7F5F94B
:10C7F80000F015BF4D207C490122FDF7EEF900F04D
:10C808000EBF002003F0BCFE00F009BF4B207749A3
:10C818000122FDF7E2F900F002BF58207449042212
:10C82800FDF7DBF900F0FBBE482072490122FDF755
:10C83800D4F900F0F4BE40206F490422FDF7CDF989
:10C8480000F0EDBE44206D490422FDF7C6F900F062
:10C85800E6BE5F206A490122FDF7BFF900F0DFBE9E
:10C868004E2068490222FDF7B8F900F0D8BE5020E2
:10C8780065490422FDF7B1F900F0D1BE542063499F
:10C888000422FDF7AAF900F0CABE5C206049022222
:10C89800FDF7A3F900F0C3BE4C205E490122FDF765
:10C8A8009CF900F0BCBE4B4B03221A7000F0B7BED7
:10C8B800FEF760F900F0B3BEFEF70EFA00F0AFBE67
:10C8C800554B9978022900F0F980032900F0FB8084
:10C8D800404A002940F03E815B78512B00F0AC8043
:10C8E80026D8472B66D011460ED8432B59D006D8E8
:10C8F800412B50D051D8402B40F0288144E0452BA3
:10C90800464A53D054D84FE04C2B00F0898006D8C3
:10C91800492B57D052D34B2B40F0188155E04F2B61
:10C9280000F0848000F285804D2B40F00F817AE082
:10C93800812B00F09980114612D8552B00F0858084
:10C9480004D8532B354A7CD07DD878E0582B00F09A
:10C958008380802B00F08480572B40F0F78077E0AD
:10C96800852B104600F0928005D8832B00F0888034
:10C9780000F2898081E0FE2B00F0978000F2988019
:10C98800F02B40F0E3808CE040F2FF70FDF7B0F947
:10C99800104B5860E0E0214B88E0204B5B784B60FF
:10C9A800DAE01E4B1B7907E0D369F8E75379F6E71D
:10C9B800D368F4E7194B9B685360CDE0174B93F8A5
:10C9C8002630ECE7154BDB7D74E0144BDB78F3E79E
:10C9D8004F5400205454002040540020E8530020B5
:10C9E8005D4D00205E4D0020614D00205F4D002010
:10C9F8006C4D00205C4D0020544D0020584D002007
:10CA0800734D0020624D0020644D0020684D0020C9
:10CA1800704D0020604D0020E053002004000020ED
:10CA2800974B9B78C8E7964B5B7DC5E7944B5B7E3D
:10CA3800B5E7934B9B7DB2E7914B1B7DBCE7136A2F
:10CA4800ADE71369ABE7937EA9E78D4BDB7EB3E7D0
:10CA58008B4B93F8272064E0894B93F828309EE7A6
:10CA6800884B93F825309AE7864B93F82530A3F145
:10CA78000400434243EB00039EE7824B1B6A8EE7A8
:10CA8800804B1B688BE7804B1B680CE07D497F4817
:10CA98004B68434303F5405339334B6023F000435D
:10CAA8008AE77B4B1B78436056E0794B1B7876E727
:10CAB800784B1B78003318BF012370E75A78764B00
:10CAC80053F822202DE05B78282B28D00CD8022B95
:10CAD8001FD004D8714AB3B1012B37D116E0092B06
:10CAE8003AD0272B32D117E02B2B6C4A22D004D80E
:10CAF800292B19D02A2B29D119E02D2B20D01CD372
:10CB08002E2B23D11FE0664B1B6855E7644B5B68EF
:10CB180052E7634B9A6804E0614BDA6801E0604BC6
:10CB28001A695E4B5A6017E05D4B5B6944E75C4BE2
:10CB38009B6941E75A4BDB693EE7594B1B6A3BE768
:10CB4800574B5B6A38E7564B9B6A35E7534B0322D2
:10CB58001A7001E004231370524B1B78002B00F06D
:10CB68005E854E4B5A68504B1A60504B2AB91A686A
:10CB780042F008021A6000F052BD1A6822F008025A
:10CB88001A6000F04CBDA378022B11D16378372BC3
:10CB98000AD8414903F5A770800001EB83010422FC
:10CBA800FDF71BF800F03BBD03232B7000F037BDE9
:10CBB80004232B7000F033BDA378022B13D13C4B18
:10CBC8005B78372B0AD8344903F5A770800001EB4E
:10CBD80083010422FDF792F800F021BD2F4B0322B8
:10CBE8001A7000F01CBD2D4B04221A7000F017BDFE
:10CBF800A378E3B92E4B5B78012B09D003D3022B22
:10CC0800264C10D109E0002001F09AFC00F007BD85
:10CC1800002001F09DFC00F002BD002001F0A0FC06
:10CC2800606000F0FCBC0323237000F0F8BC1B4BD1
:10CC380004221A7000F0F3BCA37813B1022B3ED182
:10CC480003E0FBF7EBFC00F0EABC194B5B78072B21
:10CC58000AD820B91846FBF7E4FB00F0E0BC1846F8
:10CC6800FBF706FC00F0DBBCFF2B23D1411C0ABFFD
:10CC78000D4BC0B21878FBF721FC00F0D0BC00BF08
:10CC88000400002020470020505400206D4EC6416B
:10CC9800A84D00204E540020605400205454002019
:10CCA800784D00204F54002040540020E8530020C5
:10CCB800E0530020944B03221A7000F0B0BC924B52
:10CCC80004221A7000F0ABBCFEF77AFA00F0A7BC99
:10CCD80062788E4B092A27D8DFE802F005080B0E88
:10CCE80012181B1E21251A6810181CE01A68101A41
:10CCF80019E01A68504316E01A6892FBF0F012E047
:10CD08001A6892FBF0F100FB11200CE01A68104041
:10CD180009E01A68104306E01A68504003E01A68F0
:10CD2800D2431A6000E018601A68794B2AB91A6869
:10CD380042F008021A6000F072BC1A6822F0080279
:10CD48001A6000F06CBC714B1A68714B824219680A
:10CD580004DD41F0040121F0030108E00BBF21F0DC
:10CD6800060121F0070141F0010141F002011960BB
:10CD7800674B2AB91A6842F008021A6000F04FBCE3
:10CD88001A6822F008021A6000F049BC63780C2B7C
:10CD980000F24584DFE803F0071019222B343E46E1
:10CDA8004E565E666E005A4B1B681A0740F1378470
:10CDB800584B186200F033BC554B1B681B0700F139
:10CDC8002E84544B186200F02ABC514B1B68D907BB
:10CDD80040F125844F4B186200F021BC4C4B1B6876
:10CDE800DA0700F11C844B4B186200F018BC484B62
:10CDF8001B685B0740F11384464B186200F00FBCB8
:10CE0800434B1B6813F0050F00F00984414B18626F
:10CE180000F005BC3E4B1B68990740F100843D4B70
:10CE28001862FCE33A4B1B689A0700F0F883394B09
:10CE38001862F4E3364B1B68DB0640F1F083354B90
:10CE48001862ECE3324B1B68990640F1E883314BDA
:10CE58001862E4E32E4B1B685A0640F1E0832D4B21
:10CE68001862DCE32A4B1B681B0640F1D883294B68
:10CE78001862D4E3264B1B68D90540F1D083254BB3
:10CE88001862CCE31862CAE39A6A072A00F2C783D9
:10CE98001C6A03EB82010132CC629A621862BEE31B
:10CEA8009B6A1C4A002B00F0BA83013B936202EB99
:10CEB8008303DB6A1362B2E363782E2B03D8164A26
:10CEC8000121D154ABE3FF2B04D1124B012283F88B
:10CED8004C20A4E303232B70A1E3104B5B782E2B8B
:10CEE80003D80D4A0021D15499E3FF2B04D1094BF3
:10CEF800002283F84C2092E3034B03221A708EE33E
:10CF0800FEF7B6F88BE300BF5454002040540020CD
:10CF1800E853002020470020BC4D0020E0530020AB
:10CF2800974B002283F8252079E36378142B35D8B2
:10CF3800A278A2B9934A9449927E41F82300002A24
:10CF480000F06D83002B00F06A8303F5C270013096
:10CF5800800001EB83010422FCF73FFE5FE3FF2A18
:10CF680018D163B9894D4FF4C364291920460422A6
:10CF78000434FCF732FEB4F5CD6FF6D14FE303F578
:10CF8800C27081490130800001EB83010422FCF763
:10CF980024FE44E37E4B04221A7040E303232B70E3
:10CFA8003DE36378142B39D87A4A9278BAB9764A2D
:10CFB80052F82320764B5A60774B1B78002B00F0F1
:10CFC8002E83764B1A60764B22B91A6842F0080213
:10CFD8001A6024E31A6822F008021A601FE3FF2A85
:10CFE80018D163B9694D4FF4C36429192046042246
:10CFF8000434FCF783FEB4F5CD6FF6D10FE303F5E7
:10D00800C27061490130800001EB83010422FCF702
:10D0180075FE04E35E4B04221A7000E35C4B0322A6
:10D028001A70FCE26578142D3FD85A4CA078020695
:10D038001BD5C30704D503F00FFA534B43F825005B
:10D04800504B9B7E002B00F0EA82524B5B78002B02
:10D0580000F0E58203F5C2704B490130800001EB16
:10D0680083010422FCF7B9FDD9E2D0B903F0F4F941
:10D07800444B45499B7E41F82500002B00F0CF82A8
:10D088006378002B00F0CB82A27803F5C2700130E0
:10D09800D3188018800001EB83010422FCF79DFD62
:10D0A800BDE23B4B04221A70B9E2394B03221A70D5
:10D0B800B5E26278394B0A2A40D8DFE802F0060B5D
:10D0C80011161C24292E33373A00364A196812687B
:10D0D8008A1803E0334A196812688A1A1A602DE020
:10D0E80030491A6809684A43F8E72E4A19681268ED
:10D0F80091FBF2F2F2E72B4A1968126891FBF2F001
:10D1080002FB1012EAE7274A11681A680A40E5E7A5
:10D11800244A11681A680A43E0E7224A11681A6823
:10D128004A40DBE71F4B1A68D243D7E71A681D4B02
:10D13800D4E71C4A1968106811601860174B1A6800
:10D14800174B22B91A6842F008021A6067E21A6897
:10D1580022F008021A6062E2104B1B68C4F8033020
:10D16800A37813B9FEF7C0F859E204232B7056E2EE
:10D178000A4B1B68C4F80330FDF7AEFD4FE200BF51
:10D188002047002004000020EC530020D84D002048
:10D1980054540020E05300204F54002040540020F5
:10D1A800E85300205C540020A24B5B78052B00F26A
:10D1B8003682DFE803F003090F151B219E4B1A681E
:10D1C80002F00F021A602AE29B4B1A6822F0100242
:10D1D8001A6024E2984B1A6822F020021A601EE2B4
:10D1E800954B1A6822F040021A6018E2924B1A68AE
:10D1F80022F080021A6012E28F4B1A6822F48072C1
:10D208001A600CE263782E2B04D88C4A02EB830355
:10D21800186504E203232B7001E2884B884AD3F88F
:10D228000C111160D3F81011864A1160D3F814213B
:10D23800D3F818111A62804A1160D3F81C21824968
:10D248001A75D3F82021DA61D3F824219A6193F86A
:10D258002821885C08B101208854002283F82C21F9
:10D26800DDE1A3786BB9734B5B78142B05D8744A4E
:10D278001168764A42F82310D1E1754B03221A70DF
:10D28800CDE1734B04221A70C9E100F02DFFC6E10D
:10D2980000F032FFC3E100F030FFC0E100F02EFFE4
:10D2A800BDE100F02CFFBAE100F02AFFB7E100F081
:10D2B80028FFB4E100F026FFB1E1604B002283F8BB
:10D2C8002520ACE1637813B1012B10D104E05B4B4E
:10D2D800012283F82520A2E1B0F5006F04D2574A55
:10D2E80082F8253010629AE104232B7097E103231A
:10D2F8002B7094E1514B022283F825208FE14F4B8C
:10D308000022514C83F84C2083F82C2103F14C0166
:10D318004FF0FF351046A054013200232F2A41F860
:10D32800045FF8D1454A82F8253013629362137579
:10D33800434A1360434A13603F4A13606FE1454B09
:10D348001B7D980715D403F009FC10B90A232B702C
:10D3580065E1D4F803104FF00403B1F5006F05D26E
:10D36800364A82F82530C2F8301158E1384A13702D
:10D3780055E108232B7052E1304B002283F8252019
:10D388004DE1354B01221A70324A344B9178B0F591
:10D39800006F197003D2147D14F0010409D0002223
:10D3A8005A709A70DA701A715A719A71DA71197220
:10D3B80035E101A9FCF7F0FA284B9DF804201C720E
:10D3C8005A709DF805209A709DF80620DA709DF82D
:10D3D8000A201A719DF809205A719DF808209A713F
:10D3E8009DF80720DA710122D05C197A01324118C0
:10D3F800082A1972F8D112E163787BB9164A01211B
:10D4080011701449154A8978117015490968013352
:10D4180011F8010B082B9854F9D100E1012B40F0C9
:10D42800FE800522EA716B711F220723AA712B71F6
:10D43800F5E000BFE0530020E8530020204700201B
:10D44800405400205C540020BC4D0020EC530020C8
:10D458005454002004000020445400204554002067
:10D46800000000206E4B5B78032B00F2D880DFE8C9
:10D4780003F0020F1B206B4A6B4B92F82510D971F1
:10D48800117DD2F830219971110A59711A71C6E0CB
:10D49800644A654B92F82510D971117D126A997109
:10D4A800110A59711A71BAE0604B1A685E4B5A60DA
:10D4B800B5E05F4B1A685C4B5A60B0E0584B5A783D
:10D4C800002A40F0AC809978002940F0A88040F20A
:10D4D800D243984240F0A38040F2FF70FCF720FB53
:10D4E800FCF776FA0120FBF7FBFA98E06278514BDB
:10D4F800003218BF01221A70E2784F4B1A70494B5C
:10D5080093F834214D4B1A704D4A002313704D4A3D
:10D51800137084E0434B012283F835217FE066785D
:10D5280016B1012E1ED10FE0042240F2FB7003A9B0
:10D53800FCF7E4FBD4F80320039B9A4202D10123B1
:10D548006B606CE06E606AE0A3782A2B06D140F22B
:10D55800FB703D490422FCF740FB60E0324B03229C
:10D568001A705CE003232B7059E02D4B5B78032B7A
:10D5780042D8DFE803F00902313D2A4A0023D2F8F5
:10D58800381102F59C7224E0264BD3F83821092A79
:10D5980007D803EB82010132C1F83C01C3F83821F6
:10D5A8003DE0214B09221A7039E052F8044F8442B9
:10D5B8000ED1264A013902EB830203E05068013399
:10D5C80042F8040B8B42F9D3164BC3F8381126E006
:10D5D80001338B42E9D122E0124A0023C2F83831E4
:10D5E800194602F59E7299500433282BFBD116E098
:10D5F8000D4B0A225A6012E00B4B03221A700EE000
:10D60800FDF728FE0BE040F2D243984207D1054BC4
:10D61800012283F8642102E0034B02221A707FBDC5
:10D62800E05300202047002054540020405400209C
:10D638005C540020204D0020374D0020B24D0020C2
:10D64800364D0020EB4D0020E35300205C480020BD
:10D658003549002370B50B603449354A0B603549AC
:10D668003548136293620B60137582F84C3082F868
:10D678002C314FF0FF344C321946C15401332F2B53
:10D6880042F8044FF9D12D4B0020197B02F0B4FF6A
:10D698002B4B93F8283013B9FBF75EFA01E0FBF740
:10D6A80049FA002327491A465A500433B3F5806FC4
:10D6B800FAD1234B9B7E5BB1234D4FF4C3642919E8
:10D6C800204604220434FCF719FBB4F5CD6FF6D1DB
:10D6D8001B4BDC7E64B91B4E4FF4A76506EB840137
:10D6E800284604220134FCF709FB0435382CF5D10F
:10D6F800134A1379012B08D0112B05D0A3F121046B
:10D70800634243EB040300E00123094C84F86531CC
:10D71800537D13B1FAF7A4FF08B9002300E00123F1
:10D7280084F8253070BD00BF405400205C540020B0
:10D7380020470020E8530020BC4D0020544D002015
:10D748000400002060540020D84D0020F7B50F4E8B
:10D7580005460C4696E803008DE803000C496F4621
:10D76800C1F803300B4B8A7000220D704C701A7090
:10D77800FEF7ECF931787368074A82F866119DE87C
:10D78800030086E803001846FEBD00BF545400207D
:10D79800E05300204F54002020470020014B93F80D
:10D7A800660170472047002073B51F4D034602AA43
:10D7B8000C4695E8030002E9030059781B4A002645
:10D7C800117099785170D978917019799171597946
:10D7D800517199791171DB79D370154B1E70FEF771
:10D7E800B5F9144B1A7872B922702B786270A3704D
:10D7F8006B78E370EB792371AB7963716B79A37103
:10D808002B79E37109E0012A07D10B4A334612F854
:10D81800011FE1540133082BF9D1034B02AA12E985
:10D82800030083E803007CBD54540020E05300202B
:10D838004F54002044540020455400202DE9F04F57
:10D848009C4B99B01B789C4913B991F867316BB11F
:10D858009A4B1B78062B09D00A2B07D00F2B05D023
:10D868001F2B03D0944B002283F8342191F83431D4
:10D87800914A591EC9B201293DD8012B14BF08236A
:10D8880007238F498DF81C3092F868318D4AC86893
:10D8980012788DF81D30002308908DF81E30C2B91B
:10D8A8008B688DF82B208DF82430874B19788DF8EC
:10D8B800251059788DF82610D9798DF8271099797F
:10D8C8008DF8281059791B798DF829108DF82A3090
:10D8D8000AE0012A08D17D490DF123020133585C81
:10D8E800082B02F8010FF9D107A8FBF789FD0028DA
:10D8F80040F0AD80DBE3032B724922D192F86541F9
:10D90800002C7DD10B788BB96D4D6F4CA8786E7853
:10D9180023788619F6186378F618E379F618A37948
:10D92800F6186379F6182379F61817E0012B40F0FA
:10D938008E80664D605D0134FBF798FA092CF9D1A9
:10D9480085E0042B26D15E4D5F4CA8786E780023C5
:10D9580001228619637022706360B618FBF786FA95
:10D968006878FBF783FA2078FBF780FA6078FBF792
:10D978007DFAE079FBF77AFAA079FBF777FA607914
:10D98800FBF774FAF6B22079FBF770FA3046FBF72A
:10D998006DFA5CE0072B37D192F86531002B2FD157
:10D9A8000A781ABB464B9E785F78474B8DF84860DB
:10D9B8001D785C78BE19D8798DF84A50AD199979D7
:10D9C8008DF84B4064195A798DF84C0000191B7971
:10D9D8008DF84D1009188DF84E2052188DF84F30DB
:10D9E8009B188DF849708DF850302CE0012A2AD107
:10D9F800364A985C12A958540133092BF9D122E010
:10DA0800314801F085FA22E0082B20D12E4A002364
:10DA18000120537010705360294A8DF84A0091789C
:10DA280052788DF848108DF849208A1812188DF808
:10DA38004B308DF84C308DF84D308DF84E308DF8D8
:10DA48004F308DF8502012A80921FDF73BF8204BE4
:10DA58001B78002B00F08A801E4B1F4C1B78013B63
:10DA6800062B7ED8DFE803F004043A7D7D7D5D0057
:10DA7800134A1949936809788DF8343080238DF852
:10DA880035308A238DF8363000238DF837308DF8FD
:10DA980038308DF839308DF82D308DF82E30D36828
:10DAA8008DF83A100BA807218DF82C100C93FBF772
:10DAB800A7FC56E04E54002020470020E0530020E9
:10DAC80004000020445400205454002045540020F1
:10DAD800EB4D0020B24D0020364D00209D4D23789F
:10DAE800A8786E7886190A36F618FBF7BFF96878B1
:10DAF800FBF7BCF98020FBF7B9F98A20FBF7B6F9E8
:10DB08000020FBF7B3F90020FBF7B0F90020FBF782
:10DB1800ADF9F6B22078FBF7A9F93046FBF7A6F97C
:10DB28001FE08C4B22789878597880238DF855100F
:10DB380041180A318DF856308A238DF854008DF833
:10DB480057308DF85B200023521815A809218DF84D
:10DB580058308DF859308DF85A308DF85C20FCF724
:10DB6800B1FF7D4A002313707C4A13707C4C7D4AB8
:10DB7800002384F83431137084F8673194F86431E1
:10DB880013B10120FAF7ACFF94F83521744B52B168
:10DB980093F86521D2F1010238BF002283F865218C
:10DBA800002283F8352107A8FBF77AFC002842D029
:10DBB8009DF81C30062B3ED96B4B9DF82420089904
:10DBC8001A709DF825205A709DF826209A709DF8A5
:10DBD80027209A719DF828205A719DF829201A71DA
:10DBE8009DF82A20DA709DF81D205D4B83F8682186
:10DBF800584A1269914202D1012283F86721FAF743
:10DC080031FB5A4B00221860594B1A709DF81C20A2
:10DC1800534B072A14BF0222012283F8342193F8B8
:10DC28002520531EDBB2012B524B02D9052A40F0A6
:10DC3800E880002206E14A4C94F865512646002DFA
:10DC480073D10DF15F00FBF72BF900286DD0FBF7BE
:10DC580045F908B184F86951414B9DF85F0093F884
:10DC6800692199180132D2B2092A81F86A0183F828
:10DC7800692140F0ED80002283F86921354A93F844
:10DC88006A315178994207D092F82710002900F09C
:10DC9800DF808B4240F0DC8092F827209A4203D143
:10DCA8002F4B012283F8672100231A462C4C04F5D8
:10DCB800B571595C01335218082BD2B2F6D194F8D9
:10DCC800723193422DD1284B94F86B211A7094F835
:10DCD8006C215A7094F86D219A7094F86E219A719B
:10DCE80094F86F215A7194F870211A7194F871217F
:10DCF800DA70FAF7B7FA204B204A186094F8251022
:10DD080000231370032284F834214A1ED2B2012A58
:10DD180084F86931174A02D9052918BF01231370FD
:10DD280096E0042384F8343192E096F865310C4C7F
:10DD380033B30D4800F0A5FF10B3FAF793FA0E4B72
:10DD48000E4A186000231370032284F8342194F8D3
:10DD580025204EE004000020364D0020EB4D002029
:10DD68002047002044540020E0530020A44D002008
:10DD7800184D00204F540020AC4D0020B14D00201C
:10DD8800AA4E96F86541002C43D10FAD2846FCF702
:10DD9800C5FE00283DD023462A5D01349B18082C77
:10DDA800DBB2F9D19DF844209A422ED1A04B9DF8C0
:10DDB8003D201A709DF83E205A709DF83F209A70B9
:10DDC8009DF840209A719DF841205A719DF8422093
:10DDD8001A719DF84320DA70FAF744FA954B964A7F
:10DDE800186000231370914A072182F8341192F8C1
:10DDF8002520511EC9B201291946904B03D9052A7D
:10DE080001D001221EE0197022E0884B83F83441CA
:10DE18001EE096F82530854C013BDBB2012B17D864
:10DE2800236AB3F5006F0FD2FAF71AFC60B1206AC3
:10DE38007F49431C2362FBF7AFFD092384F8343183
:10DE48007E4B01221A7003E0784B002283F82520CC
:10DE5800764C94F82530042B234604D1744E32783E
:10DE6800110640F1F98093F834313BB1042B05D009
:10DE7800082B03D0062B01D0FDF768FE6B4C94F8F5
:10DE88003431092B40F0A780FAF7ECF96C4BA26803
:10DE98001B68801A0028B8BF4042984209D9694BCC
:10DEA8001A78012A01D102221A70FAF7DBF95F4BBE
:10DEB8009860FAF7D7F95D4A614BD2685B68801AB7
:10DEC8000028B8BF4042984209D95E4B5A78012AC7
:10DED80001D102225A70FAF7C5F9544BD860FAF703
:10DEE800C1F9524A564B12699B68801A0028B8BF7C
:10DEF8004042984209D9534B9A78012A01D102220B
:10DF08009A70FAF7AFF9494B1861484B93F84C20CF
:10DF1800002A60D093F82C1100295CD14A4A93F862
:10DF280028A11268D3F80C910192484AD3F81081BD
:10DF380012681C6A0292464AD3F814C11268D3F8D0
:10DF480018710392DA69187D04929A69D3F81C61F2
:10DF5800D3F82051D3F824B10592CDF800A00A4691
:10DF6800DFF8E0A01AF80230022B1BD1DFF8E4A09A
:10DF78005AF82230B3F1FF3F0FD0D1B206460091D4
:10DF8800A446DDF814B0049D039F1C46DDF8088004
:10DF9800DDF804900121002004E0DFF8A8A00023A8
:10DFA8000AF8023001322F2ADAD1204B009AC3F83E
:10DFB8000C91C3F810811C62C3F814C1C3F818711E
:10DFC8001875C3F81C61C3F82051C3F824B183F84D
:10DFD800282183F82C11154A92F83431092B06D1DF
:10DFE80092F82530022B02D1052382F82530D2F889
:10DFF80038110E4B00295AD093F83421092A56D1EA
:10E0080093F82520012A52D1186A002203F59C733F
:10E0180053F8044FA04204D1044B052283F825206D
:10E0280045E001328A42F3D141E000BF2047002099
:10E03800E0530020AC4D0020B14D00204F5400208B
:10E04800784D0020BC4D0020405400205C54002036
:10E05800E85300207047002094F834313BB3042B78
:10E0680025D0082B23D0062B21D0124DD4F830010F
:10E078006A70D6F80330B0F5006F6B6012D2314683
:10E08800FBF788FDD4F830013146FBF7EFFC30B1DF
:10E09800D4F830310133C4F83031652300E0072368
:10E0A8002B7004E007232B70002384F8253019B067
:10E0B800BDE8F08F54540020704710B5FAF7D2F835
:10E0C800074C2368C01AB0F5FA7F07D9054B5A697F
:10E0D80082F040025A61FAF7C5F8206010BD00BF0F
:10E0E800605800200010024008B5FAF7DDFC014B2B
:10E0F800586008BD545400207047704770477047F7
:10E1080070477047704700BF2DE9F041A74B0446A0
:10E118005B7E5BB902F060FA061C204618BF012638
:10E1280002F062FA003018BF01200CE002F054FA45
:10E13800D0F10106204638BF002602F055FAD0F18A
:10E14800010038BF00209A4B03EB44131B7A03F0FD
:10E158007F0513F0800F974B1B6907D013F4806F6E
:10E1680014BF4FF000084FF0010801E0C3F3802806
:10E178006B1E072B00F2DD81DFE813F008000800B2
:10E1880008000800EA00EA00EA00EA008A4F3B5D5E
:10E19800013B0E2B00F2CD81DFE813F00F002900C0
:10E1A8002F003A0040004800530064008800A70090
:10E1B800AB00CB01C600CD00B201204602F072F9D7
:10E1C8007B4B07EB840703EB44135B7B023D7860D2
:10E1D8000121BB602046EDB202F0BCF8012D764E5D
:10E1E80001D8022300E004233355BDE8F081704ACA
:10E1F8006301D11802204873F0E0002800F09981EB
:10E20800204602F029F96D4B43F82400042380E1ED
:10E21800674A6301D1180120487303E1002E00F01A
:10E228008881204602F0CEF9062372E1604B002176
:10E2380003EB441359732046596801F0C9FF0722BC
:10E2480021E1002E40F075812046314601F0C0FFE3
:10E25800574B204603EB44135968494201F0B8FF75
:10E26800082210E1002E00F06481204602F0F4F844
:10E2780000210646204601F0ABFF504B002553F81D
:10E2880024202046921B43F82420494B03EB4413D7
:10E2980059685D7302F03EF82046314601F0F2FFFE
:10E2A8002046294602F056F80922ECE0204602F002
:10E2B8003FF9002800F03D810021204601F088FF49
:10E2C800033D0121204602F045F8EDB2002002F09E
:10E2D80041FB012D07D82046012102F03BF8344BC1
:10E2E80003EB4413C9E00E22CDE0002E00F021819B
:10E2F800D6E0002E40F01D81204602F0ADF83146F0
:10E308000546204601F064FF294B022103EB441324
:10E318005E7395FBF1F1204601F0B4FF20463146CB
:10E3280002F018F80D22AEE0204602F001F90028AC
:10E3380000F0FF80ECE007EB84031D4A996802EBCC
:10E34800441251732046596801F0E4FF0023E0E0CD
:10E35800194F3B5D013B0E2B00F2EB80DFE813F019
:10E368000F003000440054006900E9007A00E90019
:10E37800E9009700A2008500C500DC00D000204617
:10E3880002F090F80A4B07EB840703EB44135B7B1E
:10E3980078600121BB60204601F0DCFF062D01D02A
:10E3A800082D01D102226EE004226CE00400002056
:10E3B800544D0020000C0240944800201C4D0020C1
:10E3C800062D5D4B4FEA441202D19A18022103E050
:10E3D800082D02D19A1800215173620199582046DC
:10E3E80001F0F6FE03224EE06B1FDBB2012B05D8CD
:10E3F80020B1062D514B26D1042245E0B8F1000F7B
:10E4080000F097800C2384E0052D4B4B4FEA441213
:10E4180002D19A18012103E0072D02D19A18002190
:10E428005173620199582046494201F0D1FE0522F4
:10E4380029E06B1FDBB2012B07D836B1052D3F4B06
:10E4480001D1022220E00F221EE0B8F1000F70D0A7
:10E4580007235EE0B8F1000F6BD1374B022203EBC4
:10E4680044135A73204659680AE0B8F1000F60D186
:10E47800314B012203EB44135A7359682046494231
:10E4880001F0A6FE0A222D4B1A55BDE8F081B8F11D
:10E49800000F4ED0204601F0DFFF07EB8403D86061
:10E4A8000B2336E0B8F1000F43D1204601F0D4FF2A
:10E4B800214B224D03EB44135968064683F80D801F
:10E4C800204601F027FF05EB8403D968022376185C
:10E4D80096FBF3F1204601F0D5FE2046414601F0B7
:10E4E80039FF0D232B55BDE8F081204602F020F8B6
:10E4F800F8B10E2300203B55BDE8F04102F02ABADE
:10E508002046012101F026FF2046002101F060FE8F
:10E518000E233B55BDE8F08107EB8403064A996852
:10E5280002EB441251732046596801F0F3FE0023B0
:10E538003B55BDE8F08100BF544D002094480020B1
:10E54800024B1A5C0AB901221A54704794480020F9
:10E55800024B1A5C0AB10F221A54704794480020E3
:10E56800014B185C704700BF94480020034B002003
:10E578001870034B997AF9F751BF00BFB34D0020CB
:10E58800544D0020014B1878704700BFA448002064
:10E59800014B5878704700BFA4480020014B987879
:10E5A800704700BFA44800202DE9F3416E4BDA788C
:10E5B80022B96FF000425A600122DA701C7A5CB905
:10E5C800E0B2F9F78CFF684B03F10902A05401345B
:10E5D800082CF5D101221A72644FDFF8B081644E1D
:10E5E80027240025E8B2F9F77AFFEB5D834216D0BD
:10E5F800AB1CE85508EB83035B68022B05D0032BA3
:10E6080008D0012B0BD150B104E040B9325D012A8A
:10E6180005D103E0335D012B01D1022333550135C8
:10E628000134082DDED1534C637E23B94E4B587C00
:10E6380001F0D2FF30B9637E4B4C7BB1607C01F0B6
:10E64800CBFF58B9484B9A7C52B901229A74484B6F
:10E65800DA7E012A04D10222DA7601E00023A374CB
:10E66800444C637E23B9404B587C01F0BDFF30B960
:10E67800637E3D4C7BB1607C01F0B6FF58B93A4BE4
:10E68800DA7C52B90122DA74394B1A7F012A04D193
:10E6980002221A7701E00023E374364EF36993B13E
:10E6A800354C25787DB9F9F7DDFD344B1B68C01A68
:10E6B800F3690028B8BF4042984204D9284601F0BF
:10E6C80081FF012323702B4E336A93B12C4C25789C
:10E6D8007DB9F9F7C7FD2B4B1B68C01A336A0028B0
:10E6E800B8BF4042984204D9284601F06BFF012385
:10E6F80023700820FBF7A8F863281B4C01D80123D6
:10E7080005E00820FBF7A0F8692801D90023637009
:10E718000820FBF799F840F212239842124C01D9CD
:10E72800012306E00820FBF78FF8B0F5027F01D23D
:10E73800002323700920FBF787F878280A4C01D9B1
:10E74800012305E00920FBF77FF8592801D80023A9
:10E75800A3706178044A0C4B19B9117809B99278F9
:10E76800B2B104221A8315E0A4480020AD48002065
:10E77800BC4D002004000020B14D0020AC4D00200D
:10E78800184D0020A44D002000100240784D0020B4
:10E7980004225A835C4C02F0EFF9607C01F0A0FE81
:10E7A8000146607C002942D0584B02221A54FBF7DC
:10E7B800E7FE637C564A02EB4312517AB0EBD10F65
:10E7C80002D01846F9F72AFE4F4C00232375607CC7
:10E7D80001F0AEFE70B1627C4E49D31CC85C0128C2
:10E7E80001D10220C854012101FA02F2464B197DD9
:10E7F8000A431A754849494A0B7843B14248007D93
:10E80800034204D11370464B1B7803B90B7013787D
:10E818003BB13D4A127D1A409A4202D1414B012236
:10E828001A70002002B0BDE8F041FFF76DBC384D0A
:10E838003D4F05EB401393F80CE03C4A83003C4EF7
:10E84800BEF1000F08D0121800923618FB180A46BD
:10E858000196FBF723FF7AE1F9181218331801F033
:10E8680055FE607C01F0B6FD30BBF9F7FBFC637C1C
:10E878000A2104EB8304626805EB4315801AAA8B0E
:10E888000028B8BF40424A43904271DD1F4AD25C1B
:10E898001AB9284AD25C002A6AD01D4A184602EBE7
:10E8A8004312917AF9F7BAFD174B18495B7C00229D
:10E8B800CA542049CA545BE0607C05EB4013DB7FF7
:10E8C800002B39D001F086FD0646607C01F06AFD18
:10E8D8000E4A8642607C174B125C0DD0032A02D187
:10E8E8001B5C002B3AD005EB4015E97FF9F796FD44
:10E8F800054B03215B7C2FE0022A01D11B5C6BB323
:10E9080005EB4015697A22E0A4480020B34D0020A9
:10E91800544D0020BC4D0020374D0020364D0020BE
:10E92800204D0020EB4D0020384D0020284D0020C0
:10E93800514D0020B04D0020864B1B5C022B02D1AC
:10E94800854B1B5C53B1854B03EB4013597AF9F7A0
:10E9580065FD834B02215B7C7E4AD154804C7E4B03
:10E96800657C00225A55F9F77DFC04EB850460604C
:10E978007B4C7A4D607C05EB40139B69E3B1F9F75A
:10E9880087FEC8B1607C01F025FD637C0028B8BF14
:10E99800404205EB4315AA6990420DD9184601F08B
:10E9A80011FE637C6F4A0121D1546F4A0F33D15C49
:10E9B800012901D10221D154694C00232375607CBF
:10E9C80001F0B6FD70B1627C6749D31CC85C0128B0
:10E9D80001D10220C854012101FA02F2604B197DCD
:10E9E8000A431A756149624A0B7843B15C48007D55
:10E9F800034204D113705F4B1B7803B90B70137873
:10EA0800574A33B1117D1940994202D15A4B01211D
:10EA18001970507C01F0DEFC514C18B9607C01F093
:10EA2800C1FC18B1657C554B5B5D2BB3637C4B4ACD
:10EA380002EB4312D28912B9504AD35C13B3F9F7E7
:10EA480011FC474C0A21637C04EB83029269801A0B
:10EA5800424A0028B8BF404202EB4312D2894A43D7
:10EA680090420FDD464DEA5C62B91846FBF77EFE20
:10EA7800637C0122EA5405E0F9F7F4FB384B03EB19
:10EA88008505A861364C3F4D607C01F0A3FC024629
:10EA9800607C002AB8BF524255F830309A420AD2F8
:10EAA800FBF73CFD637C05EBC3056A7982420DD117
:10EAB8001846002108E0FBF731FD637C05EBC30530
:10EAC8006979884202D01846FBF700FDF9F7CAFBBE
:10EAD800234CE369C01A0028B8BF40420A2836DD33
:10EAE800607CFFF711FB607C01F074FC20B3607C54
:10EAF8001A4D05EB40135B69002B1DDD01F0ACFCE2
:10EB08000646607CF9F7CEFD637C361A05EB4315A3
:10EB18006A69002EB8BF764296420DDD184601F0AC
:10EB280051FD637C184A0121D1540F4A1533D15C39
:10EB3800012901D10221D154094C637C0133DBB294
:10EB480063740BB100236374F9F78CFBE06102B0C6
:10EB5800BDE8F081B34D0020B04D0020544D002099
:10EB6800A4480020504D0020BC4D0020374D002007
:10EB7800364D0020204D0020EB4D0020B44D0020E4
:10EB8800B54D00202C4D0020354D0020084B18684D
:10EB9800024604E02C2902D100221A7004E0117800
:10EBA800134601320029F5D1014A01331360704739
:10EBB800C448002070B50646FAF772F90D4C0546B0
:10EBC80018B100232371012070BDA368E268934245
:10EBD80007D2E218127C013301203270A360207141
:10EBE80070BD04F11000FBF787FFA560E0602846C0
:10EBF80070BD00BFC448002010B50C4C0A462379EC
:10EC08001BB9BDE81040FAF731B9236DE11881F856
:10EC18005400591C0D28216502D03F2900D822B97B
:10EC28000348FBF74FFF0023236510BDC4480020AD
:10EC38001849002010B50121044686B02020FFF7AE
:10EC4800DBFF002C04DA2D200121FFF7D5FF6442F9
:10EC580000230A2100E0034694FBF1F201FB124471
:10EC680001A830341C54581C141EF4DC1C4601AB9B
:10EC7800E05C0121FFF7C0FF14F1FF34F7D206B0C2
:10EC880010BD2DE9F74304460DF10700FFF792FF89
:10EC9800002800F0C380934B934A93F8941019BB53
:10ECA80051789DF80700403188420DD1D3F898106B
:10ECB800002940F0B380012183F89410117931F0D4
:10ECC800010140F0AB80A7E00D2801D01B2802D13C
:10ECD8000022844B05E0D3F898207E2A00F29E801B
:10ECE8000132C3F8982099E0117931F0010103D17C
:10ECF8009DF80700FFF780FF9DF80730794D1F2B1F
:10ED08000AD9D5F898207E2A77D8A918013281F82F
:10ED18009C30C5F8982070E0082B07D1D5F89830BA
:10ED2800002B6AD0013BC5F8983066E00D2B64D102
:10ED3800D5F89830002B60D06B4B1A79112A16D170
:10ED4800587801214030C0B2FFF756FF002605F180
:10ED58009C0704E0F05D0121FFF74EFF0136D5F86E
:10ED680098309E42F6D30D200121FFF745FF5D49FB
:10ED78000023C1F81C31D1F898700D681A4618465E
:10ED880001F590789C4627E001280DD002D302288F
:10ED980021D117E0554E965D202E1CD0C81880F85A
:10EDA80020610133012016E0504E965D202E0DD1D2
:10EDB800012B03D9C81880F820C1013308EB0305DB
:10EDC800022008E0494E965D202E04D001EB03098D
:10EDD80089F8206101330132BA42D5D1414A002174
:10EDE800C2F81C31D31883F820110123156082F86A
:10EDF8009F3182F89410C2F898109DF807301B2BA9
:10EE08000CD1384B0021C3F8981083F89410364B76
:10EE18001B79012B02D10D20FFF7EEFE314B93F841
:10EE28009F01002858D00026DFF8E08083F89F6112
:10EE380035464FF0070909FB05872D48394608F084
:10EE480011FE28B9BE797B79F107237034D508E023
:10EE580016F80830002B41D001350736FF2DEAD1CE
:10EE68003CE0FFF793FE23780546042B0BD121499C
:10EE780008F0F8FDF8B128461F4908F0F3FD68B11D
:10EE880028461E490EE00D2B13D11D4908F0EAFD56
:10EE980088B128461B4908F0E5FD08B9012305E0BB
:10EEA8001949284608F0DEFD10B90223637003E013
:10EEB800284608F0BDFD6070B20704D5FFF766FE6E
:10EEC80008F0B6FDA070730705D5FFF75FFE08F0E0
:10EED800AFFDC4F803000120BDE8FE8300232370C2
:10EEE800F9E700BFC4480020040000206049002062
:10EEF800E449002065990108699901086D9901089C
:10EF080073990108799901087E990108A883010875
:10EF180038B50C4D0446A87801214030C0B2FFF73F
:10EF28006BFE687801214030C0B2FFF765FE20789B
:10EF3800FFF780FE6068FFF77DFE0D200121BDE828
:10EF4800384059E60400002003464FF6FF7083421C
:10EF58004DDDB3F1807F27DBB3F1805F11DBB3F1C7
:10EF6800804F08DB394A93426FDC394A191652F848
:10EF78002120120212E0364A991552F82120D201B6
:10EF88000CE0B3F1806F324A04DB191552F82120E6
:10EF9800920103E0991452F821205201511C93FB6D
:10EFA800F2F28A1852101CE0B3F5801F284A0CDBD5
:10EFB800B3F5800F04DB191452F82120120110E078
:10EFC800991352F82120D2000BE0B3F5802F04DB0F
:10EFD800191352F82120920003E0991252F82120C7
:10EFE8005200501C93FBF2F2801840101EE0FF2BD9
:10EFF80022DDB3F5805F164A0BDBB3F5804F03DBE8
:10F00800191252F8210010E0991152F8210040100D
:10F018000BE0B3F5806F04DB191152F82100801062
:10F0280003E0991052F82100C010013000FB00F2F3
:10F038009A420ADD01387047002B04DB044A52F873
:10F048002300001170474FF0FF3070470080FE7FAB
:10F05800888401081D4B5A7E1D4BD2B9597BCB07BA
:10F0680009D51C4B1B69180705D51B4B18680028C8
:10F07800BCBF1A605A608B0726D5164B1B69D80689
:10F0880022D5154B1A68002A1EDD00221A605A6024
:10F0980070475A7BD1070AD50E4B196911F0080140
:10F0A80005D10D4B18680028BCBF1960596093073B
:10F0B8000AD5084B1A6912F0100205D1064B1968D7
:10F0C8000029C4BF1A605A60704700BF04000020BE
:10F0D800544D002000040240644A002038B51A4B01
:10F0E80005461A7A62B1FBF74FFB184B2846597A46
:10F0F800F9F794F9164A00231370164A137038BDAD
:10F108005A7A12B1012A1DD10FE01C68D4B9DA6805
:10F118001B699A4216D0FBF737FB0C4B2846597AE5
:10F12800F9F77CF90A4B1C7038BD1C6854B95B6947
:10F1380043B1FBF729FB054B2846597AF9F76EF9D5
:10F14800034B1C7038BD00BF644A0020544D00209A
:10F15800B54D00207858002008B50020FBF786FA46
:10F16800A8B9FBF70DFA013006F0AAFA14A3D3E9FF
:10F17800002306F00BFB14A3D3E9002306F030FCB0
:10F188000022154B06F002FB06F09AFD08BD002090
:10F19800FBF7F6F9013006F093FA0DA3D3E9002343
:10F1A80006F0F4FA08A3D3E9002306F019FC0022BC
:10F1B800094B06F0EBFA06F083FD08BDAFF30080BB
:10F1C80049922449924CB1401B0DE02D90A0F63F86
:10F1D80024499224496AA2400000A03F684620F0D2
:10F1E80007018D4631B5194CA36973B1184801213F
:10F1F80003F0C8FB0028F9D01548A56903F089FB7E
:10F20800C5F10305C0B264192077104CA369022B1D
:10F218000BD8A3690E48C3F10202A218013392F871
:10F228002010A36103F078FB0CE00022084871214C
:10F2380003F09AFB074B10221A83002384F824302A
:10F2480084F82530BDE8314085467047644A00207F
:10F258000030014000000240684620F007018D465A
:10F268002DE9F14F012184B04FF0804004F0ADF852
:10F27800002800F0FF8601214FF0804004F0B0F82C
:10F28800914B9A6A122A10D9012283F82C20002265
:10F298009A628E4B1A6801321A608D4B1B783BB903
:10F2A8008C4B1A6801321A6002E09A6A01329A623B
:10F2B800854B1A6B22B1012283F83420002201E029
:10F2C8001A6B01321A630020F9F790FB0020F9F756
:10F2D800E9F90390039B7C4CA36394F82C30002B32
:10F2E80060D07B4B1B78002B48D0039AE36BD31A72
:10F2F800002BB8BF5B42082B764B26DD1968226CC1
:10F30800914222D0039A62641B68A364606CE36B29
:10F31800A76CC01A06F006FE266C0546B81B06F058
:10F32800FDFD0146284606F005FF06F0DBF964A35B
:10F33800D3E9002306F02AFA06F0C2FC664B1860EF
:10F34800636CE363A36C23640CE019685E4B1A6C6E
:10F358008A1A002AB8BF5242642A03DD5E49002295
:10F368000A60DA64584B5C4AD96CD86C1268821A05
:10F37800102092FBF0F28A1ADA6413E0534A1268FA
:10F38800642A554A05DD1360E364544B08221A8049
:10F3980008E0E16CE06C13681022C31A93FBF2F3E7
:10F3A800CB1AE364484C237A062B00F0F98094F8D2
:10F3B8003420002A00F0FA85032B00F0F785637AE1
:10F3C800002B35D1E2682369D31A236594F85430A9
:10F3D80013B9A36DE3650EE0E0682369C01A00283D
:10F3E800B8BF4042FFF7B0FD0546206E4000FFF76A
:10F3F800ABFD4543E565344BD9681A69914207DD91
:10F40800D96D9A6D9142B4BFDA6D9A6D5A6112E066
:10F41800D9681A69914207DAD96D9A6D9142B4BFD9
:10F42800DA6D9A6D5242F1E700225A611A6002E0E1
:10F438006FF000432365244B19685A6991427DD0C7
:10F44800596E1A6E8A185A665A6E12149A66596E4E
:10F458009A6E12048A1A5A6693F854200AB95A699D
:10F468001A60194B19685A69914209DA1868996E35
:10F478005A694118914211DA1A689B6ED3180EE046
:10F4880019685A6991420CDD1868996E5A69411ACF
:10F49800914203DD1A689B6ED31A00E05B690A4A41
:10F4A8001360094BDA6E002A4BDD5A69C2B9186835
:10F4B800D96E0028B8BF4042884242DA1CE000BF3B
:10F4C8000000000000408F40644A0020745800206B
:10F4D800FA4B0020705800206C58002082580020F9
:10F4E8005A69002A1A4613DD1968002906DD1868CA
:10F4F800D96E884202DADA6E1A6022E01268A14BED
:10F50800002A1EDA1968DA6E5242914219DDF2E7D2
:10F518005969002915DA1968002904DA1868D96EBA
:10F528004942884207DC1268964B002A09DD1968AF
:10F53800DA6E914205DADA6E5242DDE700225A6647
:10F548009A66904C8F4D226F2368D3182367236FD8
:10F558001B146367626F236D002AB8BF5242002BE9
:10F56800B8BF5B429A42C4BF236D6367226F636F63
:10F578001B04D31A23672269636FD3182361FFF72B
:10F5880069FDA36F062B05D8EA6F696FAB6F01FAA7
:10F5980003F301E0EB6F6A6FD318EB6700F006BD69
:10F5A80094F82C30002B3ED0E26CD4F88030002A3E
:10F5B800B8BF52429A4233DDD4F88400E36CD4F8E1
:10F5C8008050002BB8BF5B425B1B4343D4F88810C4
:10F5D800D4F880208A1A93FBF2F3C4F88C30E36CD9
:10F5E800002B04DAD4F88C305B42C4F88C30654BBD
:10F5F800D3F88C10D3F884209142C4BFD3F8842068
:10F60800C3F88C20D3F88C10D3F884305D4A5B4261
:10F61800994208DAD2F884305B42C2F88C3002E0B2
:10F628000023C4F88C30574B93F83420002A00F09C
:10F638003583554A1578002D40F0D4825A7A022A2B
:10F6480000F06B82D3F890109A6D914256DDD3F892
:10F658009410D3F89820891A4C4A11605B68002BE3
:10F66800134602DA126852421A601A68002A02DA4D
:10F67800464A002111601968424BD3F89C209142F8
:10F6880002DA424A00211160404A1268D3F8A030D9
:10F6980082FB0323002A73F1000104DAFF20002112
:10F6A800121843EB0103120A42EA0362354BD3F8FE
:10F6B80090509B6DED1A364BAA425B69D8BF22EA7F
:10F6C800E275002B1ADD314A12689A4216DD2D4B7D
:10F6D80000225A611A60C3F8A4205A60D3F898200F
:10F6E800C3F89420D3F89820DA602A4B01221A70C4
:10F6F800294B5A7D012A01D102225A75214C637A7D
:10F70800002B4FD1E268D4F89830D31A236594F8C7
:10F7180054301BB9A36D5B19E3650FE0E068D4F8BA
:10F728009830C01A0028B8BF4042FFF70DFC0646C3
:10F73800206E4000FFF708FC4643E665114BD96888
:10F74800D3F89820914209DDD96D9A6D52199142EA
:10F7580001DADA6D0EE09A6D551910E0D968D3F820
:10F76800982091421ADAD96D9A6D5219914203DAAA
:10F77800DA6D52425A6118E09A6D55196D425D6111
:10F7880013E000BF644A0020785800206458002025
:10F79800544D0020354D0020BC4D002000225A61F8
:10F7A8001A6002E06FF000432365924B19685A69AA
:10F7B80091426CD0596E1A6E8A185A665A6E121493
:10F7C8009A66596E9A6E12048A1A5A6693F85420E9
:10F7D8000AB95A691A60874B19685A69914209DA55
:10F7E8001868996E5A694118914211DA1A689B6E25
:10F7F800D3180EE019685A6991420CDD1868996EA1
:10F808005A69411A914203DD1A689B6ED31A00E0C7
:10F818005B69784A1360774BDA6E002A3ADD5A69D9
:10F828003AB91868D96E0028B8BF4042884231DA20
:10F838000BE05A69002A1A4613DD1968002906DD0B
:10F848001868D96E884202DADA6E1A6022E0126805
:10F85800684B002A1EDA1968DA6E5242914219DDA5
:10F86800F2E75969002915DA1968002904DA1868D5
:10F87800D96E4942884207DC12685E4B002A09DDCE
:10F888001968DA6E914205DADA6E5242DDE7002233
:10F898005A669A66574B574C196F1A688A181A672E
:10F8A8001A6F12145A67596F1A6D0029B8BF494266
:10F8B800002AB8BF52429142C4BF1A6D5A67196FE5
:10F8C8005A6F12048A1A1A67D3F898105A6F8A184E
:10F8D800C3F898205B7A002B42D1E268D4F89430C0
:10F8E800D31AC4F8A83094F854301BB9A36DC4F8DF
:10F8F800AC3010E0E068D4F89430C01A0028B8BFE3
:10F908004042FFF721FB0546206E4000FFF71CFB35
:10F918004543C4F8AC50374BD968D3F8942091428A
:10F928000ADDD3F8AC109A6D9142B4BFD3F8AC207D
:10F938009A6DC3F8A42017E0D968D3F894209142AF
:10F9480009DAD3F8AC109A6D9142B4BFD3F8AC2061
:10F958009A6D5242EDE70022C3F8A4205A6003E0F2
:10F968006FF00043C4F8A830224B5968D3F8A4209C
:10F97800914200F08480D3F8B0101A6E8A18C3F848
:10F98800B020D3F8B0201214C3F8B420D3F8B010C4
:10F99800D3F8B42012048A1AC3F8B02093F854207C
:10F9A80012B9D3F8A4205A60124B5968D3F8A4208E
:10F9B80091420CDA5868D3F8B410D3F8A42041184F
:10F9C800914219DA5A68D3F8B430D31816E0596856
:10F9D800D3F8A420914213DD5868D3F8B410D3F8B3
:10F9E800A420411A914207DD5A68D3F8B430D31ADB
:10F9F80004E000BF644A0020D3F8A4308E4A536064
:10FA08008D4BDA6E002A3FDDD3F8A4203AB9586846
:10FA1800D96E0028B8BF4042884235DA0CE0D3F8E6
:10FA2800A420002A1A4613DD5968002906DD586803
:10FA3800D96E884202DADA6E5A6025E052687E4B47
:10FA4800002A21DA5968DA6E524291421CDDF2E747
:10FA5800D3F8A410002917DA5968002904DA58687D
:10FA6800D96E4942884207DC5268734B002A0BDD85
:10FA78005968DA6E914207DADA6E5242DCE7002200
:10FA8800C3F8B020C3F8B4206B4CD4F8B82063682E
:10FA9800D318C4F8B830D4F8B8301B14C4F8BC3044
:10FAA800D4F8BC20D4F8A830002AB8BF5242002BA2
:10FAB800B8BF5B429A42C4BFD4F8A830C4F8BC307F
:10FAC800D4F8B820D4F8BC301B04D31AC4F8B83022
:10FAD800D4F89420D4F8BC30D318C4F89430FFF785
:10FAE800B9FAD4F898202369D31AC4F8C030226927
:10FAF800D4F8C030D318236123690399039AFF32DD
:10FB0800934204DCA1F1FF029A42B8BF1A464A4B5D
:10FB18001A611A69C3F898206EE0D3F8C420002A45
:10FB280001DDFF2205E0D3F8C420002A04DA6FF0D3
:10FB3800FE02C3F8C02001E0C3F8C0503F4B597E15
:10FB48003F4B5B7BC9B9DE070AD53E4A12691507E8
:10FB580006D5394AD2F8C4000028B8BFC2F8C01088
:10FB68009C0726D5374B1B69D80622D5324BD3F8CC
:10FB7800C420002A1DDD002219E0D9070BD5314A1F
:10FB8800126912F0080106D12B4AD2F8C4000028E5
:10FB9800B8BFC2F8C0109A070BD52A4B1B6913F0DF
:10FBA800100206D1244BD3F8C410002901DDC3F894
:10FBB800C020214B1969D3F8C0208A181A61196925
:10FBC8000398039AFF32914204DCA0F1FF028A42B3
:10FBD800B8BF0A461A611A69DA601A69C3F8982028
:10FBE8001A6907E000225A611A60C3F8A4205A6013
:10FBF800D3F89820C3F894200F4B134ADC68106898
:10FC08000399201A884227DA0399D868126882185B
:10FC1800914221DA0D4A1168002903DD1368013B7E
:10FC2800136020E00A4901220A70D3F89410DB68B7
:10FC3800994218D1074B15E0644A002004000020BF
:10FC4800544D0020000402408458002068580020C9
:10FC58008058002078580020BF4B1A68BF4B1A60A4
:10FC6800BF4B00221A70BF4BBF4A0398DC6811686B
:10FC7800611A884205DB0399D86812688218914294
:10FC880002DDBA4A002111705B7A012B03D0B54B13
:10FC98005B7A022B02D1B54B00221A70B14A039944
:10FCA8001369C2F8C830B14B187820B1B04B1C6842
:10FCB800B04B186800E00A24D2F8C860D2F8CC50DB
:10FCC800A84B75196D1AC2F8D050D2F8D050C2F8A6
:10FCD800D450D2F8D050D2F8D820002DB8BF6D42F9
:10FCE800954232DCD3F8D02042B3D3F8D060D3F8B1
:10FCF800D0507443D3F8DC200A26AA1A94FBF6F4F1
:10FD080000FB0240C3F8D400D3F8D400D3F8D820BD
:10FD18009042C4BFD3F8D820C3F8D420914BD3F86D
:10FD2800D400D3F8D8205242904204DAD3F8D8202D
:10FD38005242C3F8D420D3F8D42001E0D3F8D0201D
:10FD48008918C3F8E010874B15E0D3F8D000D3F832
:10FD5800D8205242904203DAD3F8D820891A08E012
:10FD6800D3F8D000D3F8D82090420DDDD3F8D820AE
:10FD78008918C3F8E010D3F8E010D3F88C208A185B
:10FD88009205920DC3F8E420764CD4F8D03026467C
:10FD9800C4F8DC30D4F8E430E367637A022B32D15C
:10FDA800FFF7DAF9D4F8C43005468342C8BFC4F86F
:10FDB800C400D4F8C42043429A42B8BF694A694C87
:10FDC800B8BFC2F8C430D4F8C4000028B8BF404255
:10FDD80006F0A8F80646284606F0A4F8014630467C
:10FDE80006F0A8F905F07EFC59A3D3E9002305F035
:10FDF800CDFC05F065FFFF28A8BFFF20C4F8E80088
:10FE0800C4F8EC00D2E0D4F8F030002B00F0CA803F
:10FE1800D4F8F430D4F8F80023B1D4F8FC30D4F88E
:10FE2800D4B003E0D4F8FC30D4F8D0B00130C01A14
:10FE380006F078F8D4F80061BBF1000FB8BFCBF139
:10FE4800000B0546C6EB0B0006F06CF8D4F804A1CD
:10FE5800D4F8F8700646C7EB0A0006F063F8D4F841
:10FE68000891D4F800810746C8EB090006F05AF853
:10FE78000146384606F05EF90146304606F0A6F817
:10FE88000146284605F09AFF06F0F0F9354BC4F80C
:10FE9800E800D3F8E810D3F8F8209142BCBFD3F8B3
:10FEA800F820C3F8E820D3F8E800D3F804112D4A65
:10FEB8008842C4BFD2F80411C2F8E810D3F80C3154
:10FEC800284A002B04DDD2F80C31013BC2F80C3172
:10FED800244AD2F81031002B04DDD2F81031013B4E
:10FEE800C2F81031D2F8E810D2F8EC201D4B91423C
:10FEF8001DDDD3F814211AB3D3F80C21002A55D1EB
:10FF0800D3F8EC10D3F8FC208A18C3F8EC20D3F807
:10FF1800EC10D3F804219142C4BFD3F80421C3F8EC
:10FF2800EC20104BD3F81421C3F80C213EE0D3F891
:10FF3800E810D3F8EC20914238DAD3F81821DAB96E
:10FF4800D3F8E820C3F8EC2030E000BFAFF300801E
:10FF58000000000000E06F407C5800206858002036
:10FF680080580020644A00208858002078580020D3
:10FF78009458002090580020D3F81021B2B9D3F833
:10FF8800EC00D3F81C11884204DBD3F8EC10D3F84A
:10FF98001C218A1AC3F8EC20394BD3F81821C3F86E
:10FFA800102103E0D4F80431C4F8EC30344B93F852
:10FFB8002520002A58D193F82021002A54D193F8FB
:10FFC8002420002A40D19A6F062A07D8DA6F2D49D3
:10FFD800920501EB1252D2F800240CE09A6FD96F07
:10FFE800072A294A01F00F0102EB81020CBFD2F85F
:08FFF8000823D2F848231A6225
:020000040801F1
:10000000214B1A7A062A26D193F8202001920199D1
:10001000D3F8EC205143FF22B1FBF2F10191196AB0
:100020004908196293F8211002910298D3F8EC1054
:100030004143B1FBF2F20292029AD2B283F821203C
:100040001A6A52001A62019AD2B283F8202002E0A2
:10005000D3F824211A620F4B10225A830A4B002135
:10006000012283F825200C489961712102F080FC5F
:10007000054B002283F82C2083F8342004B0BDE81F
:10008000F14F8546704700BF644A0020888401080C
:10009000809501080000024000300140F8B5464B51
:1000A000464A5D6AA3F570435B6A00211360444BC6
:1000B0001960444B42F210711E881068B6B2884233
:1000C00007DD198889B2082903D91988C1F34E01BF
:1000D00019801368B3F57A7F0ADA3A4B1A8892B21C
:1000E000B2F5804F04D21A8892B2520092B21A80AE
:1000F000314C0821204603F06CF998B12F4B204673
:100100001A68082152421A6003F06EF92D4B1A88C2
:1001100092B2AA1AE2631B8801229BB2EB182364F5
:10012000294B9A82244C1021204603F052F978B1D1
:100130002046102103F058F9224B1A8892B2AA1ACD
:10014000E2631B8801229BB2ED181F4B25649A8243
:100150001A4B30461C6805F0E9FE05F0C7FA14A3F7
:10016000D3E9002305F016FB064620460F4605F0AE
:10017000DDFE05F0BBFA02460B463046394605F077
:1001800033FC124B044618680D4605F0AFFA0246E0
:100190000B462046294605F0FDFA05F095FD0C4A70
:1001A0000C4B1278186012B11A6852421A60F8BDEE
:1001B00000000000006AF840000401407058002070
:1001C000745800208258002000140040F44B002096
:1001D000F04B00206C58002010B50446084605F08E
:1001E000A5FE05F083FA08A3D3E9002305F0D2FAAF
:1001F00005F06AFD064B58615A692046C3F8A420F1
:10020000BDE81040FEF76EBF2D431CEBE2361A40EE
:10021000644A002010B50446084605F087FE05F044
:1002200065FA09A3D3E9002305F0B4FA05F04CFD03
:10023000074B18601A6820465A60BDE81040FEF768
:1002400051BF00BFAFF300802D431CEBE2361A40D4
:10025000644A002008B581EAE170A0EBE17005F086
:1002600065FE05F043FA06A3D3E9002305F092FAF0
:1002700005F02AFD044BD86608BD00BFAFF300802F
:100280002D431CEBE2361A40644A0020054B002245
:100290001A70054B1A7A12B1044A1268891AD96089
:1002A000FEF720BF78580020644A00208C580020B8
:1002B000084B10B51A7A0C4632B10020F8F7F6F95F
:1002C000054B241A1C6010BD1961BDE81040FEF7F3
:1002D00009BF00BF644A00208C58002010B50446B6
:1002E00081EAE170A0EBE17005F020FE05F0FEF977
:1002F00007A3D3E9002305F04DFA05F0E5FC064B12
:1003000018662046BDE81040FEF7ECBEAFF3008053
:100310003A8C30E28E794540644A002010B504469C
:1003200081EAE170A0EBE17005F000FE05F0DEF976
:1003300007A3D3E9002305F02DFA05F0C5FC064B11
:1003400098652046BDE81040FEF7CCBEAFF30080B4
:100350002D431CEBE2361A40644A0020022902D8E1
:10036000024BC9B25972FEF7BDBE00BF644A0020FD
:10037000054B1A7A19B12AB901221A727047062A56
:1003800008BF1972704700BF644A0020014B83F810
:1003900054107047644A0020082903D8024BC1F169
:1003A00008019967704700BF644A002008B50A4BEE
:1003B000586905F0BBFD05F099F905A3D3E90023C1
:1003C00005F012FB05F080FC08BD00BFAFF3008014
:1003D0002D431CEBE2361A40644A002008B50A4B54
:1003E000186805F0A3FD05F081F905A3D3E9002302
:1003F00005F0FAFA05F068FC08BD00BFAFF3008015
:100400002D431CEBE2361A40644A0020014BD86CA5
:10041000704700BF644A002008B5094BD86E05F04C
:1004200085FD05F063F904A3D3E9002305F0DCFAA8
:1004300005F04AFC08BD00BF2D431CEBE2361A4014
:10044000644A0020044B1A7AD8681AB1034B1B681F
:10045000C0187047704700BF644A00208C580020C5
:10046000044B1A7A18691AB1034B1B68C0187047FD
:10047000704700BF644A00208C58002008B50A4B22
:10048000186E05F053FD05F031F905A3D3E90023FB
:1004900005F0AAFA05F018FC08BD00BFAFF3008014
:1004A0003A8C30E28E794540644A002008B50A4B08
:1004B000986D05F03BFD05F019F905A3D3E900237C
:1004C00005F092FA05F000FC08BD00BFAFF3008014
:1004D0002D431CEBE2361A40644A0020014B587A47
:1004E000704700BF644A0020024B187A003018BFE2
:1004F00001207047644A0020014B93F85400704774
:10050000644A0020024B986FC0F10800C0B27047E7
:10051000644A002010B50748C469200911B1E40CF1
:1005200064010C6012B1C0F38421117003B1187022
:1005300010BD00BF644A0020074B1A7A062A08D073
:100540001869DB68C3EB000CDCF1000040EB0C0029
:100550007047024B18787047644A0020805800208A
:10056000B4235843024900F580700422F9F739BBDF
:10057000C44A0020B4235843024900F58270042283
:10058000F9F72FBBBC4A0020B4235843024900F5B9
:1005900084700422F9F725BBD04A002002494FF4A9
:1005A00080700422F9F7AEBBC44A002002494FF420
:1005B00082700422F9F7A6BBBC4A002002494FF41E
:1005C00084700422F9F79EBBD04A0020034B01221D
:1005D0005A7200225A611A60704700BF644A0020B4
:1005E000024B186900F00800C0B2704700040240D6
:1005F000024B186900F01000C0B2704700040240BE
:1006000010B5044659B101214FF08040002202F09C
:10061000CBFE20460021BDE81040F9F7DDBF0121E7
:10062000F9F7DAFF01214FF080400A46BDE810409B
:1006300002F0BABE4FF08043988900F00100704785
:10064000074A92F82400064B0028FAD10122C3F889
:10065000241183F8242093F82420002AFBD170472A
:10066000644A0020014BC3F8D8007047644A002058
:10067000014BD3F8D8007047644A0020014BC3F8FF
:10068000CC007047644A0020014BD3F8CC0070477F
:10069000644A0020034B187AA0F10603584240EB4D
:1006A00003007047644A0020014BC3F8F80070470C
:1006B000644A0020014BC3F804017047644A0020DB
:1006C000014BC3F800017047644A0020014BC3F896
:1006D00008017047644A0020014BC3F8FC007047D2
:1006E000644A0020014BC3F81C017047644A002093
:1006F00032235843014BC3F814017047644A002069
:1007000032235843014BC3F818017047644A002054
:10071000014BC3F8F0007047644A0020014BC3F856
:1007200080007047644A0020014BC3F8880070477E
:10073000644A0020014BC3F884007047644A0020DB
:10074000014B1860704700BF7C580020014B1860B7
:10075000704700BF84580020014B1860704700BFED
:1007600094580020014B1860704700BF905800203B
:10077000014B1860704700BF88580020014BD3F828
:10078000F8007047644A0020014BD3F80401704719
:10079000644A0020014BD3F800017047644A0020EE
:1007A000014BD3F808017047644A0020014BD3F88D
:1007B000FC007047644A0020014BD3F81C017047CD
:1007C000644A0020034BD3F81401322390FBF3F06A
:1007D000704700BF644A0020034BD3F8180132234E
:1007E00090FBF3F0704700BF644A0020024BD3F83F
:1007F000F000C0B2704700BF644A0020014BD3F83C
:10080000EC007047644A0020014BD3F8E8007047C1
:10081000644A0020014BD3F8D0007047644A00209E
:10082000014BD3F8E0007047644A0020014BD3F835
:10083000E4007047644A0020014BD3F88000704701
:10084000644A0020014BD3F888007047644A0020B6
:10085000014BD3F884007047644A0020014BD3F861
:100860008C007047644A0020014B1868704700BF35
:100870007C580020014B1868704700BF8458002046
:10088000014B1868704700BF94580020014B18684E
:10089000704700BF90580020014B1868704700BF98
:1008A00088580020014BD3F8C0007047644A0020EC
:1008B000014BC3F8A0007047644A0020014BD3F8F5
:1008C000A0007047644A002008B50028B8BF404225
:1008D00005F02CFB04F00AFF05A3D3E9002304F084
:1008E00059FF05F0F1F9044BC3F8900008BD00BFB3
:1008F0002D431CEBE2361A40644A002008B50A4B2F
:10090000D3F8900005F012FB04F0F0FE04A3D3E945
:10091000002305F069F805F0D7F908BDAFF30080B2
:100920002D431CEBE2361A40644A0020014BC3F809
:100930009C007047644A0020014BD3F89C0070472C
:10094000644A0020014BC3F8F4007047644A002059
:10095000014BD3F8F4007047644A0020084B10B5EF
:100960000446187A30B10020F7F7A0FE054B241A90
:100970001C6010BD2146BDE81040F7F7B1BE00BFB6
:10098000644A00208C58002008B50020F7F78EFE3E
:10099000014B1B68C01808BD8C580020014BC3F8E0
:1009A000C4007047644A0020014BD3F8C40070476C
:1009B000644A002038B51D4C237A062B04D0002051
:1009C0000121FFF7CBFC27E0637A012B24D002D36F
:1009D000022B2AD126E020682368256E80FB0301C4
:1009E0002A46EB1705F08CFC02460B46C90F52183D
:1009F00043F100035B104FEA32022368D4F89810E9
:100A0000002B0B4B1B681944CCBF8918C2EB0101AA
:100A10000020BDE8384039E400200146BDE83840F8
:100A2000FFF7DABB0023C4F8C43038BD644A0020A5
:100A30008C580020014BC3F828017047644A0020FD
:100A4000014BD3F828017047644A002038B5114C97
:100A5000237A062B14D10020FFF7A8FCD4F8282114
:100A6000E36C801A984212DC0020E56CFFF79EFCD4
:100A7000D4F82831C0188542CCBF0020012038BDF1
:100A800020686369C21A504240EB020038BD002062
:100A900038BD00BF644A002010B50A20F8F7D8FE20
:100AA00004460B20F8F7D4FE404304FB0400BDE8E5
:100AB0001040FEF74DBA034BD3F89400024B1B686D
:100AC000C0187047644A00208C58002008B50A4BB3
:100AD000D3F8A40005F02AFA04F008FE04A3D3E931
:100AE000002304F081FF05F0EFF808BDAFF30080AC
:100AF0002D431CEBE2361A40644A002008B50A4B2D
:100B0000586805F013FA04F0F1FD05A3D3E90023BA
:100B100004F06AFF05F0D8F808BD00BFAFF300800D
:100B20002D431CEBE2361A40644A0020094B1A7A26
:100B30002AB983F82C2107221A7201207047062A4D
:100B400005D10120072283F82C011A72704700207A
:100B5000704700BF644A0020014B93F82D01704795
:100B6000644A0020054B1A682AB95869D0F101007F
:100B700038BF002070470020704700BF644A002043
:100B800070B5A94C237A013B082B00F24B81DFE8BA
:100B900013F009002D006A00470059004901970031
:100BA000BE00E9000020FFF781FCC4F830010020FE
:100BB000FFF764FC4FF44841C4F834010020FFF70C
:100BC000ADFB4FF448410020FFF788FB00250020D3
:100BD000FFF7FCFC25612846E560FEF783FAF7F78E
:100BE00045FBE567C4F8380102238EE0F7F73EFBCA
:100BF000D4F838318C4DC01A0028B8BF4042B0F547
:100C0000FA7F40F30F8100200146F7F769FD4FF4AA
:100C100080630020EB600146FFF7A0FB04239FE008
:100C20000020FFF789FC002800F0FC800020F7F787
:100C30003DFD7D4B0022A0F58060C3F8CC00DA605A
:100C400005220EE00020FFF777FC002800F0EA8084
:100C50000020FFF7BBFCF7F709FB734B0322C3F837
:100C600038011A7270BDF7F701FBD4F838316E4DB8
:100C7000C01A0028B8BF4042B0F5FA7F40F3D280D6
:100C800000200146F7F72CFD0020F7F70FFD286143
:100C90002B690024EB60EB682046C5F89830EB68C0
:100CA000D5F83011C5F89430604B1C60FFF736FB67
:100CB0002046D5F83411FFF711FB6C7206234FE084
:100CC0000020FFF7F3FBC4F830010020FFF7D6FB4C
:100CD0004FF44841C4F834010020FFF71FFB4FF4E4
:100CE00048410020FFF7FAFA0020FFF76FFC4F4A57
:100CF0000023E3672361E3601360012384F82D314F
:100D0000F7F7B4FA0823C4F83801237270BDF7F777
:100D1000ADFAD4F83831444DC01A0028B8BF40426B
:100D2000FA287FDD424B00241969204621F02F412B
:100D30001961404B090E1C70F7F762FD20464FF415
:100D40008031F7F705FD20462146F7F7C9FC3A4BFD
:100D500020461B6821461B02EB60FFF7FFFA0923C0
:100D60002B7270BD0020FFF7E7FB00285AD000204F
:100D7000F7F79CFC0028044608DA00200121F7F769
:100D80003FFD2B4B1A6942F080721A6184EAE472CB
:100D9000A2EBE472294B00246FF0C705C82012E0D3
:100DA00091FBF5F68E1996420CDC91FBF0F68E194C
:100DB000B24207DC0020F7F72DFF1B4B022283F81D
:100DC0002D2105E0013453F8041FB1F1FF3FE7D1B5
:100DD0001B4B53F82430144C013305D1002384F805
:100DE0002C31032384F82D3100250020FFF7EEFB82
:100DF000256128462946E560F7F772FC94F82C3106
:100E000028465B1B18BF0123D4F83011237284F8E5
:100E10002C51FFF783FAD4F834112846BDE870400E
:100E2000FFF75CBA70BD00BF644A00208C580020F8
:100E3000544D0020F94B0020EC4B0020B80000205E
:100E4000BC0000207FB5234D234C08262E80636A0A
:100E50002988204689B2591A02F0A6F8636A2988BF
:100E6000204689B2C91802F0A1F820463146012275
:100E700002F09AFA01221021204602F095FA2E2360
:100E80000124164D8DF80C3003A802238DF80D3087
:100E90008DF80E408DF80F4002F050FD21462020C5
:100EA00001F038FB284601F00FFE4FF6FF73019367
:100EB0004FF41673ADF80030284600236946ADF8AC
:100EC0000830ADF8023001F0A9FE2846214601F0B5
:100ED0003AFF7FBD8258002000040140001400400A
:100EE0007FB50020FFF75AFB0020FFF75FFB0020D3
:100EF000FFF764FB3F4B0026FF220F213E48C3F85B
:100F0000D8200124C3F8CC60C3F8EC10C3F8F81063
:100F10000A21C3F80421C3F80061C3F80821C3F80B
:100F2000FC40C3F81C41C3F81461C3F81861C3F84E
:100F3000F040C3F8F44083F8544001602F48642522
:100F400006602F4802602F4805602F483546016033
:100F50004FF4FA61C3F8A0104B21C3F89C102B4941
:100F60002046C3F89010C3F88420294A2146C3F8CC
:100F70008020284AC3F888204FF4FA72C3F8282149
:100F800001F0C8FA4FF0804001F09EFD40F6B83302
:100F900069464FF080400193ADF80060ADF80860FD
:100FA000ADF8026001F03AFE224621464FF0804043
:100FB00002F0FAF921464FF0804001F0C4FEFFF73D
:100FC00041FF1C2303A88DF80C308DF80D408DF8DF
:100FD0000E408DF80F4002F0B1FC232303A88DF8DA
:100FE0000C308DF80D608DF80E408DF80F4002F03A
:100FF000A5FC7FBD644A0020945800209058002032
:1010000088580020845800207C580020703D0A0039
:1010100020A10700804F12007047FEE7FEE7FEE7C1
:10102000FEE7704770477047704700002E4B82B054
:101030001A6842F001021A6000229A60196821F0D1
:10104000847121F48031196028495960196821F4AC
:1010500080211960DA60009201921A6842F48032AD
:101060001A601A6802F400320192009A013200926A
:10107000019A1AB9009AB2F5A06FF2D11A4B1B6807
:1010800013F4003318BF01230193019B012B25D1D9
:10109000154B9A689A609A6842F400429A609A687E
:1010A00042F4A0529A60124A5A601A6842F0807262
:1010B0001A6019680C4A8901FBD50E4B40F2037186
:1010C0001960936823F003039360936843F002036D
:1010D0009360936803F00C03082BFAD1064B074A80
:1010E0009A6002B0704700BF003802401030002400
:1010F000081E4005003C024000ED00E000800008B2
:10110000154B16499868164A00F00C00042801D0C7
:10111000082801D00A6013E0586859685B6801F03C
:101120003F01C3F38813B2FBF1F25A430A4B5B68E9
:10113000C3F3014301335B00B2FBF3F2074B1A60C8
:10114000054B9A68054BC2F303129A181279196875
:1011500021FA02F21A6070470038024004010020B0
:101160000024F400012108B54FF4807001F01AFA50
:101170004FF480700021BDE8084001F013BA4368C5
:101180000A6823F0407323F4807313430A7930B55F
:1011900043EA02234360CA680B6984688D681A4376
:1011A000084B2A43234013434A7943EA42038360AE
:1011B0000B7DC26A013B22F47002DBB242EA0353A8
:1011C000C36230BDFDF7FFC00023036003714371AC
:1011D0008360C360036101230375704710B5074A3C
:1011E000074B51680B4090E8120021438468C068A7
:1011F000214301430B43536010BD00BF0023014056
:10120000E030FCFF0023036043608360C3607047ED
:10121000836811B143F0010301E023F0010383600F
:101220007047436823F4400323F40073194341607B
:101230007047416282627047436823F01F0319437D
:1012400041607047044B5A6810B142F4000201E05B
:1012500022F400025A60704700230140044B5A6890
:1012600010B142F4800201E022F480025A6070471B
:1012700000230140092970B54FF003040DD94C43F8
:1012800007251E3C05FA04F503FA04F3C66826EAAE
:10129000050545EA0304C4600BE04C43072505FA45
:1012A00004F503FA04F4066926EA050545EA040391
:1012B0000361062A4FF005030CD8013A53431F225D
:1012C00002FA03F201FA03F3446B24EA0202134325
:1012D000436370BD0C2A0DD853431F22233B02FAEF
:1012E00003F201FA03F1046B24EA020242EA010369
:1012F000036370BD53431F22413B02FA03F201FA1C
:1013000003F1C46A24EA020242EA0103C36270BD27
:10131000836843F08043836070478068C0F38050E7
:101320007047836811B143F4806301E023F4806364
:1013300083607047836811B143F0020301E023F03A
:101340000203836070474368013923F4604343EA32
:10135000413141607047436811B143F4006301E0DB
:1013600023F4006343607047C06C80B27047014B48
:101370001868704708230140836811B143F48073F3
:1013800001E023F4807383607047836811B143F4F4
:10139000007301E023F4007383607047044B5A68C4
:1013A00010B142F4005201E022F400525A6070473A
:1013B00000230140092970B54FF003040DD94C43B7
:1013C00007251E3C05FA04F503FA04F3C66826EA6D
:1013D000050545EA0304C4600BE04C43072505FA04
:1013E00004F503FA04F4066926EA050545EA040350
:1013F0000361836BC3F30154121B02320524D2B282
:1014000062431F2404FA02F401FA02F123EA0403FE
:101410000B43836370BD836B013923F4401343EAAC
:1014200001518163704782B0002301930190019BB9
:10143000C9180191019B1A6002B07047836823F4B8
:101440007023194381607047836823F44013194364
:1014500081607047836843F48003836070478068CD
:10146000C0F380507047436811B143F4806301E0DA
:1014700023F4806343607047436811B143F48053A1
:1014800001E023F480534360704782B0002301934E
:101490000190019B283359180191019B186880B273
:1014A00002B070470123C9B203FA01F143680AB1DF
:1014B000194301E023EA01014160704703681942C2
:1014C0000CBF002001207047C9430160704743688A
:1014D000006810EA112007D00122C9B202FA01F116
:1014E00019420CBF0020012070476FEA11210160F2
:1014F000704700BF08B50B4B984207D14FF0007002
:10150000012101F043F84FF0007006E04FF08060D9
:10151000012101F03BF84FF080600021BDE8084058
:1015200001F034B800640040036823F00203036054
:10153000036843F0010303604FF480334268D2072D
:1015400001D4013BFAD1436813F0010356D08B79E3
:10155000012B03680CBF43F0800323F0800303607A
:10156000CB79012B03680CBF43F0400323F0400309
:1015700003600B7A012B03680CBF43F0200323F0B8
:10158000200303604B7A012B03680CBF43F0100368
:1015900023F0100303608B7A012B03680CBF43F028
:1015A000080323F008030360CB7A012B03680CBF08
:1015B00043F0040323F0040303608B78CA789B078D
:1015C00043EA02630A7943EA02434A7943EA02534F
:1015D0000A88013A1343C361036823F001030360DF
:1015E0004FF480334268D20701D5013BFAD14368FA
:1015F00013F0010F14BF00200120704718467047F8
:10160000837A012101FA03F170B5354BCC43D3F84D
:10161000002242F00102C3F80022D3F81C2222402B
:10162000C3F81C22027BAAB9D3F80C22C688224038
:10163000C3F80C22827A4588483245EA064543F8C9
:10164000325003888288857A43EA0242254BED00B6
:10165000EB185A60037B012B16D1214B0688D3F877
:101660000C2245880A43C3F80C22827A45EA0645D3
:10167000483243F83250C3888288857A43EA02426E
:10168000184BED00EB185A60C37A154A1BB9D2F813
:101690000432234002E0D2F804320B430589C2F839
:1016A00004320F4B2DB9D2F814522C40C2F8144218
:1016B00006E0012D04D1D3F814220A43C3F8142202
:1016C000427B012A04D1D3F81C221143C3F81C1217
:1016D000D3F8002222F00102C3F8002270BD00BF3F
:1016E000006400404066004000238371C3710372B0
:1016F00043728372C3728370C37003230371022326
:1017000043710123038070470D4BD3F8002242F050
:101710000102C3F80022D3F8002222F47C5222F006
:101720000E02C3F80022D3F8002242EA0020C3F8D8
:101730000002D3F8002222F00102C3F80022704711
:1017400000640040036811B143F4803301E023F4E6
:10175000803303607047036899B143F080030360EE
:10176000D0F8843143F48073C0F88431D0F89431D8
:1017700043F48073C0F89431D0F8A43143F48073FB
:1017800012E023F080030360D0F8843123F48073E7
:10179000C0F88431D0F8943123F48073C0F89431C8
:1017A000D0F8A43123F48073C0F8A431704770B529
:1017B00082680346500107D49A68120106D49A68D9
:1017C000D0004AD5022002E0002000E0012000F114
:1017D000180212019C5804F001049C500C7A9D5888
:1017E00024B90E684C7A44EA465404E04E6844EA50
:1017F000C6042C434D7A2C439C508A7A00F118047D
:10180000240102F00F028A721A19556825F00F059B
:10181000556055688E7A354355604E7B8A7B360419
:1018200046EA0266CA7A16430A7B46EA022603EBB8
:101830000012C2F8886102F5C4754A7C8E7C1204DD
:1018400042EA0662CE7B097C324342EA01226A60A8
:101850001A5942F001021A5170BD042070BD0129CD
:1018600006D002D302290AD105E082680E4B04E0BB
:1018700082680E4B01E082680D4B134000E00023AC
:10188000094A93420BD001D83BB10AE0074A934280
:1018900005D0074A934204D101E00220704701209D
:1018A00070470020704700BF0300000400030008D9
:1018B00000000310012907D002D302290DD108E04E
:1018C000836843F0800302E0836843F4004383604D
:1018D0007047836843F400038360704730B501F1BB
:1018E0001B042301C55805F00405EDB21572C35859
:1018F00015B95B0D136001E0DB0853602401031987
:10190000045904F0020454725C6804F00F049472E9
:101910005B681B0AD37400EB0113D3F8B85103F5CD
:10192000DC74D572D3F8B8512D0A1573D3F8B851B9
:101930002D0C5573D3F8B8311B0E93736368D373B2
:1019400063681B0A137463681B0C537463681B0E73
:10195000937421B9C36843F02003C36030BD0369A9
:1019600043F02003036130BD21B9C36843F0200375
:10197000C3607047036943F020030361704709B9EE
:10198000C06802E0012903D1006900F0030070473C
:101990000020704799B9036823F0030343F0010363
:1019A00003604FF48033426802F00302012A01D041
:1019B000013BF8D1406800F00300012828E001292C
:1019C00011D1036823F0030303604FF480334268AE
:1019D000920701D0013BFAD1436813F0030F14BF03
:1019E000002001207047022916D1036823F0030369
:1019F00043F0020303604FF48033426802F00302B5
:101A0000022A01D0013BF8D1406800F0030002280F
:101A100014BF00200120704700207047036823F0A6
:101A2000030343F002030360406800F00300A0F1E9
:101A30000201484240EB01007047036823F00203B3
:101A400003604FF480334268920701D5013BFAD11D
:101A5000436813F0020F14BF002001207047806913
:101A600000F0700070478069000E70478069C0F315
:101A70000740704743690AB1194301E023EA0101B5
:101A80004161704711F4700F01D083690AE0CB0106
:101A900001D5436806E00A0101D5836802E08B01A5
:101AA00009D5C36823F07F4323F470030B420CBFB6
:101AB000002001207047036923F07F4323F4700363
:101AC0000B420CBF0020012070470B4B994202D102
:101AD00000238361704721F07F438A0123F4700360
:101AE00001D5C36070474A0101D5036170470A01FF
:101AF0004CBF8360436070477000F03043690B4017
:101B00005DD040293CD00ED804292DD004D801291D
:101B100021D0022955D125E0102929D020292DD006
:101B200008294ED122E0B1F5006F3DD009D8B1F5BA
:101B3000007F33D0B1F5806F34D0B1F5807F40D1D4
:101B400028E0B1F5803F1DD0B1F5003F1ED0B1F5C2
:101B5000004F36D12FE083681B481840003018BF73
:101B600001207047C06804E0C0680CE0C0680EE067
:101B7000006910F0030018BF01207047006902E0FF
:101B8000006904E04068C0F3C00070474068C0F3DB
:101B900000107047806900F0010070478069C0F351
:101BA00040007047806907E0836913F0700F0CBF35
:101BB0000020012070474068C0F38000704718463D
:101BC00070470020704700BF01010100B1F5807F20
:101BD00035D00CD8082924D004D801291CD00429D8
:101BE00034D11CE020291FD040292FD11EE0B1F5AF
:101BF000006F22D006D8B1F5007F20D0B1F5806FFC
:101C000024D11CE0B1F5803F13D0B1F5003F12D0D4
:101C1000B1F5004F1AD115E00D4B836070470823D2
:101C200000E01023C3607047082300E01023036125
:101C30007047082304E0102302E00023836104239B
:101C4000436070470023836104234360704700BFF3
:101C500001010100036823F0010303600023036016
:101C600043608360C3600361212343612C4B98422E
:101C70001CD02C4B984220D02B4B984225D02B4B7C
:101C800098422AD02A4B98422FD02A4B984233D0E0
:101C9000294B984237D0294B984204D14FF03D52FE
:101CA00043F8AC2C7047264B984203D13D2243F8B1
:101CB000082C7047234B984204D14FF4746243F8C8
:101CC000202C7047204B984204D14FF4741243F8F3
:101CD000382C70471D4B984204D14FF0746243F882
:101CE000502C70471A4B984203D11A4A43F8642C7F
:101CF0007047194B984203D1184A43F87C2C70471F
:101D0000174B984203D1174A43F8942C7047164B4F
:101D1000984204BF4FF03D5243F8AC2C704700BFCF
:101D2000106002402860024040600240586002405B
:101D30007060024088600240A0600240B8600240CB
:101D4000106402402864024040640240586402402B
:101D5000706402403D00002088640240400F002073
:101D6000A064024000003D20B86402400268134BAA
:101D700010B51340CC680A6822434C6922438C6931
:101D80002243CC6922430C6A22434C6A22438C6A68
:101D900022434C6B22438C6B224313430360426902
:101DA0000C6BCB6A22F007022343134343610B6998
:101DB00043604B6883608B68C36010BD3F801CF03C
:101DC0000023036043608360C360036143618361F8
:101DD000C361036243628362C362036343638363D9
:101DE0007047036811B143F0010301E023F00103E0
:101DF00003607047036811B143F4004301E023F42A
:101E0000004303607047036811B143F0200301E011
:101E100023F020030360704741607047406880B240
:101E20007047036812B143F4002301E023F4002358
:101E3000036001617047036811B143F4802301E03E
:101E400023F48023036070470AB101617047C160C9
:101E500070470068C0F3C0407047006800F00100A0
:101E60007047406900F03800704710B5084A094BC8
:101E7000094CA0428CBF104618468B00074B4CBF44
:101E8000426802680B4013420CBF0020012010BDC5
:101E900000640240006002400F6402407D0F7D0F2D
:101EA00010B5084B084A094CA0428CBF1046184692
:101EB000074B11F0005F01EA030314BFC3608360A6
:101EC00010BD00BF00600240006402400F64024089
:101ED0007D0F7D0F0B0607D5436912B143F08003D8
:101EE00001E023F080034361802909D001F01E0145
:101EF000036812B119430160704723EA01010160D0
:101F00007047104B10B5104A104CA0428CBF1446BD
:101F10001C460F4B0B402BB1026802F01E0202EA76
:101F2000D12202E0426902F080028800094B4CBFD6
:101F3000606820680B40184002D0101C18BF0120B8
:101F400010BD00BF00600240006402400F64024008
:101F50003C0F3C0F7D0F7D0F10B5084B084A094C14
:101F6000A0428CBF10461846074B11F0005F01EAF3
:101F7000030314BFC360836010BD00BF0060024054
:101F8000006402400F6402407D0F7D0F044B00226D
:101F90001A605A609A60DA60024A5A61704700BF5C
:101FA000003C0140FFFF7F00837910B5002B29D052
:101FB0001A4B01681C68CA4314401C605C682240CC
:101FC0005A60027902F1804202F59E321468214380
:101FD000116002689C68D1430C409C60DC68214021
:101FE000D9604179102906D1996811439960D9685F
:101FF0000A43DA6010BD01F1804303F59E3319688E
:102000000A4308E00379016803F1804303F59E3336
:102010001A6822EA01021A6010BD00BF003C0140AC
:1020200000230C2203600371427183717047024BDD
:102030001A69104318617047003C0140034B5B690B
:1020400018420CBF00200120704700BF003C014037
:10205000014B5861704700BF003C0140054B1A68B6
:102060005B69034004D010420CBF00200120704780
:1020700018467047003C0140014B5861704700BF53
:10208000003C014008B52C4B984205D10120014687
:1020900000F058FA012048E0284B984205D1022070
:1020A000012100F04FFA02203FE0254B984205D174
:1020B0000420012100F046FA042036E0214B98422A
:1020C00005D10820012100F03DFA08202DE01E4B2B
:1020D000984205D11020012100F034FA102024E0AC
:1020E0001A4B984205D12020012100F02BFA202024
:1020F0001BE0174B984205D14020012100F022FA45
:10210000402012E0134B984205D18020012100F0BD
:1021100019FA802009E0104B98420BD14FF48070DF
:10212000012100F00FFA4FF480700021BDE8084053
:1021300000F008BA08BD00BF0000024000040240E1
:1021400000080240000C024000100240001402404F
:1021500000180240001C0240002002402DE9F04718
:102160000023D1F800801A464FF0010C03270CFA27
:1021700002F404EA0805A54231D107FA03F406681F
:10218000E443264006600E79D0F8009006FA03FA80
:10219000013EF6B24AEA0909012EC0F8009015D8AE
:1021A00091F80590866809FA03F9264086608668EA
:1021B00049EA06068660466826EA050545608D7987
:1021C000466805FA02F5ADB235434560C5682C4056
:1021D000C460CC79C56804FA03F42C43C4600132AE
:1021E0000233102AC3D1BDE8F0874FF6FF730360B6
:1021F0000023037143718371C371704782B04FF440
:1022000080330193019B0B430193019BC361C16127
:10221000019BC361C3690193C369019302B0704715
:10222000036919420CBF002001207047006980B289
:102230007047436919420CBF002001207047406974
:1022400080B2704701837047418370470AB10183B0
:10225000704741837047416170474369594041610C
:10226000704701F0070330B59B000F2404FA03F414
:1022700002FA03F3C908083150F8215025EA040492
:1022800040F8214050F82140234340F8213030BD30
:102290000A4B1A6842F001021A6000229A6019681B
:1022A00021F0847121F48031196005495960196861
:1022B00021F480211960DA60704700BF00380240C5
:1022C00010300024024B00221A701870704700BFB3
:1022D00002380240034B1A6822F0F80242EAC000BA
:1022E0001860704700380240014B1860704700BF0B
:1022F00000004742064B002201281A701A7002D0D3
:10230000042804D101E01870704705221A70704744
:1023100070380240014B1860704700BF800E474282
:10232000014341EA8212009942EA01615A08013AE6
:10233000024B41EA02425A60704700BF0038024037
:10234000014B1860704700BF600047428001034B9B
:1023500040EA0170C3F88400704700BF00380240B3
:10236000014B1860704700BF68004742014B18607E
:10237000704700BF4C004742034B9A6822F0EC6262
:10238000104308439860704700380240034B9A6836
:1023900022F07842104308439860704700380240AA
:1023A000034B9A6822F0030210439860704700BF05
:1023B00000380240024B986800F00C00704700BFE4
:1023C00000380240034B9A6822F0F00210439860F4
:1023D000704700BF00380240034B9A6822F4E05275
:1023E00010439860704700BF00380240034B9A6862
:1023F00022F4604242EAC000986070470038024010
:1024000010B51A4B1A4A996801F00C01042913D02F
:10241000082911D15C6859685B6801F03F01C3F37A
:102420008813B2FBF1F25A43104B5B68C3F30143CC
:1024300001335B00B2FBF3F20C4902608B680D4A7A
:10244000C3F30313D35C046824FA03F343608C687A
:10245000C4F38224145D23FA04F484608968C1F310
:102460004231525C23FA02F3C36010BD00380240CF
:102470000024F4001801002000F44073B3F5407FFD
:10248000084B08D1996820F0704221F4F81122F429
:1024900040720A439A601A6F000542EA10501867AA
:1024A000704700BF00380240014B1860704700BF02
:1024B0003C0E4742014B1860704700BF400E474238
:1024C000014B1860704700BF5C014742044B1A6B18
:1024D00009B1104301E022EA00001863704700BF11
:1024E00000380240044B5A6B09B1104301E022EA64
:1024F00000005863704700BF00380240044B9A6BDD
:1025000009B1104301E022EA00009863704700BF60
:1025100000380240044B1A6C09B1104301E022EA72
:1025200000001864704700BF00380240044B5A6C2A
:1025300009B1104301E022EA00005864704700BF6F
:1025400000380240044B1A6909B1104301E022EA45
:1025500000001861704700BF00380240044B5A6900
:1025600009B1104301E022EA00005861704700BF42
:1025700000380240044B9A6909B1104301E022EA95
:1025800000009861704700BF00380240044B1A6A8F
:1025900009B1104301E022EA00001862704700BF51
:1025A00000380240044B5A6A09B1104301E022EAA4
:1025B00000005862704700BF00380240044B1A6D9B
:1025C00009B1104301E022EA00001865704700BF1E
:1025D00000380240044B5A6D09B1104301E022EA71
:1025E00000005865704700BF00380240044B9A6DE8
:1025F00009B1104301E022EA00009865704700BF6E
:1026000000380240044B1A6E09B1104301E022EA7F
:1026100000001866704700BF00380240044B5A6E35
:1026200009B1104301E022EA00005866704700BF7C
:1026300000380240044B1A7809B1104301E022EA45
:1026400000001870704700BF0D3802404309012B8D
:10265000074A01D1136803E0022B0CBF136F536FBD
:1026600000F01F0023FA00F000F00100704700BFE7
:102670000038024007B5002301933120FFF7E6FF41
:10268000019B01330193019BB3F5A06F01D000289A
:10269000F3D03120FFF7DAFF003018BF01200EBD64
:1026A000024B5A6F42F080725A67704700380240FE
:1026B000034BDB6818420CBF00200120704700BFAD
:1026C00000380240014B1870704700BF0E380240BE
:1026D00008B5154B98420BD101214FF48050FFF7FC
:1026E00061FF4FF480500021BDE80840FFF75ABF5A
:1026F0000E4B984207D14FF480400121FFF746FF6F
:102700004FF4804009E00A4B98420BD14FF400404F
:102710000121FFF73BFF4FF400400021BDE80840D6
:10272000FFF734BF08BD00BF003001400038004053
:10273000003C00400B8810B54C88028823438C88ED
:1027400002F441522343CC8823430C8923434C8910
:1027500023438C892343CC89234313439BB20380B7
:10276000838B23F400631B041B0C83830B8A03827B
:1027700010BD838BF0B523F47A6323F01F031B0491
:102780001B0C8383022303848B68858B022BADB2E1
:1027900038D0294A8E889468002E14BF022601265C
:1027A000240203D5946824F400049460D2F8844091
:1027B000D2F884705268DFF884C002F03F02BCFB9C
:1027C000F2F2C4F388145443C7F30272B4FBF2F478
:1027D000CA88B2F5007F4FF00A0201D1240A02E054
:1027E0007601B4FBF6F46243B2FBF3F305330A223D
:1027F0009BB2B3FBF2F303F001021202C3F34F03E7
:1028000092B200E000229C1EA4B2FE2C28BF00223F
:10281000CC8828BF0223134323439BB203840B8835
:102820004A882B4343F4006313438A8813438A89FD
:1028300013439BB28383F0BD003802400024F400B0
:102840000023038043808380C3800381438183818D
:10285000C381072303827047002302220380438041
:102860008380C380826083817047038819B19BB2E3
:1028700043F0400303E023F040031B041B0C0380E0
:102880007047838B19B19BB243F4806303E023F458
:1028900080631B041B0C83837047038823F400634D
:1028A0001B041B0C038003889BB2194301807047F3
:1028B000B1F5804F038803D19BB243F4804303E01A
:1028C00023F480431B041B0C038070474FF6FF6307
:1028D0009942038803D09BB243F4807303E023F44E
:1028E00080731B041B0C03807047838819B19BB253
:1028F00043F0040303E023F004031B041B0C838058
:102900007047838819B19BB243F0100303E023F0B2
:1029100010031B041B0C83807047808980B27047B2
:1029200081817047038819B19BB243F4005303E0DF
:1029300023F400531B041B0C0380704703889BB2D5
:1029400043F4805303807047012902D0008B80B28A
:102950007047808A80B27047008A80B2704783884F
:102960009BB20AB1194301E023EA0101818070475B
:102970000123090903FA01F1838889B29BB20AB1E4
:10298000194301E023EA010181807047038919425C
:102990000CBF002001207047C94389B201817047F4
:1029A000012301F00F0203FA02F210B584880089B6
:1029B000A4B280B2104006D0090903FA01F31C4208
:1029C0000CBF0020012010BD01F00F01012303FA0C
:1029D00001F3DB439BB20381704700BF012108B5BF
:1029E0004FF48040FFF7DEFD4FF480400021BDE84A
:1029F0000840FFF7D7BD014B186070470038014011
:102A000001F0030230B592000F2404FA02F400FA38
:102A100002F2074B8908023153F8215025EA0404D9
:102A200043F8214053F82140224343F8212030BD90
:102A300000380140014B1860704700BFDC0027429E
:102A4000014B1860704700BF00042742024B186A10
:102A5000C0F30020704700BF0038014030B5048C3F
:102A600024F001042404240C0484058B048CADB2EE
:102A700025F0F305A4B22A4342EA031224F00A0324
:102A800043F0010392B219430283018430BD30B593
:102A9000058C25F010052D042D0C0584048B058C68
:102AA00024F440742405240DADB244EA022242EA23
:102AB000033225F0A00343F0100343EA011192B260
:102AC00089B20283018430BD08B5474B984205D1D5
:102AD00001200146FFF766FD01203DE0B0F1804F87
:102AE00005D101200146FFF751FD012076E03F4B63
:102AF000984205D102200121FFF748FD02206DE038
:102B00003B4B984205D104200121FFF73FFD0420F3
:102B100064E0384B984205D108200121FFF736FDCB
:102B200008205BE0344B984205D110200121FFF7CB
:102B30002DFD102052E0314B984205D1202001217B
:102B4000FFF724FD202049E02D4B984209D10220B7
:102B50000121FFF727FD02200021BDE80840FFF713
:102B600021BD284B984207D14FF480300121FFF757
:102B700019FD4FF48030EFE7234B984207D14FF413
:102B800000300121FFF70EFD4FF40030E4E71F4B4A
:102B9000984207D14FF480200121FFF703FD4FF445
:102BA0008020D9E71A4B984205D140200121FFF738
:102BB000EDFC402012E0174B984205D18020012106
:102BC000FFF7E4FC802009E0134B98420BD14FF44F
:102BD00080700121FFF7DAFC4FF480700021BDE81E
:102BE0000840FFF7D3BC08BD0000014000040040CE
:102BF00000080040000C004000100040001400409D
:102C000000040140004001400044014000480140F0
:102C100000180040001C0040002000401C4A0388AF
:102C200090429BB212D002F5806290420ED0B0F179
:102C3000804F0BD0A2F58032904207D002F580621F
:102C4000904203D002F58062904203D14A8823F07B
:102C5000700313430F4A904208D002F580629042FD
:102C600004D023F440730A899BB2134303804B685A
:102C7000C3620B880385064B984203D003F580633B
:102C8000984201D18B7A038601238382704700BF6B
:102C900000000140001000404FF0FF33436000236C
:102CA000038003814380837270470185828270476D
:102CB000038823F070031B041B0C0B430380704735
:102CC00041627047C1627047406A7047008D80B2B0
:102CD0007047038819B19BB243F0020303E023F06D
:102CE00002031B041B0C03807047038819B19BB2BD
:102CF00043F0040303E023F004031B041B0C0380D4
:102D00007047038819B19BB243F0800303E023F0BE
:102D100080031B041B0C03807047038823F0080307
:102D20001B041B0C038003889BB21943018070476E
:102D3000038823F440731B041B0C038003889BB29D
:102D4000194301807047038819B19BB243F0010316
:102D500003E023F001031B041B0C03807047038C6A
:102D600070B523F001031B041B0C0384038C8488BF
:102D7000028B0D8822F073021204120C2A434E8833
:102D80008D8923F002031B0435431B0CADB22B438A
:102D90000E4DA4B2A84203D005F58065A8420ED11D
:102DA000CD8923F008032B438D8823F004032B43A4
:102DB0004E8A0D8A24F440743543ADB22C4384808E
:102DC00002838A684263038470BD00BF0000014033
:102DD000038C30B523F010031B041B0C0384038CFD
:102DE0008288048B0D8824F4E6442404240C23F008
:102DF000200344EA05241B048D891B0C43EA0513B8
:102E00004D8892B243EA0513124DA4B2A8429BB278
:102E100003D005F58065A84215D1CD8923F0800344
:102E20009BB243EA05134FF6BF751D408B8822F411
:102E3000406245EA03130D8A9BB242EA85024D8A3D
:102E400042EA850292B282808A68048382630384A4
:102E500030BD00BF00000140038C30B523F4807307
:102E60001B041B0C0384038C8288848B0D8824F044
:102E700073042404240C23F400731B042C438D8955
:102E80001B0C43EA05234D8892B243EA0523124DF9
:102E90009BB2A84203D005F58065A84215D1CD8923
:102EA00023F400639BB243EA05234FF6FF351D4030
:102EB0008B8822F4405245EA03230D8A9BB242EAF2
:102EC00005124D8A42EA051292B282808A68848392
:102ED000C263038430BD00BF00000140038C30B5E5
:102EE00023F480531B041B0C0384038C8488828B83
:102EF0000D8822F4E6421204120C23F4005342EA35
:102F000005221B048D891B0C43EA05334D88A4B2AE
:102F100043EA05330A4D92B2A8429BB203D005F5AD
:102F20008065A84205D10D8A24F4804444EA8514C2
:102F3000A4B2848082838A680264038430BD00BFA7
:102F400000000140002303804380838083608381ED
:102F5000C38103824382704730B5012404FA01F42F
:102F6000058C00F11803ADB225EA0404048409B10C
:102F7000082907D14908CC584FF68F702040C85017
:102F8000C8580AE00439C1F34E01CC5848F6FF7026
:102F90002040C8501202C85892B20243CA5030BDF5
:102FA0004163704781637047C16370470164704734
:102FB000038B23F070031B041B0C0B43038370472C
:102FC000038B23F4E0431B041B0C43EA01239BB255
:102FD00003837047838B23F070031B041B0C0B438C
:102FE00083837047838B23F4E0431B041B0C43EA69
:102FF00001239BB283837047038B23F008031B04D8
:103000001B0C0B4303837047038B23F400631B04E7
:103010001B0C43EA01239BB203837047838B23F08D
:1030200008031B041B0C0B4383837047838B23F41F
:1030300000631B041B0C43EA01239BB2838370478C
:10304000038B23F004031B041B0C0B430383704707
:10305000038B23F480631B041B0C43EA01239BB204
:1030600003837047838B23F004031B041B0C0B4367
:1030700083837047838B23F480631B041B0C43EA18
:1030800001239BB283837047038B23F080031B04CF
:103090001B0C0B4303837047038B09025B0441EA5B
:1030A000534189B201837047838B23F080031B0453
:1030B0001B0C0B4383837047838B09025B0441EA3B
:1030C000534189B281837047038C23F002031B04B0
:1030D0001B0C0B4303847047038C23F008031B0471
:1030E0001B0C0B4303847047038C23F020031B0449
:1030F0001B0C43EA01139BB203847047038C23F03B
:1031000080031B041B0C43EA01139BB2038470472A
:10311000038C23F400731B041B0C43EA01239BB2B2
:1031200003847047038C23F400631B041B0C43EAE5
:1031300001239BB203847047038C23F400531B04C8
:103140001B0C43EA01339BB203847047012303FA4B
:1031500001F302FA01F110B5048CA4B224EA0303CE
:103160000384038C194389B2018410BD042303FA3C
:1031700001F302FA01F110B5048CA4B224EA0303AE
:103180000384038C194389B2018410BD00230122FA
:10319000038043808280C38003817047406B704707
:1031A000806B7047C06B7047006C7047038B23F0D7
:1031B0000C031B041B0C0383038B9BB21943018379
:1031C0007047038B23F440631B041B0C0383038BA6
:1031D0009BB243EA012189B201837047F8B50C46DE
:1031E00005464988A288208800290CBF02270027AD
:1031F000012A14BF01260226238988B92846FFF731
:103200002DFCE1882846FFF7D1FF2846394623895F
:103210003246FFF73CFCE1882846BDE8F840D0E79D
:103220002846FFF734FCE1882846FFF7CAFF284606
:10323000394623893246FFF711FCE1882846BDE86C
:10324000F840B3E7838B23F00C031B041B0C838330
:10325000838B9BB2194381837047838B23F4406334
:103260001B041B0C8383838B9BB243EA012189B22D
:10327000818370470B8870B50D4604464988AA883B
:103280003BB92B89FFF7EAFBE9882046BDE870408F
:103290008CE7042B07D12B89FFF7F9FBE98820463F
:1032A000BDE870408DE7082B2E89038C1CD123F4D8
:1032B00080731B041B0C0384808B238C80B29BB215
:1032C00020F0F30023F4206340EA061643EA0121CC
:1032D000B6B289B2324341F48071A2832184E98875
:1032E0002046BDE87040ADE723F480531B041B0C5F
:1032F0000384808B238C20F4407023F4005300055A
:103300005B04000D5B0C40EA022243EA013342EA0F
:1033100006329BB2E98892B243F480532046A283DE
:103320002384BDE8704098E74A880B8813438A8855
:103330001343CA8813430A8913434A8913438A896A
:1033400013439BB2A0F844307047002303804380AE
:103350008380C3800381438183817047B0F8443008
:1033600029B16FEA43436FEA53439BB201E05B0428
:103370005B0CA0F844307047838819B19BB243F0CE
:10338000040303E023F004031B041B0C8380704739
:10339000838819B19BB243F0010303E023F00103DA
:1033A0001B041B0C8380704783899BB20AB11943AD
:1033B00001E023EA01018181704781827047038A1D
:1033C00019420CBF002001207047C94389B2018215
:1033D0007047038A828911EA030092B203D0114236
:1033E0000CBF002001207047C94389B20182704799
:1033F0001143A0F84810704783899BB20AB1194362
:1034000001E023EA010181817047838819B19BB2F1
:1034100043F0080303E023F008031B041B0C838024
:103420007047038923F007031B041B0C03817047BB
:10343000038923F070031B041B0C0B4303810389D6
:103440009BB243F007030381704738B50D46114620
:103450000122602D044602D1FFF719FB01E0FFF7BE
:10346000FDFA238923F070031B041B0C1D432581E7
:1034700023899BB243F00703238138BD038923F0DE
:1034800070031B041B0C0B4303817047838823F0DC
:1034900070031B041B0C838083889BB219438180BB
:1034A0007047038923F007031B041B0C0381038966
:1034B0009BB2194301817047038923F080031B04E9
:1034C0001B0C038103899BB219430181704710B51E
:1034D0000489E4B221430A4342EA032292B2028100
:1034E00010BD10B50446FFF7F2FF23899BB243F4E9
:1034F0008043238110BD10B50446FFF7E8FF238900
:1035000023F077031B041B0C43F07703238110BDCA
:1035100070B50589048B25F00705068C2D0424F46D
:1035200040742D0CB6B224F003042943240426F081
:103530002205240C2A4344F4807442EA031244F026
:10354000010492B201810483028470BD838819B1A1
:103550009BB243F0800303E023F080031B041B0CA9
:1035600083807047A0F85010704700BF08B5234B08
:10357000984205D110200121FFF714F8102037E000
:103580001F4B984207D14FF400300121FEF7FEFF98
:103590004FF4003009E01B4B98420BD14FF48020D0
:1035A0000121FEF7F3FF4FF480200021BDE8084021
:1035B000FEF7ECBF144B984207D14FF400200121D5
:1035C000FEF7E4FF4FF40020EFE7104B984207D1DD
:1035D0004FF480100121FEF7D9FF4FF48010E4E78B
:1035E0000B4B984209D120200121FEF7DBFF202060
:1035F0000021BDE80840FEF7D5BF08BD001001401E
:103600000044004000480040004C00400050004092
:103610000014014030B5038ACA889BB223F440539A
:10362000134303820D4683890989AA8823F4B05382
:103630000A43698923F00C031B040A431B0C92B252
:1036400013438381838AAA899BB223F44073134373
:1036500085B0838204466846FEF7D2FE1A4B9C4230
:1036600003D003F580639C4201D1039B00E0029BE1
:10367000A2894FF0190112B2002A01FB03F12A6856
:1036800001DA520000E092006423B1FBF2F1B1FBD9
:10369000F3F21201100903FB1011A08900B20028F7
:1036A00006DAC9003231B1FBF3F303F0070305E09A
:1036B00009013231B1FBF3F303F00F031A4392B265
:1036C000228105B030BD00BF001001404FF41653F9
:1036D00003600C2200238380C380038142818381A5
:1036E00070470B8810B54C88028A23438C88C988A0
:1036F000234392B20B4322F470629BB213430382C2
:1037000010BD0023038043808380C380704783897A
:1037100019B19BB243F4005303E023F400531B049C
:103720001B0C83817047038B03F47F430383038B5C
:103730009BB2194301837047838929B16FEA4343E0
:103740006FEA53439BB201E05B045B0C83817047DB
:10375000838A19B19BB243F4006303E023F400634E
:103760001B041B0C83827047C905C90D81807047FB
:103770008088C005C00D7047038A23F00F031B0427
:103780001B0C0382038A9BB2194301827047838911
:1037900019B19BB243F0020303E023F002031B04C0
:1037A0001B0C83817047838923F400631B041B0C6B
:1037B000838183899BB2194381817047038A23F0F7
:1037C00020031B041B0C0382038A9BB21943018252
:1037D0007047038A19B19BB243F4804303E023F49A
:1037E00080431B041B0C0382704783899BB243F008
:1037F000010383817047838A19B19BB243F00803A8
:1038000003E023F008031B041B0C83827047038B27
:10381000DBB20383038B9BB243EA01210183704730
:10382000838A19B19BB243F0200303E023F0200305
:103830001B041B0C83827047838A19B19BB243F02F
:10384000100303E023F010031B041B0C838270475A
:10385000838A23F004031B041B0C8382838A9BB29C
:10386000194381827047838A19B19BB243F00203E6
:1038700003E023F002031B041B0C83827047838A3E
:103880009BB20AB1194301E023EA0101818270472A
:10389000C1F3421310B5012401F01F01A34204FA41
:1038A00001F101D10C3004E0022B01D1103000E015
:1038B000143003680AB1194301E023EA01010160F1
:1038C00010BD038819420CBF002001207047C94376
:1038D00089B20180704710B5C1F34214012201F092
:1038E0001F03012C02FA03F201D1838903E0022CA9
:1038F0000CBF038A838A9BB21340028892B243B101
:10390000090A012303FA01F111420CBF0020012032
:1039100010BD184610BD090A012303FA01F3DB4369
:103920009BB20380704700BF40F0BE60024B40F482
:103930002020D860704700BF00ED00E0C37810B5CC
:1039400003B3164B4278DB688478DB43C3F302236E
:10395000C3F10401C9B202FA01F10F2242FA03F2E3
:10396000C9B222400A430E4B01781201CB18D2B2E1
:1039700083F8002303780122590903F01F0302FA98
:1039800003F307E003780122590903F01F0302FA49
:1039900003F32031024A42F8213010BD00ED00E06F
:1039A00000E100E021F0604121F07F01014B08437C
:1039B0009860704700ED00E0044B1A6909B11043AC
:1039C00001E022EA00001861704700BF00ED00E04E
:1039D000044B04281A680CBF42F0040222F00402CF
:1039E0001A60704710E000E0D0F8E83510B51B69A8
:1039F00004469847032384F81231002010BD08B50F
:103A000090F8123180F81331042380F81231D0F885
:103A1000E835DB689847002008BD08B5D0F8E435E4
:103A2000DB6903B19847002008BD08B5D0F8E4353C
:103A30001B6A9847002008BD08B5D0F8E4355B6ADA
:103A40009847002008BDD0F8E83510B55B690446FA
:103A50009847012384F81531002010BDD0F8E835CF
:103A600010B59B6904469847D4F8E43520465B6856
:103A700000219847002084F8150110BD002110B5E1
:103A8000402204460B4601F06BF9802140220023BE
:103A9000204601F065F9012384F81231D4F8E835A5
:103AA000A0785B689847002010BD13B569460446AE
:103AB00000F078FA9DF8001001F01F03012B07D0E9
:103AC000022B0AD073B92046694600F015FB0FE0BF
:103AD0002046694600F0F6FA0AE02046694600F002
:103AE00091FA05E021F07F01C9B2204601F0AAF960
:103AF00000201CBD38B50446002948D190F811318A
:103B0000022B38D1D0F83821D0F824319A4211D97B
:103B1000C178D21A0129C0F8382104D1D0F828116F
:103B2000CB18C0F8283192B22046D4F8281100F002
:103B3000F3F920E0D0F83C21B2FBF3F503FB1525A7
:103B400065B99A420AD3D0F840319A4206D2294642
:103B50002A4600F0E1F9C4F840510CE0D4F8E4350D
:103B6000DB682BB194F81221032A01D12046984733
:103B7000204600F002FA94F81631012B10D1094AC0
:103B8000236912685A60002384F8163108E0D0F8DF
:103B9000E4355B6923B190F81221032A00D19847DC
:103BA000002038BD9858002010B5044659BB90F845
:103BB0001131032B30D1D0F89023D0F87C339A42C6
:103BC00014D9C178D21A0129C0F8902304D1D0F8B1
:103BD0008013C918C0F880139A4228BF1A4692B2BF
:103BE0002046D4F8801300F0B0F915E0D0F8E435A1
:103BF0001B6923B190F81221032A00D1984720466F
:103C000000F0ACF908E0D0F8E4359B6923B190F8F6
:103C10001221032A00D19847002010BD2DE9F04160
:103C2000069F0446164698460D46F6F7CDFE2046FA
:103C30002946C4F8E485C4F8E875C4F8EC6501F0D9
:103C400041F8D4F8E8351B6898472046BDE8F041B4
:103C5000F6F70CBF00207047D0F8E43510B51B68AC
:103C600004469847D4F8E8359B689847002010BD73
:103C700008B5D0F8E4355B689847002008BD00BF60
:103C800043230B80004870475801002038B51D4B76
:103C90001A68511C052A196031D1197900220129AD
:103CA0001A602CD09968B1F5006F08BF9A60154B67
:103CB0009968DC681A46A14202D100221A711EE0FE
:103CC00095BFC1EB0404C1F500631461136115696C
:103CD0000C4C402D8AB205D94031403DA160256190
:103CE000402304E06918A1600021ABB221610549BD
:103CF00001240C7104498A18812101F087F8002001
:103D000038BD00BFBC4B00202759002038B5282300
:103D100003FB0101074C084B0546B1F88C131B69E6
:103D200020469847284601212246402301F052F8B8
:103D3000002038BDDF580020A800002070B50B78A7
:103D4000064613F060050C4625D0202D1FD1CD88E6
:103D5000B5B113F0800F487808D0224B22492A468B
:103D60009B689847E28830461F4928E01F4B1E4950
:103D700058641F4B30465D612A4600F0D6F820E0BB
:103D8000184B48789B6829462A46984728E000F057
:103D90002BF9022524E04B780A2B14D00B2B17D0DB
:103DA000062B1DD14B881B0A212B05D1CA8811492E
:103DB0003A2A28BF3A2201E00F493A22304600F061
:103DC0009BF800250CE00D49012200F095F807E072
:103DD0008B781BB9064A1D46936101E000F004F997
:103DE000284670BDA80000201F590020580100205F
:103DF000BC4B00206A01002061010020D44B002050
:103E000010B58121044600F0CCFF0121204600F0CE
:103E1000C8FF8221204600F0C4FF024B5B68984730
:103E2000002010BDA800002038B5812104464022A2
:103E3000022300F095FF012140220223204600F0DA
:103E40008FFF822108220323204600F089FF084BC0
:103E5000022200251A715D71064B1B6898472046A7
:103E60000121054A402300F0B5FF284638BD00BFB8
:103E700044000020A8000020DF58002010B5074CA7
:103E8000606CFF2807D0064B064A9B6806495269BA
:103E90009847FF236364002010BD00BF5801002035
:103EA000A8000020BC4B00201F59002038B5104945
:103EB0000B79012B19D10C690CB90C7115E0402C50
:103EC00007D98B68403C9AB240338B600C61402329
:103ED00006E08D68A3B22C198C600024AAB20C6194
:103EE00004495218812100F091FF002038BD00BF25
:103EF000BC4B00202759002010B513460C46C0F8D3
:103F00003C21C0F83821022280F8112100212246EC
:103F100000F07CFF002010BD10B50C4613460021B8
:103F2000224600F073FF002010BD10B513460C466A
:103F3000C0F89423C0F89023032280F811210021B7
:103F4000224600F047FF002010BD10B50C46134676
:103F50000021224600F03EFF002010BD0021042376
:103F600010B50A46044680F811310B4600F04EFFAA
:103F7000204600F0CFFD002010BD0021052310B524
:103F80000A46044680F811310B4600F023FF204614
:103F900000F0C0FD002010BD282303FB0100B0F895
:103FA0008C03704790F8CC350B7090F8CD354B7082
:103FB00090F8CF2590F8CE3503EB02234B8090F894
:103FC000D12590F8D03503EB02238B8090F8D325D0
:103FD00090F8D23503EB02239BB2CB80C0F840317E
:103FE000012380F81131704710B58021044600F09C
:103FF00029FF2046002100F025FF2046BDE81040A3
:1040000000F088BD38B50D466B780446012B097960
:1040100010D027D3032B51D190F81231022B28D086
:10402000032B47D16B889BB991B1802910D000F048
:1040300009FF0DE090F81231022B1AD0032B39D171
:104040006B88002B3AD149B1802907D000F018FFC6
:10405000D4F8E43520469B68294698472046FFF768
:104060007DFF2BE090F81231022B02D0032B21D1DF
:1040700006E019B3802921D0204600F0E3FE1DE0C0
:1040800011F0800F4FF0280306D001F07F0103FBF1
:10409000010393F81E2103E003FB010191F876234D
:1040A000074B02B101221A60204605490222FFF7A0
:1040B00023FF03E020462946FFF796FF002038BD86
:1040C000D84B002038B590F812310446032B0D462A
:1040D0000CD10B79012B09D8D0F8E4359B689847AF
:1040E000EB883BB92046FFF739FF03E0204629461D
:1040F000FFF77AFF002038BD73B54B7804460D46B4
:10410000092B00F21C81DFE813F0CD0008011A0131
:10411000E0001A0172000A001A01BD0091006B88CC
:104120001A0A013A062A00F20A81DFE812F00700B3
:104130001A0027000801080108010801D0F8EC3531
:104140000DF106011B6880789847EB880146402BEB
:1041500003D094F81231012B3AD10823ADF8063080
:1041600036E0D0F8E4350DF106019B6A8078984777
:10417000022343700146C4F8F00529E0DBB2052BA9
:1041800000F2DD80DFE803F003080D12171CD0F801
:10419000EC3580785B6817E0D0F8EC3580789B6868
:1041A00012E0D0F8EC358078DB680DE0D0F8EC3523
:1041B00080781B6908E0D0F8EC3580785B6903E013
:1041C000D0F8EC3580789B690DF1060198470146DF
:1041D000BDF80630002B00F0B680EA88002A00F017
:1041E000B2809A4228BF1A46ADF8062058E0AB8844
:1041F000002B40F0A480EB88002B40F0A08090F8CA
:1042000012216B88032A00F09A8003F07F0580F862
:104210001451294600F05EFE2046FFF79FFE0DB1C7
:10422000022300E0012384F812318CE0A978474E84
:104230000129317100F2838090F81231022B02D0F3
:10424000032B7CD108E0002963D00121032380F8EF
:10425000101180F8123111E039B9022380F81231BF
:1042600080F81011FFF704FD53E090F810110129B8
:1042700050D0FFF7FDFC317984F810112046FFF78C
:10428000EBFC46E0EA88012A59D190F81231022B62
:1042900002D0032B53D101E02D4913E000F58871C2
:1042A00020460FE090F81231023B012B47D8274BF4
:1042B0000122DA60D0F818210AB10322DA60254918
:1042C00020460222FFF718FE3DE06B88012B2DD01F
:1042D000022B38D1AB8813F0FF0F34D102691B0ACF
:1042E000013B5268042B0FD8DFE803F003050709F0
:1042F0000B00012306E0022304E0032302E0042371
:1043000000E0052363F30612134B1A60012384F8BF
:1043100016312046FFF722FE15E090F81231023BDD
:10432000012B0CD86B88012B0DD10023C4F8183158
:10433000D4F8E43520469B6829469847E9E72046AB
:104340002946FFF751FE00207CBD00BFD84B00205E
:10435000E04B0020E44B00209858002030B5C8B155
:104360000023DDB20133C41814F8014C002CF8D13D
:104370006B1C5B0013800B7003234B70022305E062
:10438000CA545A1CD2B202338C54DBB210F8012B3F
:10439000002AF5D130BD00BF37B50023104C0546CB
:1043A00001930320F6F776FBEB68013C1A69019252
:1043B00013D0019A002AF4DA019A42F00102019224
:1043C000019A1A61064A1969013A019102D00199CC
:1043D000C907F8D40320F6F75DFB00203EBD00BFFF
:1043E000410D030010B5C47874B900EB82000333AB
:1043F0009B10D0F8D000224603E051F8044C013263
:10440000046004319A42F8D1002010BD033230B567
:104410009210D0F8D0400B46002003E02568013010
:1044200043F8045C04339042F8D101EB800030BDC6
:104430000122F0B50023827040220129C3708280DE
:104440000CD108230370042343704FF4A073C3807E
:1044500002230372C1724FF0A04309E041B90C235B
:104460000370062343704FF4A063C3801F4BC172D7
:1044700003F500620261C3604678044601461A46AD
:10448000002508E002F5106C02F530620A65C1F8FB
:1044900014C001353A460431B54202F12007F1D388
:1044A00003F58062426103F58862C0F8CC2006788B
:1044B00003F5A0650146002203E0C1F88C500132EB
:1044C00020350431B242F8D31946002202E0C4F884
:1044D000CC1001320434B24201F58051F7D303F518
:1044E0006063C0F80C310020F0BD00BF0000044044
:1044F00038B5037A0025012B0446C2681FD1936B9F
:10450000417A65F3104309B143F480139363D36890
:1045100020466FF386136FF396536FF351436FF397
:10452000D343D360FFF738FFE378012B19D105237C
:1045300063F34405E36845F020059D6011E0D3680E
:1045400043F04003D360FFF727FF637AE268002B54
:104550000CBF4FF450234FF4E81393631420F6F785
:10456000A3FAE378012B07D1E36805229D6862F383
:10457000440545F020059D60002038BDC36800203B
:104580009A6842F001029A607047C36800209A68F6
:1045900022F001029A60704707B500230193019B46
:1045A00043F020030193019B61F38A130193019B64
:1045B000C2681361064B1169013B019102D0019958
:1045C0008806F8D40320F6F765FA00200EBD00BF78
:1045D000410D030007B500230193019B43F0100335
:1045E0000193019BC2681361064B1169013B019164
:1045F00002D00199C906F8D40320F6F74BFA00203F
:104600000EBD00BF410D030008B5C2680129D36883
:104610006FF35D736FF39E7302D143F0005302E0BA
:1046200009B943F080433220D360F6F73DFA002009
:1046300008BDC368586900F001007047C3685B6932
:1046400013F0010F14BF002001207047C3685869A0
:1046500000F001007047C3685A69986910407047BC
:10466000C3685868704703691A6861F301021A60E9
:104670007047C268002393614FF0FF316FF08043B1
:104680005361516053610C4B9361C3789169002B66
:1046900014BF4FF400634FF4016343F0804343F4CD
:1046A000701343F4405343F00C0321EA03010B431E
:1046B00093610020704700BF00080080F8B5D0F873
:1046C0000C3100221A60036915461A68044665F326
:1046D000CC221A60C37A012B21D10321FFF7C3FF3B
:1046E000E36880214FF4001261F30F0259629A626D
:1046F000A02262F30F0561F31F454FF49072C3F8D7
:10470000045162F30F05C0F220054FF4A072C3F804
:10471000085162F30F056FF31F45C3F80C511021C8
:104720002046FFF739FF2046FFF754FF2269002398
:104730004FF0FF311361204653611E469161FF2502
:10474000D361214610E08269013317680430C7F352
:10475000076707F08007FFB2002F14BF4FF09047A4
:10476000002717601661956062789342EBD30023AF
:104770001D46FF2010E04A6D013316680431C6F370
:10478000076606F08006F6B2002E14BF4FF0904682
:10479000002616601561906062789342EBD323691E
:1047A0001A6942F480721A61E278012A04D1054A3A
:1047B000402161F359421A632046FFF75AFF002057
:1047C000F8BD00BF0301010003699B68C3F3410307
:1047D000013B022B9ABF024AD05C0320704700BF06
:1047E0000899010810B5036981699C680A68C4F3D7
:1047F0004100022802D06FF30A0202E0032060F3B6
:104800000A020A605A68002042F480725A6010BDA1
:1048100030B54D780B780022012D00EB830405D1D3
:1048200005FA03F3A46963F30F0205E0012505FA15
:1048300003F3646D63F31F422368C3F3072505F098
:104840008005EDB26DB98D6865F30A03CD78C9882E
:1048500065F3934361F3995343F0805343F400436A
:10486000236003690020D9690A43DA6130BD30B59D
:104870004D780B780024012D224600EB830105D1F1
:1048800005FA03F3896963F30F0205E0012505FAD0
:1048900003F3496D63F31F4203696FF3CF340C6078
:1048A000D969002021EA0202DA6130BDF8B54F78FB
:1048B0000B78012F00EB830349D19E694C69356861
:1048C00033692A4664F3120314B967F3DC430BE03F
:1048D0008F68E419013CB4FBF7F7CC7867F3DC434D
:1048E000012C08BF64F35E733361C378012B06D1DA
:1048F0000B780C6900EB83039B695C610CE0CB785F
:10490000012B09D04B693BB10C78012707FA04F45D
:1049100003695E6B34435C63CB78012B07D1036979
:104920009B68DB0554BF45F0005245F080520B7880
:1049300042F0044200EB83039B691A60CB78012BA1
:1049400038D10A788B8AC968FFF74CFD32E05E6D7A
:104950004F6935688C682A4633692FB964F31203AE
:10496000012464F3DC430AE03F19013FB7FBF4F78D
:10497000BF05BF0D7C4367F3DC4364F3120333616F
:10498000C378012B05D10B780C6900EB83035B6DB9
:104990005C61CB78012B06D14B7913B145F0005205
:1049A00001E045F080520B7842F0044200EB8300B6
:1049B000436D1A600020F8BD73B54D78012D3DD1CF
:1049C00083694A691E681C690094E4B242B962F3C3
:1049D00006048DF800409DF8024065F3C4040EE023
:1049E0008D68AA4286BF4D6165F3060462F3060432
:1049F0008DF800409DF80240012262F3C4048DF856
:104A00000240009A1A61C278012A05D10A780C691D
:104A100000EB82029269546146F004421A60C37846
:104A2000002B34D14B69002B31D00A78012101FAD7
:104A300002F20369586B02435A6328E00B784E690F
:104A400000EB83035B6D8C681A681D690095EDB2FD
:104A500006B14C6164F306059DF802408DF80050E4
:104A6000012565F3C4048DF80240009C1C61C378E5
:104A7000012B05D10B780C6900EB83035B6D5C6146
:104A80000B7842F0044200EB8300436D1A60002073
:104A90007CBD4B78012B0B7800EB83000AD1826937
:104AA0001368C3F3076101F08001C9B221B143F07B
:104AB000804301E0426D136843F40013136000204B
:104AC00070474B78012B0B78C97800EB83000CBF43
:104AD0008269426D02391368C9B26FF355530129D7
:104AE00098BF43F0805313600020704703699A69B0
:104AF000D8691040000C704700EB81014B6D0269D2
:104B00009B6850691840704703699869DB691840D1
:104B100080B2704782B000230093C0238DF8033029
:104B20000122002362F3C4038DF8023018238DF8AC
:104B30000030009A436D1A61C278012A07D100F54E
:104B4000B8600C3058611A684FF080221A6002B0C9
:104B50007047D0F8183110B50446D3B103699A688C
:104B6000D20716D5827A42B1D0F80C21D0F80C11B8
:104B70006FF341026FF300020A605A68052042F0A9
:104B800001025A60F5F790FF23695A6822F001028A
:104B90005A6010BD837A63B103699B68D90708D551
:104BA000D0F80C31D0F80C216FF341036FF3000300
:104BB00013607047012310B5002280F812310446BB
:104BC0000346FF2104E0586901328160186D81605D
:104BD000607804338242F6D3236900221A615A6155
:104BE000DA614FF0FF329A612046FFF7F3FC20466E
:104BF0001021BDE81040CFE44B78012B0B7800EB7F
:104C000083000FD183691868C0F3074000F02003C8
:104C1000DBB2CBB900F00200C0B200280CBF3020DC
:104C200020207047436D1868C0F3074000F0200350
:104C3000DBB25BB900F00200C0B200280CBF4FF439
:104C400040504FF400507047102070474FF4805090
:104C500070474B7810B5012B0B7800EB83030AD11A
:104C60009C69102A236802D1BDE8104011E7202A70
:104C70000CD0302A0FE05C6DB2F5805F236802D162
:104C800043F400131BE0B2F5005F02D143F0006370
:104C900015E0B2F5405F0FD1C3F3074202F02002E6
:104CA000D2B222B100234B71BDE8104009E743F0B6
:104CB000806343F0802302E00AB962F3CF332360BC
:104CC00010BD00BFF8B50446FFF7B2FB0122002378
:104CD00084F8122184F814312827164619464025F5
:104CE00010E007FB034080F81C31A0F8223180F867
:104CF0001D6180F81F11C0F82451C0F82811C0F8B8
:104D00003011013362789342EBD3002328261946F1
:104D1000402510E006FB034080F87433A0F87A3396
:104D200080F8751380F87713C0F87C53C0F88013AF
:104D3000C0F88813013362789342EBD32046FFF723
:104D400024FC2046FFF7D4FB00212046FFF75CFC43
:104D50002046FFF7B3FC2046BDE8F840FFF70EBC45
:104D600070B5CDB20C464FF0280601F07F0106FB6E
:104D7000010115F0800F14BF01F58E7101F55D7111
:104D800004F07F04ED090C704D708A60CB7005B1A2
:104D9000CC80022B01D100230B71FFF739FD0020DD
:104DA00070BD10B501F07F034FF0280404FB03032E
:104DB000CAB212F0800F14BF03F58E7303F55D7352
:104DC00001F07F01D20919705A701946FFF74FFDA3
:104DD000002010BD38B501F07F05282404FB050430
:104DE00004F55D714B6100238B614B70EBB2CA60BF
:104DF00084F87433C478012C08BF0A6113B9FFF733
:104E0000DBFD01E0FFF752FD002038BD70B501F079
:104E10007F04282505FB040505F58E710126E4B203
:104E2000CA600A61002285F81C414E7005F58C7538
:104E30008A614B6114B9FFF7BFFD01E0FFF736FD52
:104E4000002070BDCAB212F0800F10B54FF02803D9
:104E500006D001F07F0403FB040303F58E7303E027
:104E600003FB010303F55D73D209012401F07F0107
:104E700019709C705A701946FFF70BFE002010BD88
:104E8000CAB212F0800F10B54FF0280306D001F01F
:104E90007F0403FB040303F58E7303E003FB0103AC
:104EA00003F55D730024D20901F07F0119709C7035
:104EB0005A701946FFF705FE204610BD08B50B06CF
:104EC00004D501F07F01FFF767FB01E0FFF782FBEC
:104ED000002008BD0369002261F30A1219680A4321
:104EE0001A607047036903205A686FF341025A60E1
:104EF000F5F7DABD036903205A6842F002025A60EE
:104F0000F5F7D2BD11F0800F4FF0280306D001F065
:104F10007F0103FB010101F58E7103E003FB010139
:104F200001F55D71FFF768BE11F0800F4FF02803A7
:104F300006D001F07F0103FB010101F58E7103E052
:104F400003FB010101F55D71FFF783BE2DE9F04F11
:104F500085B00446FFF772FB002800F05D82204612
:104F6000FFF779FB0546002800F05682C0F30740A2
:104F700000F00800C0B200285AD02046FFF7B6FD66
:104F800027468246A1464FF00008DFF868B32E4658
:104F900049E01AF0010F3FD05FFA88F2114620462F
:104FA0000092FFF7A9FD10F0010F0546009A20D0EE
:104FB0007B6D01259D60E178A94207D11B69D9F875
:104FC0007C13C3F31203CB1AC9F88C33DBF800301F
:104FD00020461B6811469847E378012B09D1B8F1A8
:104FE000000F06D194F81131052B02D12046FFF7AE
:104FF00091FD05F00203DBB213B17B6D02259D60CC
:1050000005F00805EDB23DB1DBF8003020469B68A5
:1050100098477B6D0820986008F101084FEA5A0A0A
:10502000043709F12809BAF1000FB2D13546012041
:10503000C5F3074303F00403DBB2002B00F0A180AB
:105040002046FFF761FD274683464FF00008019593
:1050500091E01BF0010F00F0898023695FFA88F965
:1050600019695D6B04EB890225FA09F59269ED0176
:105070009268EDB20D431540EA071CD5012000FAF5
:1050800008F15A6B054622EA01025A63BB69994A44
:105090009860136820465B6849469847E378AB42BE
:1050A00009D1B8F1000F06D194F81131042B02D1C7
:1050B0002046FFF72FFD05F00803DBB213B1BB69F3
:1050C00008259D6005F01003DBB213B1BB69102504
:1050D0009D6005F04003DBB213B1BB6940259D60C4
:1050E00005F00203DBB213B1BB6902259D6025F018
:1050F0007F0515F0FF0F39D0282505FB084505F57C
:105100008E75AB696A69C246C3EB020CAB68A046F8
:105110009C4528BF9C460CF1030CBB694FEA9C0CD4
:105120009B69664614E0AA681C1B944228BF14467B
:10513000A3B24046E9684A46FFF754F9EB68E61C1B
:105140001B19EB60AB69B6081C19AC61BB699B69A4
:105150009BB2B34205D9AC696B699C4201D2002B6A
:10516000E1D1BB69802544469D60D04608F1010825
:105170004FEA5B0B0437BBF1000F7FF46AAF019D70
:10518000012005F00203DBB213B1E36802225A6189
:10519000C5F3076303F08003DBB2CBB1A37A43B15D
:1051A000D4F80C31D4F80C216FF341036FF30003F2
:1051B0001360236920465A6822F001025A604D4B61
:1051C0001B689B699847E3684FF000425A610120D1
:1051D000C5F3072303F00803DBB2002B2ED0002316
:1051E0008DF80F3094F8123120468DF80F30414B76
:1051F0001B685B6998472369E2684FF400619B680C
:105200005161A27ACAB1DB0717D594F815010128BC
:1052100013D19DF80F30032B10D1D4F80C311A683C
:1052200042F001021A601A6842F003021A60324B1F
:105230001A6942F006021A6100E0012005F0080335
:10524000DBB243B12B4B20461B68DB689847E36811
:1052500008225A61012005F01003DBB2002B34D084
:10526000E36828269A6922F010029A611F6A07F003
:105270000F0306FB0346C7F34343022B06F55D7697
:1052800002D0062B1BD10EE047F6F0733B40B3B1C2
:10529000C7F30A172046F1683A46FFF7B7F8F368F4
:1052A000DB19F36008E004F5B8610C3120460822F0
:1052B000FFF7ACF8C7F30A17B369DF19B761E36802
:1052C00001209A6942F010029A61C5F3072303F0A6
:1052D0001003DBB2002B38D0236900265A68314610
:1052E00022F001025A602046FFF756F92346324663
:1052F000FF2108E02801002000ED00E0586901329C
:105300008160186D8160607804338242F6D323692E
:1053100001274FF0FF3267F30F069A6167F31F46CC
:105320000B22DE615A611A611A6820466FF30A1275
:105330001A60FFF7EFFBE3684FF480525A61384B75
:1053400020461B681B6998473846C5F3072303F0BE
:105350002003DBB2EBB12046FFF744FAE3682046B6
:10536000DE68FFF731FA032806D10023A3704FF45B
:105370000073A380092304E00123A3704023A380CA
:10538000052363F38D26E3684FF40052DE600120AD
:105390005A61C5F3074303F01003DBB24BB1204B56
:1053A00020461B68DB699847E3684FF480125A6116
:1053B0000120C5F3074303F02003DBB24BB1184BC8
:1053C00020461B681B6A9847E3684FF400125A6135
:1053D0000120C5F3076303F04003DBB24BB1104B70
:1053E00020461B685B6A9847E3684FF080425A6129
:1053F000012005F00405EDB275B1E3685D6805F0C4
:105400000403DBB223B1064B20461B689B6A984716
:10541000E36801205D60FFE705B0BDE8F08F00BFE5
:105420002801002081F0004102E000BF83F000432A
:1054300030B54FEA41044FEA430594EA050F08BF2F
:1054400090EA020F1FBF54EA000C55EA020C7FEAF3
:10545000645C7FEA655C00F0E2804FEA5454D4EB70
:105460005555B8BF6D420CDD2C4480EA020281EA3A
:10547000030382EA000083EA010180EA020281EA72
:105480000303362D88BF30BD11F0004F4FEA0131C4
:105490004FF4801C4CEA113102D0404261EB4101D3
:1054A00013F0004F4FEA03334CEA133302D0524259
:1054B00063EB430394EA050F00F0A780A4F1010415
:1054C000D5F1200E0DDB02FA0EFC22FA05F280184F
:1054D00041F1000103FA0EF2801843FA05F3594135
:1054E0000EE0A5F120050EF1200E012A03FA0EFCB4
:1054F00028BF4CF0020C43FA05F3C01851EBE371DE
:1055000001F0004507D54FF0000EDCF1000C7EEBFA
:1055100000006EEB0101B1F5801F1BD3B1F5001F38
:105520000CD349085FEA30004FEA3C0C04F1010457
:105530004FEA445212F5800F80F09A80BCF1004F80
:1055400008BF5FEA500C50F1000041EB045141EA02
:10555000050130BD5FEA4C0C404141EB010111F403
:10556000801FA4F10104E9D191F0000F04BF0146AE
:105570000020B1FA81F308BF2033A3F10B03B3F18C
:1055800020020CDA0C3208DD02F1140CC2F10C021C
:1055900001FA0CF021FA02F10CE002F11402D8BF7A
:1055A000C2F1200C01FA02F120FA0CFCDCBF41EA46
:1055B0000C019040E41AA2BF01EB0451294330BD15
:1055C0006FEA04041F3C1CDA0C340EDC04F11404F2
:1055D000C4F1200220FA04F001FA02F340EA0300C9
:1055E00021FA04F345EA030130BDC4F10C04C4F10F
:1055F000200220FA02F001FA04F340EA03002946EF
:1056000030BD21FA04F0294630BD94F0000F83F438
:10561000801306BF81F480110134013D4EE77FEA1B
:10562000645C18BF7FEA655C29D094EA050F08BF67
:1056300090EA020F05D054EA000C04BF1946104648
:1056400030BD91EA030F1EBF0021002030BD5FEA8C
:10565000545C05D14000494128BF41F0004130BDB4
:1056600014F580043CBF01F5801130BD01F0004508
:1056700045F0FE4141F470014FF0000030BD7FEA7B
:10568000645C1ABF194610467FEA655C1CBF0B4676
:10569000024650EA013406BF52EA033591EA030F8D
:1056A00041F4002130BD00BF90F0000F04BF002185
:1056B000704730B54FF4806404F132044FF00005B8
:1056C0004FF0000150E700BF90F0000F04BF002131
:1056D000704730B54FF4806404F1320410F0004597
:1056E00048BF40424FF000013EE700BF42004FEA92
:1056F000E2014FEA31014FEA02701FBF12F07F430F
:1057000093F07F4F81F06051704792F0000F14BF0B
:1057100093F07F4F704730B54FF4607401F000454F
:1057200021F0004120E700BF50EA010208BF7047A6
:1057300030B54FF000050AE050EA010208BF70479B
:1057400030B511F0004502D5404261EB41014FF404
:10575000806404F132045FEA915C3FF4DCAE4FF008
:1057600003025FEADC0C18BF03325FEADC0C18BFEF
:10577000033202EBDC02C2F1200300FA03FC20FA40
:1057800002F001FA03FE40EA0E0021FA02F114448D
:10579000C1E600BF70B54FF0FF0C4CF4E06C1CEAA2
:1057A00011541DBF1CEA135594EA0C0F95EA0C0F17
:1057B00000F0DEF82C4481EA030621EA4C5123EA8A
:1057C0004C5350EA013518BF52EA033541F48011B9
:1057D00043F4801338D0A0FB02CE4FF00005E1FB6C
:1057E00002E506F00042E0FB03E54FF00006E1FBB6
:1057F00003569CF0000F18BF4EF0010EA4F1FF04F9
:10580000B6F5007F64F5407404D25FEA4E0E6D4138
:1058100046EB060642EAC62141EA55514FEAC52049
:1058200040EA5E504FEACE2EB4F1FD0C88BFBCF5C5
:10583000E06F1ED8BEF1004F08BF5FEA500E50F176
:10584000000041EB045170BD06F0004646EA01013C
:1058500040EA020081EA0301B4EB5C04C2BFD4EB6E
:105860000C0541EA045170BD41F480114FF0000E67
:10587000013C00F3AB8014F1360FDEBF002001F0D5
:10588000004170BDC4F10004203C35DA0C341BDC4F
:1058900004F11404C4F1200500FA05F320FA04F021
:1058A00001FA05F240EA020001F0004221F0004155
:1058B00010EBD37021FA04F642EB06015EEA430EC8
:1058C00008BF20EAD37070BDC4F10C04C4F12005F8
:1058D00000FA04F320FA05F001FA04F240EA0200AB
:1058E00001F0004110EBD37041F100015EEA430E7C
:1058F00008BF20EAD37070BDC4F1200500FA05F29C
:105900004EEA020E20FA04F301FA05F243EA02031A
:1059100021FA04F001F0004121FA04F220EA020029
:1059200000EBD3705EEA430E08BF20EAD37070BD6F
:1059300094F0000F0FD101F00046400041EB01014F
:1059400011F4801F08BF013CF7D041EA060195F031
:10595000000F18BF704703F00046520043EB0303EB
:1059600013F4801F08BF013DF7D043EA06037047D8
:1059700094EA0C0F0CEA135518BF95EA0C0F0CD0E3
:1059800050EA410618BF52EA4306D1D181EA030129
:1059900001F000414FF0000070BD50EA410606BF23
:1059A0001046194652EA430619D094EA0C0F02D168
:1059B00050EA013613D195EA0C0F05D152EA0336AD
:1059C0001CBF104619460AD181EA030101F00041CB
:1059D00041F0FE4141F470014FF0000070BD41F014
:1059E000FE4141F4780170BD70B54FF0FF0C4CF4EE
:1059F000E06C1CEA11541DBF1CEA135594EA0C0F0D
:105A000095EA0C0F00F0A7F8A4EB050481EA030E59
:105A100052EA03354FEA013100F088804FEA033340
:105A20004FF0805545EA131343EA12634FEA02220E
:105A300045EA111545EA10654FEA00260EF00041CF
:105A40009D4208BF964244F1FD0404F5407402D221
:105A50005B084FEA3202B61A65EB03055B084FEAB2
:105A600032024FF480104FF4002CB6EB020E75EBAF
:105A7000030E22BFB61A754640EA0C005B084FEAD7
:105A80003202B6EB020E75EB030E22BFB61A754654
:105A900040EA5C005B084FEA3202B6EB020E75EB9F
:105AA000030E22BFB61A754640EA9C005B084FEA17
:105AB0003202B6EB020E75EB030E22BFB61A754624
:105AC00040EADC0055EA060E18D04FEA051545EA13
:105AD00016754FEA06164FEAC30343EA52734FEABC
:105AE000C2025FEA1C1CC0D111F4801F0BD141EA35
:105AF00000014FF000004FF0004CB6E711F4801F9A
:105B000004BF01430020B4F1FD0C88BFBCF5E06F79
:105B10003FF6AFAEB5EB030C04BFB6EB020C5FEA89
:105B2000500C50F1000041EB045170BD0EF0004EDE
:105B30004EEA113114EB5C04C2BFD4EB0C0541EA10
:105B4000045170BD41F480114FF0000E013C90E60D
:105B500045EA060E8DE60CEA135594EA0C0F08BFD1
:105B600095EA0C0F3FF43BAF94EA0C0F0AD150EAD0
:105B700001347FF434AF95EA0C0F7FF425AF104663
:105B800019462CE795EA0C0F06D152EA03353FF48B
:105B9000FDAE1046194622E750EA410618BF52EA08
:105BA00043067FF4C5AE50EA41047FF40DAF52EADC
:105BB00043057FF4EBAE12E74FF0FF3C06E000BF79
:105BC0004FF0010C02E000BF4FF0010C4DF804CD86
:105BD0004FEA410C7FEA6C5C4FEA430C18BF7FEA46
:105BE0006C5C1BD001B050EA410C0CBF52EA430C74
:105BF00091EA030F02BF90EA020F0020704710F1F4
:105C0000000F91EA030F58BF994208BF90422CBF82
:105C1000D8176FEAE37040F0010070474FEA410C7B
:105C20007FEA6C5C02D150EA013C07D14FEA430C99
:105C30007FEA6C5CD6D152EA033CD3D05DF8040B0A
:105C4000704700BF8446104662468C46194663463C
:105C500000E000BF01B5FFF7B7FF002848BF10F113
:105C6000000F01BD4DF808EDFFF7F4FF0CBF012058
:105C700000205DF808FB00BF4DF808EDFFF7EAFFD4
:105C800034BF012000205DF808FB00BF4DF808ED8F
:105C9000FFF7E0FF94BF012000205DF808FB00BF84
:105CA0004DF808EDFFF7CEFF94BF012000205DF80E
:105CB00008FB00BF4DF808EDFFF7C4FF34BF01201B
:105CC00000205DF808FB00BF4FEA410212F5001208
:105CD00015D211D56FF47873B3EB625212D94FEA33
:105CE000C12343F0004343EA505311F0004F23FA1D
:105CF00002F018BF404270474FF00000704750EA72
:105D0000013005D111F0004008BF6FF0004070472E
:105D10004FF00000704700BF4FEA4102B2F1E0438C
:105D200024BFB3F5001CDCF1FE5C0DD901F0004C82
:105D30004FEAC0024CEA5070B2F1004F40EB8300D2
:105D400008BF20F00100704711F0804F21D113F1FE
:105D50003872BCBF01F00040704741F480114FEA37
:105D60005252C2F11802C2F1200C10FA0CF320FAC0
:105D700002F018BF40F001004FEAC1234FEAD323DD
:105D800003FA0CFC40EA0C0023FA02F34FEA430347
:105D9000CCE77FEA625307D150EA01331EBF4FF0D0
:105DA000FE4040F44000704701F0004040F0FE40EB
:105DB00040F40000704700BF80F0004002E000BFE8
:105DC00081F0004142001FBF5FEA410392EA030FE6
:105DD0007FEA226C7FEA236C6AD04FEA1262D2EB30
:105DE0001363C1BFD218414048404140B8BF5B4235
:105DF000192B88BF704710F0004F40F4000020F0CE
:105E00007F4018BF404211F0004F41F4000121F0E3
:105E10007F4118BF494292EA030F3FD0A2F101022D
:105E200041FA03FC10EB0C00C3F1200301FA03F16B
:105E300000F0004302D5494260EB4000B0F5000F8E
:105E400013D3B0F1807F06D340084FEA310102F14D
:105E50000102FE2A51D2B1F1004F40EBC25008BFFF
:105E600020F0010040EA03007047490040EB0000C9
:105E700010F4000FA2F10102EDD1B0FA80FCACF1F8
:105E8000080CB2EB0C0200FA0CF0AABF00EBC250F7
:105E900052421843BCBFD0401843704792F0000FE5
:105EA00081F4000106BF80F400000132013BB5E738
:105EB0004FEA41037FEA226C18BF7FEA236C21D0AE
:105EC00092EA030F04D092F0000F08BF0846704713
:105ED00090EA010F1CBF0020704712F07F4F04D1E1
:105EE000400028BF40F00040704712F100723CBFF4
:105EF00000F50000704700F0004343F0FE4040F41E
:105F0000000070477FEA226216BF08467FEA2363DB
:105F10000146420206BF5FEA412390EA010F40F4C6
:105F2000800070474FF0000304E000BF10F0004312
:105F300048BF40425FEA000C08BF704743F09643F9
:105F400001464FF000001CE050EA010208BF704714
:105F50004FF000030AE000BF50EA010208BF70479B
:105F600011F0004302D5404261EB41015FEA010CB0
:105F700002BF84460146002043F0B64308BFA3F1A8
:105F80008053A3F50003BCFA8CF2083AA3EBC2538A
:105F900010DB01FA02FC634400FA02FCC2F12002A9
:105FA000BCF1004F20FA02F243EB020008BF20F0E0
:105FB0000100704702F1200201FA02FCC2F1200246
:105FC00050EA4C0021FA02F243EB020008BF20EA3B
:105FD000DC7070474FF0FF0C1CEAD0521EBF1CEA69
:105FE000D15392EA0C0F93EA0C0F6FD01A4480EA57
:105FF000010C400218BF5FEA41211ED04FF0006340
:1060000043EA501043EA5111A0FB01310CF000406B
:10601000B1F5000F3EBF490041EAD3715B0040EA91
:10602000010062F17F02FD2A1DD8B3F1004F40EB61
:10603000C25008BF20F00100704790F0000F0CF034
:10604000004C08BF49024CEA502040EA51207F3AF8
:10605000C2BFD2F1FF0340EAC250704740F40000D3
:106060004FF00003013A5DDC12F1190FDCBF00F0C4
:1060700000407047C2F10002410021FA02F1C2F172
:10608000200200FA02FC5FEA310040F1000053EA0E
:106090004C0308BF20EADC70704792F0000F00F05C
:1060A000004C02BF400010F4000F013AF9D040EA62
:1060B0000C0093F0000F01F0004C02BF490011F4F6
:1060C000000F013BF9D041EA0C018FE70CEAD153F4
:1060D00092EA0C0F18BF93EA0C0F0AD030F0004C74
:1060E00018BF31F0004CD8D180EA010000F0004028
:1060F000704790F0000F17BF90F0004F084691F0E6
:10610000000F91F0004F14D092EA0C0F01D142021F
:106110000FD193EA0C0F03D14B0218BF084608D1E8
:1061200080EA010000F0004040F0FE4040F4000032
:10613000704740F0FE4040F4400070474FF0FF0CC5
:106140001CEAD0521EBF1CEAD15392EA0C0F93EA0C
:106150000C0F69D0A2EB030280EA010C49024FEA5E
:10616000402037D04FF0805343EA111143EA101317
:106170000CF000408B4238BF5B0042F17D024FF4CF
:10618000000C8B4224BF5B1A40EA0C00B3EB510FAA
:1061900024BFA3EB510340EA5C00B3EB910F24BF93
:1061A000A3EB910340EA9C00B3EBD10F24BFA3EB18
:1061B000D10340EADC001B0118BF5FEA1C1CE0D1E0
:1061C000FD2A3FF650AF8B4240EBC25008BF20F093
:1061D000010070470CF0004C4CEA50207F32C2BFE7
:1061E000D2F1FF0340EAC250704740F400004FF084
:1061F0000003013A37E792F0000F00F0004C02BFB5
:10620000400010F4000F013AF9D040EA0C0093F07E
:10621000000F01F0004C02BF490011F4000F013BD8
:10622000F9D041EA0C0195E70CEAD15392EA0C0F40
:1062300008D142027FF47DAF93EA0C0F7FF470AF78
:10624000084676E793EA0C0F04D14B023FF44CAFBB
:1062500008466EE730F0004C18BF31F0004CCAD150
:1062600030F000427FF45CAF31F000437FF43CAF8C
:106270005FE700BF4FEA4002B2F1FE4F0FD34FF08D
:106280009E03B3EB12620DD94FEA002343F00043A3
:1062900010F0004F23FA02F018BF404270474FF051
:1062A0000000704712F1610F01D1420205D110F0D8
:1062B000004008BF6FF0004070474FF0000070478B
:1062C00042000ED2B2F1FE4F0BD34FF09E03B3EB60
:1062D000126209D44FEA002343F0004323FA02F08C
:1062E00070474FF00000704712F1610F01D1420278
:1062F00002D14FF0FF3070474FF00000704700BFF1
:1063000073B96AB9002908BF0028BCBF00204FF04C
:106310000041C4BF6FF000414FF0FF3001F072B890
:1063200082B0EC462DE9005000F006F8DDF804E0FC
:1063300002B00CBC704700BF2DE970431546804683
:1063400089461C4601F060F805FB01F6A5FB002319
:1063500000FB0464E318069CB8EB020269EB03033C
:10636000C4E90023BDE87083F8B5144606460F461D
:106370001D4601F0ADF900FB05F5A0FB042304FB6D
:106380000154E318069CB21A67EB0303C4E9002327
:10639000F8BD00BF036803B11B181846704700BF63
:1063A00003685A004CBF43F0004323F00043C01879
:1063B000704700BF2DE9F84F0446914641B301F103
:1063C000FF3BDA46002707EB0A0000EBD0756D10A3
:1063D00004EBC5063046FFF7E3FFAB45804610D01F
:1063E000691C04EBC100FFF7DBFF0138C84504D985
:1063F000BD4209D005F1FF3AE5E7484505D26F1CDB
:10640000E1E74FF0FF30F1E700263046BDE8F88FB6
:106410000E463046BDE8F88F30B52B4B83B00446AE
:106420008D1E002B49D0284601A9AFF300800346FA
:10643000002822D02A4618460199FFF7BBFF0546DF
:1064400000281DD0FFF7ACFF6B68A064012B10D0B3
:10645000281D002B22DBFFF7A3FF0021E06421654C
:106460000368002B0FDBFFF79BFF2061002003B0C8
:1064700030BD002323610520F9E720610920F6E7FC
:1064800020610920F3E7C3F3036058B101280CD061
:1064900002280ED0002020610920E8E70122E064F4
:1064A0002265DDE7094B2361E1E7094A002022610B
:1064B000DDE7084900202161D9E7074A074913466B
:1064C000881AC2100192B5E700000000DD690108DA
:1064D000D9690108D5690108E49A0108CC9B010833
:1064E000036810B50446D80706D4990704F148009C
:1064F00009D500F009FD23685A0709D518070ED5FC
:10650000D90613D510BD00F0F7FC23685A07F5D45F
:1065100004F1D00000F000FD23681807F0D404F562
:10652000D87000F001FD2368D906EBD404F50C7097
:10653000BDE8104000F03CBD2DE9F047ADF5916D90
:1065400002AC0F1D261D054691460FCF0FC60FCF7B
:106550000FC60FCF0FC697E80F00D5F80C800027A5
:10656000D5F818A086E80F00216C28462760FFF7B1
:1065700053FF0646B94514BF4FF00A094FF0090909
:10658000FEB1A16B49F01009616401208DE810048F
:1065900049462A462B46C04700282BD1002E2AD137
:1065A000204692A94FF4107201F048FE082F28D11E
:1065B000216C2846FFF730FF06464FF00909002EF0
:1065C000DFD1206C21464FF41072686192A801F06F
:1065D00035FE2F69294692AA4846B847A09B074630
:1065E000636401208DE8100449462A462B46C047C3
:1065F0000028D3D00926304622B00DF5806DBDE8C5
:10660000F087072FF6D1201D00F06AFC38B504464C
:106610000D46296C2046FFF7FFFE50B92A6C012079
:106620006261236921462A4698470828F1D0072845
:1066300001D001F0FBFD281D00F052FC11B933B16F
:106640000220704704298CBF0220012070470F2AC6
:1066500001D90220704700EB820042681846009B77
:106660001A60704710B50A4684B000210B4603AC8F
:106670000094FFF7E3FF039804B010BD11B933B1E4
:106680000220704704298CBF0220012070470F2A86
:1066900001D902207047009900EB82020968184670
:1066A0005160704700B585B004AB43F8042D0A462D
:1066B000002100930B46FFF7E1FF05B000BD00BFCE
:1066C0002DE9F04FCD6C0C4655F8041B8BB01746E6
:1066D00000F008021E46039200F003080795002B05
:1066E00040F0E08009020691216D8DF821300323EE
:1066F000B8F1020F8DF8203008BFA56B11F001032F
:1067000040F0E480019304F158030293D5F800901F
:10671000B9F1000F00F0DC80022E00F0BF80B5F868
:106720000090B5F802A00435A26C0F212AF0010BED
:1067300038469344FFF796FF834518D829F0010C9B
:10674000E3440AF0010A09F00103584543EA4A0903
:106750002CBF00200120B9F1010F12D032D2B8F1C4
:10676000000F02D0002840F017810435CEE70AF070
:10677000010A09F0010343EA4A090020B9F1010FB7
:10678000ECD1B8F1000F40F0C880C8B16B68D5F803
:1067900000909A1C19D0029A013309920DD0281D3D
:1067A000FFF7F8FD4FEAD972014609AB2046AFF377
:1067B0000080002800F0EC80099A002A40F0CC808C
:1067C0000835A3E7B9F1020F03D009200BB0BDE8EB
:1067D000F08F2B6823F000420092B8F1000F40F0D8
:1067E0008380002853D00398002840F0B28000989E
:1067F000002800F0B180009B05F1040ADB07DDF8FA
:106800000C9010D4029950460991FFF7C3FD039AEA
:10681000014609AB2046AFF30080002833D10AF1CE
:10682000040A4FF00109CDF81080AB46B846504637
:106830000596029F11E000998E4200F0C0800997F2
:10684000FFF7A8FD5246014609AB2046AFF3008092
:10685000B14698B9281D06F10109051D0997FFF7F2
:1068600099FD09AB014600222046AFF30080824625
:1068700009F101062846BAF1000FDCD04746059E13
:10688000DDF810805D46009A4A4565D02B68002BE4
:106890007CDB0099481C05EB800537E7D5F804A0A0
:1068A000083541E70B04C1F30740216D0222B8F11E
:1068B000020F069305EB800508BFA56B11F00103DD
:1068C0008DF821008DF820203FF41CAF00200190AE
:1068D000384606A900F004FC00287FF476AF019A40
:1068E000002A43D1082071E70D213846D4F82090C2
:1068F000FFF7B8FE8145C9D1A26A9542C6D100987A
:10690000291D00220423A062E262236361632868D8
:10691000002857DB01220192BBE70D213846D4F84D
:106920002090FFF79FFE81457FF44AAFA16A8D4218
:106930007FF446AF2846FFF733FD0F210246384665
:10694000FFF7B0FE384600212246FFF7ABFE0720D6
:106950003CE7009900299AD138460D21FFF782FEC5
:10696000099B20626362A56206202FE70F2138464B
:10697000FFF778FE0E2102463846FFF793FE3846B1
:106980000F21134AFFF78EFE07201FE7043580E72B
:10699000CDF824800835B9E62846FFF701FD043517
:1069A0000646A5632046AFF3008000283FF40DAFF4
:1069B00038460F213246FFF775FE072006E75D4691
:1069C0004746C9E7009B591C05EB8100B3E700BFB0
:1069D00000000000022373E6012371E600236FE646
:1069E0002DE9F0470446E8B004290CD8DFE801F0AF
:1069F000390392940F00150C012B96B200F07881A8
:106A0000052B00F0C880022068B0BDE8F087002B9D
:106A1000F9D1102AF7D82368D90600F1738164A848
:106A2000019200F0CFFA019AA36BD00744BF53F84C
:106A3000040B6490910744BF53F8041B6591500701
:106A400048BF53F8041B64A848BF6691110748BFAC
:106A500053F8042BA36348BF679200F0A9FA002003
:106A6000D2E7002BCFD1A36BD00791B244BF53F82C
:106A7000042B62608A0744BF53F8042BA2604807C6
:106A800044BF53F8042BE2600A0744BF53F8042BB9
:106A90002261C80644BF53F8042B62618A0644BFD2
:106AA00053F8042BA261480644BF53F8042BE2615B
:106AB0000A0644BF53F8042B2262C80544BF53F8AA
:106AC000042B62628A0544BF53F8042BA262480576
:106AD00044BF53F8042BE2620A0544BF53F8042B69
:106AE0002263C80444BF53F8042B626311F40050BE
:106AF0001CBF53F8042BA2634A0444BF53F8042B71
:106B0000E2630A0444BF53F8042B2264002840D1F6
:106B1000A36379E7012077E7032B7FF474AF160CAA
:106B200095B2AA19102A3FF66EAF2368180700F134
:106B30000A8144A800F01AFAA76B4FEA450E3B46BB
:106B40000DB30EF1FF3C44A953F8040B01EBC6064C
:106B500062460CF0010146F8040B92B129B153F8DA
:106B6000041B013A46F8041B0BD0184650F8045B8E
:106B7000314641F8045B5D68031D75600E1D023AE5
:106B8000F3D107EB8E0344A8A36300F0CDF90020F6
:106B90003AE7002038E777192022BA42FFF433AFF2
:106BA000012B00F0A8800F2D40F2A8803746F6B1E7
:106BB000052B7FF428AF0F2D11D82268D0070ED5F2
:106BC00022F00101052B216000F0DA8022F003029F
:106BD000204640F8482B019300F092F9019B1FB129
:106BE0002268510700F1B780012B00F0BE800F2D05
:106BF00074D9002F40F09F80D4F83890002EC846FA
:106C00002EDD49464FEA46080DF1080C51F8046B99
:106C10000CEBC50208F1FF3000F0010A42F8046BEA
:106C2000A8F1020CD0B1BAF1000F08D051F8040B52
:106C30000CF1FF3CBCF1FF3F42F8040B0ED00E46B6
:106C400056F804AB104640F804AB4968ACF1020CAE
:106C50005160311D021DBCF1FF3FF0D109EB8808E6
:106C60009FB3102D2CBF2E46102668AA414602EB7A
:106C7000C60A4FEA470951F8046BAAF5C87209F130
:106C8000FF3000F0010A42F8046BA9F1020CD0B108
:106C9000BAF1000F08D051F8040B0CF1FF3CBCF125
:106CA000FF3F42F8040B0ED00E4656F804AB1046D8
:106CB00040F804AB4968ACF1020C5160311D021D73
:106CC000BCF1FF3FF0D108EB8908012B2BD00F2D31
:106CD000C4F8388008D9FFB9384695E602A8019370
:106CE00000F016F9019B84E702A800F00DF9F2E725
:106CF0007719102251E70F2D3FF685AE102F10D9CE
:106D0000103F55E723F01003236004F50C70019247
:106D100000F058F9019A82E624A800F0FDF800205E
:106D200072E6002747E708F1040302A8A36300F016
:106D3000E3F8002068E624A80193C5F1100600F0EE
:106D4000EFF8019B58E723F0080704F5D870276097
:106D500000F00CF9EDE622F00401204640F8D01BCB
:106D6000019300F0DDF8019B3EE702A8019300F0DB
:106D7000C7F8019B002F3FF43FAFC5F110063BE77A
:106D800041F00201204640F8481B019300F0C0F892
:106D9000019B24E7406C7047F0B50D46C96BADF51B
:106DA000117D296401AE2F1D04460FCF0FC60FCFF2
:106DB0000FC60FCF0FC697E80F0086E80F004FF001
:106DC000FF33009310992046FFF726FB58B9266938
:106DD00021466A46B04708280646F3D06846FFF7C2
:106DE0007FFB062E03D009200DF5117DF0BD204656
:106DF0002946FFF70BFC00BF10B4DC6BC160826159
:106E0000194600221C6410BCFFF796BB38B54269D6
:106E1000C36804460D460A6423B10122FFF78CFBC8
:106E200001F004FA0369214602202A469847072800
:106E300003D0082804D001F0F9F9281D00F050F81B
:106E400020462946FFF7E2FBC36823B1CA6B0A64F8
:106E50000022FFF771BB9FE7704700BF08B583684A
:106E600001460BB10120984708BD00BFF0B5D46BB7
:106E7000ADF5277D146401AE171D05460C460FCFF6
:106E80000FC60FCF0FC60FCF0FC697E80F0086E8CB
:106E90000F004FF0FF330093109990A8FFF7BCFA52
:106EA000034690AA68460C21BBB9FFF7FBFB2146BD
:106EB0006846A847064690A908206A466EB9949B82
:106EC00098470528064601D00928E5D16846FFF70E
:106ED00007FB30460DF5277DF0BD0926F6E700BF1C
:106EE00000F1340191E838009C46A6464CF8045D58
:106EF00090E8FF0FE54600BD90EC210B704700BF06
:106F000080EC210B704700BF90EC200B704700BF56
:106F100080EC200B704700BFD0EC200B704700BF07
:106F2000C0EC200B704700BFF0EC0201F0EC021146
:106F3000F0EC0221F0EC0231F0EC0241F0EC0251F5
:106F4000F0EC0261F0EC0271F0EC0281F0EC0291E5
:106F5000F0EC02A1F0EC02B1F0EC02C1F0EC02D1D5
:106F6000F0EC02E1F0EC02F1704700BFE0EC02014E
:106F7000E0EC0211E0EC0221E0EC0231E0EC024135
:106F8000E0EC0251E0EC0261E0EC0271E0EC028125
:106F9000E0EC0291E0EC02A1E0EC02B1E0EC02C115
:106FA000E0EC02D1E0EC02E1E0EC02F1704700BF5E
:106FB000B0FC0181B0FC0191B0FC01A1B0FC01B1B9
:106FC000704700BFA0FC0181A0FC0191A0FC01A1C1
:106FD000A0FC01B1704700BFEC4600B52DE90050A0
:106FE0002DE9FF1F4FF000032DE90C0001A9FFF769
:106FF000D3FEDDF840E012B0704700BFEC4600B5AC
:107000002DE900502DE9FF1F4FF000032DE90C0082
:1070100001A9FFF7FBFEDDF840E012B0704700BFAA
:10702000EC4600B52DE900502DE9FF1F4FF000039D
:107030002DE90C0001A9FFF707FFDDF840E012B0D1
:10704000704700BFEC4600B52DE900502DE9FF1F49
:107050004FF000032DE90C0001ABFFF7CDFEDDF88A
:1070600040E012B0704700BFEC4600B52DE900507B
:107070002DE9FF1F4FF000032DE90C0001AAFFF7D7
:10708000F5FEDDF840E012B0704700BF027A03461B
:107090001AB9427A42B9B02070470068013A010239
:1070A0001A72000E196070474168501E587251F8EC
:1070B000040B0322596001021A72000E1960704716
:1070C00010B5002184B00C220DEB02040B46009495
:1070D000FFF7B4FA039804B010BD00BFF0E700BF9B
:1070E0002DE9F043064685B00D464FF000094FF4F8
:1070F0007F672846FFF7CAFFB028044600F0B1803A
:1071000010F0800120D000F0F003802B75D0902B80
:1071100037D0A02B45D0B02B56D0C02B00F08680A6
:1071200000F0F800D0280BD104F007035A1C42F4F9
:107130000022304601210523FFF752FC0028D8D059
:10714000092005B0BDE8F0834FEA800203A85FFA8A
:1071500082F800900D220B463046FFF76FFA039B32
:10716000600608F104084CBFC8EB0303434403ACBA
:1071700003930094002130460D220B46FFF77EFA60
:10718000B7E700F00F020D2ADAD00F2AD8D000217D
:1071900003AC009430460B4603ACFFF74FFA009463
:1071A000E8E7C24302F0070C47FA0CF0210700F4AD
:1071B0007F6248BF42F48042002130460B46FFF711
:1071C0000FFC0028BCD194E7B1285ED0B2286FD064
:1071D000B32800F0968000F0FC0CBCF1B40F46D050
:1071E00000F007014A1C42F40022012130460B4600
:1071F000FFF7F6FB0028A3D17BE72846FFF746FF01
:10720000210240EA0104B4F5004F99D02305002182
:107210001A0C30460B462401FFF7E2FB00288FD101
:1072200014F4004F18BF4FF0010962E7C62873D06D
:10723000C72800F0848000F0F801C02900F0928097
:10724000C82800F0A680C9287FF47AAF2846FFF747
:107250001DFF00F00F0100F0F0024B1C43EA023268
:1072600067E7B9F1000F00F08380002069E700F0C4
:107270000300431C022143F4802230460B46FFF7F3
:10728000AFFB00287FF45CAF33E72846FFF7FEFE34
:10729000024600283FF454AF10F0F0017FF450AFE5
:1072A00030460B46FFF79CFB00287FF449AF20E7F0
:1072B00000210D220B4603AC30460094FFF7BEF9C7
:1072C0002846FFF7E3FE022402060DD500F07F00FA
:1072D00000FA04FE039B284603EB0E010391FFF71F
:1072E000D5FE07340306F1D400F07F0E0EFA04F445
:1072F000039903AB01F5017C0CEB040200930392AC
:1073000038E72846FFF7C2FE00F00F014A1C00F0E4
:10731000F00042EA003268E72846FFF7B7FE00F0C7
:107320000F02531C00F0F00043EA00320321304604
:107330000B46FFF755FB00287FF402AFD9E628463D
:10734000FFF7A4FE024600283FF4FAAE10F0F00367
:107350007FF4F6AE30460421FFF742FB00287FF4AD
:10736000EFAEC6E600F00F03581C40F42022DDE724
:1073700003AC49460E224B4630460094FFF75EF9B7
:10738000304649460F224B460094FFF777F94846AE
:10739000D7E62846FFF77AFE00F0F00200F00F0073
:1073A0001032411C41EA0232C3E600BF10B5C26C84
:1073B00084B0032054688DF80C00D379240208327D
:1073C000084601A9019402928DF80D30FFF788FE5E
:1073D00004B010BD08B5FFF781FE806C08BD00BF8A
:1073E00008B5FFF77BFEC16CC87901EB800303F1A0
:1073F000080008BD08B500F019FF00BF08B500F08F
:1074000015FF00BF704700BF2DE9F00F00291D4692
:10741000C0F29D800024002DC0F2948007460D46E6
:1074200016469C46002B3DD18A4253D9B2FA82F3CC
:1074300043B1C3F1200620FA06F501FA03F19A40A0
:1074400098402943130CB1FBF3F697B203FB1611D6
:1074500007FB06F54FEA104C4CEA01418D4209D971
:10746000891806F1FF3C80F014818D4240F21181B1
:10747000023E8918491BB1FBF3F503FB151307FB0B
:1074800005F780B240EA03439F4207D9691E9B1863
:1074900080F005819F4240F20281023D45EA0642AA
:1074A000002303E08B420AD900231A4610461946EE
:1074B00014B1404261EB4101BDE8F00F7047B3FAEF
:1074C00083F3002B40F087808C4501D38242ECD8B7
:1074D0000122EBE712B90127B7FBF2F2B2FA82F60A
:1074E000002E3AD1891A150C1FFA82FC0123B1FB38
:1074F000F5F705FB17110CFB07F64FEA104848EAB1
:1075000001418E4207D9891807F1FF3802D28E4215
:1075100000F2DA804746891BB1FBF5F605FB161130
:107520000CFB06FC80B240EA0140844507D9711E7D
:10753000821880F0B080944540F2AD80023E46EA69
:107540000742B3E7E443524263EB430366E740423A
:1075500061EB41014FF0FF345DE7B240C6F1200519
:1075600021FA05F320FA05F901FA06F1150CB3FB2F
:10757000F5F805FB18371FFA82FC0CFB08F349EA03
:1075800001094FEA194141EA0747B040BB420AD915
:10759000BF1808F1FF3180F09580BB4240F2928025
:1075A000A8F10208BF18FE1AB6FBF5F305FB136736
:1075B0000CFB03F61FFA89F949EA07418E4206D906
:1075C0005F1E891878D28E4276D9023B8918891BB2
:1075D00043EA08438BE7C3F1200122FA01F80CFAD1
:1075E00003F725FA01FB20FA01F205FA03F548EA50
:1075F000070C4FEA1C48BBFBF8F908FB19B71FFA48
:107600008CFA0AFB09FB15432A0C42EA0747BB45E3
:1076100006FA03F609D917EB0C0709F1FF324FD22E
:10762000BB454DD9A9F102096744CBEB0701B1FB7A
:10763000F8F208FB12170AFB02FAADB245EA07415D
:107640008A4507D9551E11EB0C0137D28A4535D929
:10765000023A614442EA09421FFA86F84FEA124CA4
:1076600008FB0CF7360C95B208FB05F806FB057510
:1076700006FB0CFC05EB1845AF4288BF0CF5803CBF
:10768000CAEB01010CEB1546B14212D309D000231D
:107690000CE76646EEE60E4646EA074206E70D466A
:1076A000FCE600FA03F31FFA88F808EB0545AB4245
:1076B000EDD2013A0023F9E63B4688E72A46C9E7BE
:1076C0009146B2E788466EE7023F891823E700BF7C
:1076D0002DE9F007144605460E46002B3FD18A429D
:1076E0004AD9B2FA82F343B1C3F1200025FA00F27D
:1076F00001FA03F69C409D401643230CB6FBF3F1C0
:10770000A0B203FB116C00FB01F22F0C47EA0C4600
:10771000B24208D94F1E361980F0FF80B24240F2C3
:10772000FC8002393619B61AB6FBF3F203FB12637A
:1077300000FB02F0ADB245EA0343984207D9561E5A
:107740001B1980F0EC80984240F2E980023A42EA4C
:107750000142002310461946BDE8F00770478B42EE
:1077600043D8B3FA83F4002C42D18B42234601D391
:1077700082423BD80122EDE712B90127B7FBF2F4B0
:10778000B4FA84F2002A40F08A80091B260CA7B2C2
:107790000123B1FBF6F006FB101107FB00F24FEAE4
:1077A000154C4CEA01418A4207D9091900F1FF3C06
:1077B00002D28A4200F2D4806046C2EB010CBCFBCC
:1077C000F6F206FB12C107FB02F7ADB245EA01452E
:1077D000AF4207D9511E2C1980F0A380A74240F276
:1077E000A080023A42EA0042B4E700231A46B1E719
:1077F000C4F1200703FA04F822FA07F321FA07F983
:1078000020FA07FA01FA04F143EA08031E0CB9FB57
:10781000F6FC06FB1C991FFA83F808FB0CF74AEAF2
:10782000010A4FEA1A4545EA0945AF4202FA04F94E
:1078300005D9ED180CF1FF32C0F087809446EA1BA1
:10784000B2FBF6F706FB172608FB07F81FFA8AFAC1
:107850004AEA0641884503D97A1EC91870D31746EB
:1078600047EA0C42170C1FFA89FC0CFB07F695B28D
:107870004FEA19430CFB05FC03FB056503FB07F30B
:1078800005EB1C45AE4288BF03F58033C8EB010110
:1078900003EB1543994250D347D000235AE7944055
:1078A000C2F1200621FA06F520FA06F901FA02F1E2
:1078B000260CB5FBF6F806FB1855A7B207FB08F334
:1078C00049EA01094FEA194141EA054C634500FACA
:1078D00002F509D91CEB040C08F1FF323ED26345D6
:1078E0003CD9A8F10208A444C3EB0C02B2FBF6F3A6
:1078F00006FB132007FB03F21FFA89F949EA00414E
:107900008A4206D9581E091926D28A4224D9023B36
:107910000919891A43EA08433BE7394603E7324627
:1079200015E70A4642EA004214E700FA04F01FFA9B
:107930008CF101EB0545A842AFD2013A002309E7DB
:1079400088458CD9023FC9188AE7AF427FF676AFE7
:10795000ACF1020CED1872E70346DAE79046C3E794
:107960000238091929E700BF002103E00A4B5B58E0
:107970004350043109480A4B42189A42F6D3094A47
:1079800002E0002342F8043B074B9A42F9D3F9F78F
:107990004DFB00F00DF87047D89B01080000002057
:1079A00004060020080600202C620020FEE70000EC
:1079B00010B562B61B4CF0F75FFCF1F797FDF0F7DE
:1079C00041FCF1F785FEF2F7ABF92078F1F732F9D7
:1079D00022696079A168F1F7C3FBF3F7B7F8F2F712
:1079E00011FCF0F757FFF9F77BFAF5F735FEF6F7DC
:1079F00067FBF6F7BFFD0C4B04225A83F5F722FF15
:107A0000F6F75FFBF6F7D4FDF0F716FEF0F738FE59
:107A10000028F3D0F2F7F6FBF5F71EFEF6F7AAFD05
:107A2000ECE700BF040000200010024001460020E7
:107A30000246034600F0DAB800210A2200F0C8B876
:107A400038B5084D084C641BA41006D005EB84051E
:107A500055F8043D9847013CFAD1BDE8384002F0A2
:107A600023B800BFD49B0108D89B01080F4B70B40A
:107A70001E68054615F8013B11F8014BF2185078C5
:107A80001A4600F00300012808BF03F12002331951
:107A90005878234600F00300012808BF04F12003B2
:107AA000D01A01D1002BE5D170BC7047FC05002035
:107AB0002DE9F00F454C82B0246801900846057806
:107AC0000646671997F801A001301AF0080A074620
:107AD000F5D12D2D5BD02B2D04BF7578B71C002B55
:107AE00042D0102B40D099466619BAF1000F767833
:107AF0000CBF6FF0004B4FF0004BBBFBF9F84FF0A1
:107B0000000C16F0040F09FB18BB604613D0303D83
:107B1000AB421ADDBCF1FF3F06D040452ED82BD03A
:107B200009FB00504FF0010C17F8015B66197678DD
:107B300016F0040FEBD116F0030606D0012E14BF89
:107B400057263726AD1BAB42E4DCBCF1FF3F23D008
:107B5000BAF1000F19D11AB1BCF1000F13D11160A5
:107B600002B0BDE8F00F7047302D20D0002BBAD105
:107B7000302D27D00A23B6E75D45D1DD4FF0FF3C1D
:107B800017F8015BD2E7791EE9E74042E3E7757831
:107B9000B71C4FF0010AA2E7BAF1000F019C0CBF1D
:107BA0006FF000404FF0004022232360D3E7387885
:107BB000782801D05828D9D14FF010097D784B464C
:107BC000023791E7082399468EE700BFFC050020A5
:107BD00030B440F2F853C2F200031D680C4613465D
:107BE00001462246284630BCFFF762BF2DE9F0412E
:107BF0000546274884B00468D4F84801002841D0DD
:107C000046681F2E1CDD234810B94FF0FF301EE0E0
:107C10004FF4C870039102920193AFF3008003996F
:107C2000029A019B0028F0D0D4F84861002780E830
:107C3000C000C4F848013E46C0F88871C0F88C7195
:107C400045B9B31C013640F823104660002004B04B
:107C5000BDE8F081012404FA06F4D0F8887100EB45
:107C6000860847EA040C022D4746C8F88820C0F869
:107C700088C1C8F80831E4D1D0F88C311C43C0F871
:107C80008C41DEE704F5A670C4F84801B8E700BFF0
:107C90008C99010800000000024B13B10248FFF765
:107CA000C5BE704700000000417A01082DE9D043AD
:107CB0008AB006460F4600F077F8384C804694F9B3
:107CC00000308946013336D03046394600F06CFA30
:107CD000002830D03046394600220023FDF7EAFF65
:107CE000002828D12E4B2478019300230893CDE956
:107CF0000267CDE90467002C22D04FF000094FF055
:107D00000008CFF6F0793046394600220023CDE94D
:107D10000689FDF7A7FF002822D002239C4200938A
:107D200031D0684600F074FA00282CD0089B002B54
:107D300024D1DDE90689404649460AB0BDE8D08332
:107D40004FF6FF794FF06048CCF2EF793046394674
:107D500000220023CDE90689FDF784FF0028DCD14D
:107D60000123022C009313D0684600F051FA78B139
:107D70000C4800F04FFACDE90601D7E700F050FAC1
:107D8000089B0360D5E700F04BFA22230360CDE7A0
:107D900000F046FA21230360EAE700BF0006002056
:107DA000949A0108989A01082DE9F04FB1F5801FC7
:107DB00087B00B460C465FDA21F00043034300F026
:107DC000FD800029C0F2AC8100230022C4F25033B0
:107DD000FDF7E0FC4FF6FF720B46C7F6EF729342D9
:107DE0006FF035074FDC23F07F4545F6647425F4CA
:107DF0007005C0F209042C1904F4801484F07E523A
:107E00001E1582F4E002002342EA0501C3F6F07376
:107E10000022FDF70BFBA6F57E76AB1C073E23F494
:107E20007003F6190022022B06EB145482468B468F
:107E300030DC0023FDF716FF002800F0C880002C7E
:107E400000F077812046FDF73FFCA1A3D3E9002392
:107E500004460D46FDF79EFC9FA3D3E9002306468A
:107E60000F4620462946FDF795FC02460B46304654
:107E70003946FDF7DDFA0AE04FF6FF72C7F6EF72FA
:107E800000279342AFDD02460B46FDF7D1FA07B05B
:107E9000BDE8F08F4FF08043FDF7CAFA02460B466B
:107EA00050465946FDF7A0FDCDE900012046FDF7FB
:107EB0000BFCCDE90201DDE9000102460B46FDF7AE
:107EC00069FC02460B4680468946FDF763FC84A3A5
:107ED000D3E9002306460F46FDF75CFC82A3D3E9F5
:107EE0000023FDF7A5FA32463B46FDF753FC80A37D
:107EF000D3E90023FDF79CFA32463B46FDF74AFCE6
:107F00007DA3D3E90023FDF793FA42464B46FDF7E4
:107F100041FC7BA3D3E9002380468946304639469D
:107F2000FDF738FC78A3D3E90023FDF781FA324648
:107F30003B46FDF72FFC76A3D3E90023FDF778FA43
:107F400032463B46FDF726FC02460B464046494674
:107F5000FDF76EFA4EF686334BF65102CFF6F97303
:107F6000C0F20602EB18521B1343002B06460F46C5
:107F700056DD00230022C3F6E07350465946FDF754
:107F800009FC52465B46FDF705FC80468946002CFD
:107F90006AD132463B46FDF74BFADDE90023FDF797
:107FA000F9FB02460B4640464946FDF73FFA0246BA
:107FB0000B4650465946FDF739FA68E70021002084
:107FC00000220023CCF25031FDF70EFD5FE7524650
:107FD0005B4650465946FDF7DDFB4FA3D3E900232E
:107FE00006460F4650465946FDF7D4FB0B46002186
:107FF0000246C3F6E0710020FDF718FA02460B4670
:1080000030463946FDF7C6FB06460F46002C40F0C9
:1080100093805046594632463B46FDF707FA36E70D
:10802000002C00F0AD802AA3D3E90023DDE9020192
:10803000FDF7B0FB32463B468046894650465946DE
:10804000FDF7F4F9DDE90023FDF7A4FB22A3D3E952
:10805000002304460D46DDE90201FDF79BFB0246C5
:108060000B46204629467EE019A3D3E90023DDE92B
:108070000201FDF78FFB3246CDE904013B46404645
:108080004946FDF7D5F9DDE90023FDF783FB12A38F
:10809000D3E9002304460D46DDE90201FDF77AFB32
:1080A00002460B4620462946FDF7C2F902460B461A
:1080B00040464946FDF7BAF952465B46FDF7B6F928
:1080C00002460B46DDE90401FDF7B0F9DFE600BF2B
:1080D0000000E0FE422EE63F763C7935EF39EA3D7E
:1080E00044523EDF12F1C23FDE03CB966446C73FE7
:1080F000599322942449D23F935555555555E53F00
:108100009FC678D0099AC33FAF788E1DC571CC3F0A
:1081100004FA97999999D93F555555555555D53FD5
:1081200002460B46FDF782F900220023FDF75CFCB6
:10813000ADE600200021AAE62046FDF7C5FA16A309
:10814000D3E9002304460D46FDF724FB14A3D3E92D
:1081500000238046894620462946FDF71BFB024640
:108160000B4630463946FDF761F952465B46FDF74E
:108170005DF902460B4640464946FDF757F986E64B
:1081800032463B4650465946FDF750F9DDE900239B
:10819000FDF700FB0BE700BF0000E0FE422EE63FCC
:1081A000763C7935EF39EA3D0B4661B1B1F1004FCC
:1081B00009D04FF6FF72A3F58011C7F6DF72914226
:1081C00005D8042070470028F3D10220704703F13E
:1081D000FE4101F570019142F3D94FF6FF72C0F2F2
:1081E0000F02934201D80320704703F100419142EE
:1081F000F9D90022C7F6F072934204D013F5801F1C
:1082000001D000207047D0F1010038BF0020704736
:108210000020704700210020C7F6F871704700BFAA
:1082200040F2F853C2F200031868704708B5062000
:1082300000F072F80120F0F7F9FC00BF0F2AF0B44B
:108240003AD941EA00039B0738D10C46034615464C
:108250002668103D1E6066685E60A6689E60E668DF
:108260001034DE6010330F2DF2D8A2F1100424F088
:108270000F0402F00F021034032A00EB0403214420
:1082800011D90E461D46144656F8047B043C032CB7
:1082900045F8047BF8D8141F24F00304043402F0DA
:1082A000030209191B192AB111F8014B013A03F80D
:1082B000014BF9D1F0BC70470346F4E70346F3E7FE
:1082C0001F2938B50C46054620D8D0F8DC229AB1D3
:1082D00052F8213083B1012B0CD0591C06D0002557
:1082E000204642F824509847284638BD162303609C
:1082F000012038BD002038BD284600F02BF822466A
:1083000001462846BDE8384000F010B81623036047
:108310004FF0FF3038BD00BF40F2F853C2F2000307
:108320001B6801461846FFF7CBBF00BF38B5084CA5
:1083300000230546084611462360F0F778FC431CED
:1083400000D038BD2368002BFBD02B6038BD00BFA8
:1083500028620020F0F76CBC50C3000088130000B6
:10836000018008080000000000000100000000007B
:1083700000000000C8000000EF8D2100B81E0500BD
:1083800000000000000000000000000000000000ED
:1083900000000000000000000000000000000000DD
:1083A0000000000000000000524F52000001065281
:1083B0004F4C000002064D5354000003024D56502E
:1083C00000000407534150000005074741500000DA
:1083D0000603535441500007035253415000080311
:1083E0005347500000090747475000000A03535401
:1083F0004750000B0352534750000C0352465300A2
:10840000000D0353494F00000E0747494F00000F6E
:108410000353414300001D0753434F00001E07470D
:10842000434F00001F0343434F0000200341434FCD
:108430000000270355463000004007554631000034
:1084400041075546320000420755463300004307B6
:10845000554634000044075546350000450755464B
:1084600036000046075546370000470752554E0074
:1084700000810553544F5000800042494E00008B4C
:1084800000000000000000000000000010000000DC
:10849000160000001B000000200000002300000068
:1084A000270000002A0000002D000000300000001E
:1084B00032000000350000003700000039000000E5
:1084C0003B0000003D0000004000000041000000B3
:1084D0004300000045000000470000004900000084
:1084E0004B0000004C0000004E0000005000000057
:1084F000510000005300000054000000560000002E
:1085000057000000590000005A0000005B00000006
:108510005D0000005E0000006000000061000000DF
:1085200062000000630000006500000066000000BB
:1085300067000000680000006A0000006B00000097
:108540006C0000006D0000006E0000007000000074
:108550007100000072000000730000007400000051
:108560007500000076000000770000007800000031
:10857000790000007A0000007B0000007C00000011
:108580007D0000007E0000008000000080000000F0
:1085900081000000820000008300000084000000D1
:1085A00085000000860000008700000088000000B1
:1085B000890000008A0000008B0000008C00000091
:1085C0008D0000008E0000008F0000009000000071
:1085D0009000000091000000920000009300000055
:1085E0009400000095000000960000009600000036
:1085F0009700000098000000990000009A00000019
:108600009B0000009B0000009C0000009D000000FB
:108610009E0000009F000000A0000000A0000000DD
:10862000A1000000A2000000A3000000A3000000C1
:10863000A4000000A5000000A6000000A7000000A4
:10864000A7000000A8000000A9000000AA00000088
:10865000AA000000AB000000AC000000AD0000006C
:10866000AD000000AE000000AF000000B000000050
:10867000B0000000B1000000B2000000B200000035
:10868000B3000000B4000000B5000000B500000019
:10869000B6000000B7000000B7000000B8000000FE
:1086A000B9000000B9000000BA000000BB000000E3
:1086B000BB000000BC000000BD000000BD000000C9
:1086C000BE000000BF000000C0000000C0000000AD
:1086D000C1000000C1000000C2000000C300000093
:1086E000C3000000C4000000C5000000C500000079
:1086F000C6000000C7000000C7000000C80000005E
:10870000C9000000C9000000CA000000CB00000042
:10871000CB000000CC000000CC000000CD00000029
:10872000CE000000CE000000CF000000D00000000E
:10873000D0000000D1000000D1000000D2000000F5
:10874000D3000000D3000000D4000000D4000000DB
:10875000D5000000D6000000D6000000D7000000C1
:10876000D7000000D8000000D9000000D9000000A8
:10877000DA000000DA000000DB000000DB0000008F
:10878000DC000000DD000000DD000000DE00000075
:10879000DE000000DF000000E0000000E00000005C
:1087A000E1000000E1000000E2000000E200000043
:1087B000E3000000E3000000E4000000E50000002A
:1087C000E5000000E6000000E6000000E700000011
:1087D000E7000000E8000000E8000000E9000000F9
:1087E000EA000000EA000000EB000000EB000000DF
:1087F000EC000000EC000000ED000000ED000000C7
:10880000EE000000EE000000EF000000F0000000AD
:10881000F0000000F1000000F1000000F200000094
:10882000F2000000F3000000F3000000F40000007C
:10883000F4000000F5000000F5000000F600000064
:10884000F6000000F7000000F7000000F80000004C
:10885000F8000000F9000000F9000000FA00000034
:10886000FA000000FB000000FB000000FC0000001C
:10887000FC000000FD000000FD000000FE00000004
:10888000FE000000FF00000001F0010002F0010006
:1088900004F0010005F0010007F0010008F00100FC
:1088A0000AF001000BF001000DF001000EF00100D4
:1088B00010EE010011EE010013EE010015EE0100B3
:1088C00016EE010018EE010019EE01001BEE01008A
:1088D0001CEC01001EEC01001FEC010021EC01006A
:1088E00022EC010024EA010025EA010027EA010048
:1088F00028EA01002AE801002BE801002DE8010028
:108900002EE8010030E6010031E6010033E6010007
:1089100034E4010036E4010037E4010039E20100EB
:108920003AE201003CE201003DE001003EE00100CE
:1089300040E0010041DE010043DE010044DC0100B3
:1089400046DC010047DC010049DA01004ADA010097
:108950004CD801004DD801004FD6010050D601007F
:1089600051D4010053D4010054D2010056D2010069
:1089700057D0010059D001005ACE01005BCE010052
:108980005DCC01005ECA010060CA010061C801003F
:1089900062C8010064C6010065C4010067C401002B
:1089A00068C2010069C201006BC001006CBE010019
:1089B0006DBE01006FBC010070BA010072B8010009
:1089C00073B8010074B6010076B4010077B40100F9
:1089D00078B201007AB001007BAE01007CAE0100EC
:1089E0007EAC01007FAA010080A8010081A80100DF
:1089F00083A6010084A4010085A2010087A00100D4
:108A0000889E0100899E01008A9C01008C9A0100C9
:108A10008D9801008E9601008F94010091920100C3
:108A20009292010093900100948E0100968C0100B7
:108A3000978A010098880100998601009A840100B4
:108A40009C8201009D8001009E7E01009F7C0100B0
:108A5000A07A0100A1780100A3760100A4740100AE
:108A6000A5720100A6700100A76E0100A86C0100AC
:108A7000A96A0100AA680100AC660100AD640100AA
:108A8000AE620100AF600100B05E0100B15C0100A8
:108A9000B25A0100B3580100B4540100B5520100AC
:108AA000B6500100B74E0100B84C0100B94A0100B0
:108AB000BA480100BB460100BC420100BD400100B4
:108AC000BE3E0100BF3C0100C03A0100C1380100B8
:108AD000C2340100C3320100C4300100C52E0100C0
:108AE000C62C0100C7280100C8260100C9240100C6
:108AF000C9220100CA1E0100CB1C0100CC1A0100D2
:108B0000CD180100CE140100CF120100CF100100DA
:108B1000D00E0100D10A0100D2080100D3060100E5
:108B2000D4020100D4000100D5FE0000D6FC0000F4
:108B3000D7F80000D7F60000D8F40000D9F0000004
:108B4000DAEE0000DAEC0000DBE80000DCE6000012
:108B5000DCE40000DDE00000DEDE0000DFDA000023
:108B6000DFD80000E0D60000E1D20000E1D0000034
:108B7000E2CE0000E2CA0000E3C80000E4C4000046
:108B8000E4C20000E5C00000E5BC0000E6BA000059
:108B9000E7B60000E7B40000E8B20000E8AE00006D
:108BA000E9AC0000E9A80000EAA60000EAA2000083
:108BB000EBA00000EB9E0000EC9A0000EC98000097
:108BC000ED940000ED920000EE8E0000EE8C0000AF
:108BD000EE880000EF860000EF820000F0800000C9
:108BE000F07C0000F07A0000F1780000F1740000E1
:108BF000F1720000F26E0000F26C0000F2680000FA
:108C0000F3660000F3620000F3600000F45C000013
:108C1000F45A0000F4560000F4540000F55000002F
:108C2000F54E0000F54A0000F5480000F64400004B
:108C3000F6420000F63E0000F63C0000F638000068
:108C4000F7360000F7320000F7300000F72C000084
:108C5000F72A0000F7260000F7220000F7200000A6
:108C6000F81C0000F81A0000F8160000F8140000C4
:108C7000F8100000F80E0000F80A0000F8080000E4
:108C8000F8040000F8020000F8020200F8040200F4
:108C9000F8080200F80A0200F80E0200F8100200BC
:108CA000F8140200F8160200F81A0200F81C02007C
:108CB000F7200200F7220200F7260200F72A02003E
:108CC000F72C0200F7300200F7320200F7360200FC
:108CD000F6380200F63C0200F63E0200F6420200C0
:108CE000F6440200F5480200F54A0200F54E020083
:108CF000F5500200F4540200F4560200F45A020047
:108D0000F45C0200F3600200F3620200F36602000A
:108D1000F2680200F26C0200F26E0200F1720200D0
:108D2000F1740200F1780200F07A0200F07C020097
:108D3000F0800200EF820200EF860200EE8802005F
:108D4000EE8C0200EE8E0200ED920200ED94020025
:108D5000EC980200EC9A0200EB9E0200EBA00200ED
:108D6000EAA20200EAA60200E9A80200E9AC0200B9
:108D7000E8AE0200E8B20200E7B40200E7B6020083
:108D8000E6BA0200E5BC0200E5C00200E4C202004F
:108D9000E4C40200E3C80200E2CA0200E2CE02001C
:108DA000E1D00200E1D20200E0D60200DFD80200EA
:108DB000DFDA0200DEDE0200DDE00200DCE40200B9
:108DC000DCE60200DBE80200DAEC0200DAEE020088
:108DD000D9F00200D8F40200D7F60200D7F802005A
:108DE000D6FC0200D5FE0200D4000300D40203002A
:108DF000D3060300D2080300D10A0300D00E0300FB
:108E0000CF100300CF120300CE140300CD180300CF
:108E1000CC1A0300CB1C0300CA1E0300C9220300A6
:108E2000C9240300C8260300C7280300C62C03007A
:108E3000C52E0300C4300300C3320300C234030054
:108E4000C1380300C03A0300BF3C0300BE3E03002C
:108E5000BD400300BC420300BB460300BA48030008
:108E6000B94A0300B84C0300B74E0300B6500300E4
:108E7000B5520300B4540300B3580300B25A0300C0
:108E8000B15C0300B05E0300AF600300AE6203009C
:108E9000AD640300AC660300AA680300A96A03007E
:108EA000A86C0300A76E0300A6700300A572030060
:108EB000A4740300A3760300A1780300A07A030042
:108EC0009F7C03009E7E03009D8003009C82030024
:108ED0009A8403009986030098880300978A030008
:108EE000968C0300948E03009390030092920300EB
:108EF000919203008F9403008E9603008D980300D7
:108F00008C9A03008A9C0300899E0300889E0300BC
:108F100087A0030085A2030084A4030083A60300A6
:108F200081A8030080A803007FAA03007EAC030091
:108F30007CAE03007BAE03007AB0030078B203007E
:108F400077B4030076B4030074B6030073B803006B
:108F500072B8030070BA03006FBC03006DBE03005B
:108F60006CBE03006BC0030069C2030068C203004B
:108F700067C4030065C4030064C6030062C803003D
:108F800061C8030060CA03005ECA03005DCC030031
:108F90005BCE03005ACE030059D0030057D0030024
:108FA00056D2030054D2030053D4030051D403001B
:108FB00050D603004FD603004DD803004CD8030011
:108FC0004ADA030049DA030047DC030046DC030009
:108FD00044DC030043DE030041DE030040E0030005
:108FE0003EE003003DE003003CE203003AE2030000
:108FF00039E2030037E4030036E4030034E40300FD
:1090000033E6030031E6030030E603002EE80300F8
:109010002DE803002BE803002AE8030028EA0300F8
:1090200027EA030025EA030024EA030022EC0300F8
:1090300021EC03001FEC03001EEC03001CEC0300FA
:109040001BEE030019EE030018EE030016EE0300FA
:1090500015EE030013EE030011EE030010EE030003
:109060000EF003000DF003000BF003000AF0030004
:1090700008F0030007F0030005F0030004F003000C
:1090800002F0030001F0030001F1030002F103000C
:1090900004F1030005F1030007F1030008F10300E8
:1090A0000AF103000BF103000DF103000EF10300C0
:1090B00010EF030011EF030013EF030015EF03009F
:1090C00016EF030018EF030019EF03001BEF030076
:1090D0001CED03001EED03001FED030021ED030056
:1090E00022ED030024EB030025EB030027EB030034
:1090F00028EB03002AE903002BE903002DE9030014
:109100002EE9030030E7030031E7030033E70300F3
:1091100034E5030036E5030037E5030039E30300D7
:109120003AE303003CE303003DE103003EE10300BA
:1091300040E1030041DF030043DF030044DD03009F
:1091400046DD030047DD030049DB03004ADB030083
:109150004CD903004DD903004FD7030050D703006B
:1091600051D5030053D5030054D3030056D3030055
:1091700057D1030059D103005ACF03005BCF03003E
:109180005DCD03005ECB030060CB030061C903002B
:1091900062C9030064C7030065C5030067C5030017
:1091A00068C3030069C303006BC103006CBF030005
:1091B0006DBF03006FBD030070BB030072B90300F5
:1091C00073B9030074B7030076B5030077B50300E5
:1091D00078B303007AB103007BAF03007CAF0300D8
:1091E0007EAD03007FAB030080A9030081A90300CB
:1091F00083A7030084A5030085A3030087A10300C0
:10920000889F0300899F03008A9D03008C9B0300B5
:109210008D9903008E9703008F95030091930300AF
:109220009293030093910300948F0300968D0300A3
:10923000978B030098890300998703009A850300A0
:109240009C8303009D8103009E7F03009F7D03009C
:10925000A07B0300A1790300A3770300A47503009A
:10926000A5730300A6710300A76F0300A86D030098
:10927000A96B0300AA690300AC670300AD65030096
:10928000AE630300AF610300B05F0300B15D030094
:10929000B25B0300B3590300B4550300B553030098
:1092A000B6510300B74F0300B84D0300B94B03009C
:1092B000BA490300BB470300BC430300BD410300A0
:1092C000BE3F0300BF3D0300C03B0300C1390300A4
:1092D000C2350300C3330300C4310300C52F0300AC
:1092E000C62D0300C7290300C8270300C9250300B2
:1092F000C9230300CA1F0300CB1D0300CC1B0300BE
:10930000CD190300CE150300CF130300CF110300C6
:10931000D00F0300D10B0300D2090300D3070300D1
:10932000D4030300D4010300D5FF0200D6FD0200E0
:10933000D7F90200D7F70200D8F50200D9F10200F0
:10934000DAEF0200DAED0200DBE90200DCE70200FE
:10935000DCE50200DDE10200DEDF0200DFDB02000F
:10936000DFD90200E0D70200E1D30200E1D1020020
:10937000E2CF0200E2CB0200E3C90200E4C5020032
:10938000E4C30200E5C10200E5BD0200E6BB020045
:10939000E7B70200E7B50200E8B30200E8AF020059
:1093A000E9AD0200E9A90200EAA70200EAA302006F
:1093B000EBA10200EB9F0200EC9B0200EC99020083
:1093C000ED950200ED930200EE8F0200EE8D02009B
:1093D000EE890200EF870200EF830200F0810200B5
:1093E000F07D0200F07B0200F1790200F1750200CD
:1093F000F1730200F26F0200F26D0200F2690200E6
:10940000F3670200F3630200F3610200F45D0200FF
:10941000F45B0200F4570200F4550200F55102001B
:10942000F54F0200F54B0200F5490200F645020037
:10943000F6430200F63F0200F63D0200F639020054
:10944000F7370200F7330200F7310200F72D020070
:10945000F72B0200F7270200F7230200F721020092
:10946000F81D0200F81B0200F8170200F8150200B0
:10947000F8110200F80F0200F80B0200F8090200D0
:10948000F8050200F8030200F8030000F8050000E8
:10949000F8090000F80B0000F80F0000F8110000B8
:1094A000F8150000F8170000F81B0000F81D000078
:1094B000F7210000F7230000F7270000F72B00003A
:1094C000F72D0000F7310000F7330000F7370000F8
:1094D000F6390000F63D0000F63F0000F6430000BC
:1094E000F6450000F5490000F54B0000F54F00007F
:1094F000F5510000F4550000F4570000F45B000043
:10950000F45D0000F3610000F3630000F367000006
:10951000F2690000F26D0000F26F0000F1730000CC
:10952000F1750000F1790000F07B0000F07D000093
:10953000F0810000EF830000EF870000EE8900005B
:10954000EE8D0000EE8F0000ED930000ED95000021
:10955000EC990000EC9B0000EB9F0000EBA10000E9
:10956000EAA30000EAA70000E9A90000E9AD0000B5
:10957000E8AF0000E8B30000E7B50000E7B700007F
:10958000E6BB0000E5BD0000E5C10000E4C300004B
:10959000E4C50000E3C90000E2CB0000E2CF000018
:1095A000E1D10000E1D30000E0D70000DFD90000E6
:1095B000DFDB0000DEDF0000DDE10000DCE50000B5
:1095C000DCE70000DBE90000DAED0000DAEF000084
:1095D000D9F10000D8F50000D7F70000D7F9000056
:1095E000D6FD0000D5FF0000D4010100D403010026
:1095F000D3070100D2090100D10B0100D00F0100F7
:10960000CF110100CF130100CE150100CD190100CB
:10961000CC1B0100CB1D0100CA1F0100C9230100A2
:10962000C9250100C8270100C7290100C62D010076
:10963000C52F0100C4310100C3330100C235010050
:10964000C1390100C03B0100BF3D0100BE3F010028
:10965000BD410100BC430100BB470100BA49010004
:10966000B94B0100B84D0100B74F0100B6510100E0
:10967000B5530100B4550100B3590100B25B0100BC
:10968000B15D0100B05F0100AF610100AE63010098
:10969000AD650100AC670100AA690100A96B01007A
:1096A000A86D0100A76F0100A6710100A57301005C
:1096B000A4750100A3770100A1790100A07B01003E
:1096C0009F7D01009E7F01009D8101009C83010020
:1096D0009A8501009987010098890100978B010004
:1096E000968D0100948F01009391010092930100E7
:1096F000919301008F9501008E9701008D990100D3
:109700008C9B01008A9D0100899F0100889F0100B8
:1097100087A1010085A3010084A5010083A70100A2
:1097200081A9010080A901007FAB01007EAD01008D
:109730007CAF01007BAF01007AB1010078B301007A
:1097400077B5010076B5010074B7010073B9010067
:1097500072B9010070BB01006FBD01006DBF010057
:109760006CBF01006BC1010069C3010068C3010047
:1097700067C5010065C5010064C7010062C9010039
:1097800061C9010060CB01005ECB01005DCD01002D
:109790005BCF01005ACF010059D1010057D1010020
:1097A00056D3010054D3010053D5010051D5010017
:1097B00050D701004FD701004DD901004CD901000D
:1097C0004ADB010049DB010047DD010046DD010005
:1097D00044DD010043DF010041DF010040E1010001
:1097E0003EE101003DE101003CE301003AE30100FC
:1097F00039E3010037E5010036E5010034E50100F9
:1098000033E7010031E7010030E701002EE90100F4
:109810002DE901002BE901002AE9010028EB0100F4
:1098200027EB010025EB010024EB010022ED0100F4
:1098300021ED01001FED01001EED01001CED0100F6
:109840001BEF010019EF010018EF010016EF0100F6
:1098500015EF010013EF010011EF010010EF0100FF
:109860000EF101000DF101000BF101000AF1010000
:1098700008F1010007F1010005F1010004F1010008
:1098800002F1010001F10100E0C0020060C003002C
:1098900060C10300E0C10200E0C1000060C101003E
:1098A00060C00100E0C00000E0C0020060C0030032
:1098B00060C10300E0C10200E0C1000060C101001E
:1098C00060C00100E0C00000B4690100B46801009C
:1098D000B4680300B4690300B4690100B46801000E
:1098E000B4680300B4690300B4690100B4680100FE
:1098F000B4680300B4690300B4690100B4680100EE
:10990000B4680300B46903000201023133313156F7
:109910003130370056435020496E7465726661637A
:10992000650056435020436F6E66696700544D438F
:1099300031333131005472696E616D6963204D6F4E
:1099400074696F6E20436F6E74726F6C00544D4378
:109950004D2D3133313120287669727475616C2058
:10996000434F4D29004142530052454C00434F4F55
:1099700052440053544152540053544F50005354D6
:10998000415455530000000043000000D001002066
:1099900000202020202020202020282828282820BF
:1099A00020202020202020202020202020202020B7
:1099B000208810101010101010101010101010101F
:1099C000100404040404040404040410101010100F
:1099D00010104141414141410101010101010101D9
:1099E000010101010101010101010101101010102B
:1099F00010104242424242420202020202020202AB
:109A000002020202020202020202020210101010FE
:109A10002000000000000000000000000000000026
:109A20000000000000000000000000000000000036
:109A30000000000000000000000000000000000026
:109A40000000000000000000000000000000000016
:109A50000000000000000000000000000000000006
:109A600000000000000000000000000000000000F6
:109A700000000000000000000000000000000000E6
:109A800000000000000000000000000000000000D6
:109A9000000000006C6F670000000000F8B500BF18
:109AA000F8BC08BC9E467047F8B500BFF8BC08BCBF
:049AB0009E46704717
:109AB400A1B20181B0B0AE010000000008B1018183
:109AC400B0B000840000000008B10181B0B000848F
:109AD4000000000008B10181B0B000840000000063
:109AE40054C8FF7FB03784807CC8FF7FAB08B18047
:109AF400A0C8FF7F010000001CC9FF7FB0A902803D
:109B0400DCC9FF7FB0B0A8802CCAFF7FA4FFFF7F11
:109B1400F8CAFF7FA908B18020CBFF7F01000000B5
:109B24009CCBFF7FB0AF0A80A8CEFF7F010000006E
:109B3400ACCEFF7FAE3F278058D2FF7F01000000EC
:109B440054D2FF7FAB10B280ACD2FF7F0100000083
:109B5400B8D2FF7FA908B180ECD2FF7F01000000DA
:109B6400F8D2FF7F58FFFF7F00D3FF7FAB26B28080
:109B74006CD3FF7F0100000044D5FF7FB0A80380B1
:109B840058D5FF7F0100000054D5FF7FB0AD04809D
:109B940018D8FF7FB0A8038038D8FF7F2CFFFF7F41
:109BA4003CD8FF7F30FFFF7F48D8FF7F01000000D3
:109BB40054D8FF7FB0B0A78014DBFF7FB0B0A6807D
:089BC400A4DDFF7F0100000099
:089BCC00997C0108AD8100083D
:049BD400898100087B
:109BD8000B990108000102000008000001000000C4
:109BE800020000000000000000000000000000006B
